:02000004080CE6
:100000005071002079CF0C0881CF0C0883CF0C08E9
:1000100085CF0C0887CF0C0889CF0C0800000000A2
:100020000000000000000000000000008BCF0C0862
:100030008DCF0C08000000008FCF0C085D0F0C085E
:1000400093CF0C0893CF0C0893CF0C0893CF0C08D8
:1000500093CF0C0893CF0C0893CF0C0893CF0C08C8
:1000600093CF0C0893CF0C0893CF0C0893CF0C08B8
:10007000632A0C0893CF0C084D2A0C081D740C0839
:1000800093CF0C08912A0C0893CF0C0893CF0C083F
:1000900093CF0C0893CF0C0893CF0C0893CF0C0888
:1000A00097390C0893CF0C0893CF0C085F680C08A5
:1000B00093CF0C0893CF0C0893CF0C0893CF0C0868
:1000C00093CF0C0893CF0C0893CF0C0893CF0C0858
:1000D00093CF0C085B0B0C0893CF0C08850B0C0816
:1000E00093CF0C0893CF0C0893CF0C0893CF0C0838
:1000F000BF0F0C0893CF0C088B250C0893CF0C086E
:1001000093CF0C0893CF0C08156C0C0893CF0C08F8
:1001100053190C0893CF0C08B5380C08CB380C08D1
:1001200093CF0C0893CF0C0893CF0C0893CF0C08F7
:1001300093CF0C0893CF0C0893CF0C0827480C08DA
:100140003D460C0893CF0C0841470C0893CF0C0890
:1001500093CF0C0893CF0C08F1730C0893CF0C08C5
:1001600093CF0C0893CF0C0893CF0C0893CF0C08B7
:1001700093CF0C0893CF0C0893CF0C0893CF0C08A7
:1001800093CF0C0800F002F800F04AF80AA090E8BB
:10019000000C82448344AAF10107DA4501D100F042
:1001A0003FF8AFF2090EBAE80F0013F0010F18BFC5
:1001B000FB1A43F001031847A8010100C801010020
:1001C0000A4410F8014B14F00F0508BF10F8015B4A
:1001D000240908BF10F8014B6D1E05D010F8013B33
:1001E0006D1E01F8013BF9D1641E03D0641E01F8B5
:1001F000015BFBD19142E4D370470000002300244F
:1002000000250026103A28BF78C1FBD8520728BF26
:1002100030C148BF0B6070471FB51FBD10B510BD82
:1002200010F045F81146FFF7F7FF00F079F810F0ED
:1002300063F803B4FFF7F2FF03BC10F067F80000A7
:100240007FB501205D490870481E00785C49087040
:1002500001205C490870002048705B49087006F076
:10026000BEFE68460CF0AFFF4FF47A720198B0FB07
:10027000F2F1B1F1807F00D31DE021F07F40401EFC
:100280004FF0E022506150170F22002807DA1307C1
:100290001D0E4E4B00F00F04241F1D5503E01307E5
:1002A0001C0E4B4B1C5400BF00204FF0E02290610D
:1002B0000720106100BF07F06FFD00F0C8F800F0E4
:1002C00057FD00F0CDFE02F025FC01F01FFA01F011
:1002D00094FA03F0A3FA06F0A3FE06F0A0FD03F0E3
:1002E000CFF80AF049FE0120364908700020487016
:1002F000022138480DF071FA7FBD10B536A00CF020
:1003000009FA00214FF000600DF055F94FF000613F
:10031000086880F3088800BF34480068804710BD33
:100320002648C01C006831490860FFF789FF01209A
:100330002F49087000202F49087001202E490870AD
:1003400001F052F901202D490870012404E0002039
:100350002B490855601C84B240F226208442F6DD09
:1003600028A00CF0FEFC00202749087027490870DF
:100370002749087027A00CF0CDF91EE01F4800782F
:1003800008B9FFF7BAFF274800884CF2503188427D
:1003900002DB00202349088001F09DF901F09BF960
:1003A00021480088062807D10020154908701E49F9
:1003B00008800CF031FA00BF00BFDFE701FF012029
:1003C00059000020C70000205800002018ED00E070
:1003D00000E400E00010024052657475726E2074F3
:1003E0006F204D61696E4170700D00005C0000204F
:1003F0005500002056000020570000205400002027
:100400000A0B00202A310D0053000020500000206C
:1004100051000020454F424420697320616C697689
:10042000650D00000A0000201C00002000BFBFF383
:100430004F8FFC48006800F4E060FB490843001D52
:10044000F8490860BFF34F8F00BF00BFFEE700B55B
:1004500087B0012108460CF025FF012102200CF095
:1004600021FF012108200CF01DFF012110200CF0BC
:100470005DFF012188040CF048FF07220921EB48A9
:100480000DF0C1F907220A21E8480DF0BCF9072256
:100490000B21E6480DF0B7F907220C21E3480DF0D7
:1004A000B2F907220A21E2480DF0ADF907220B212B
:1004B000DF480DF0A8F907220B21DE480DF0A3F963
:1004C00007220C21DB480DF09EF94FF400700190DB
:1004D00002208DF808008DF8090000208DF80A0030
:1004E00001208DF80B0001A9D0480DF009F94FF457
:1004F0008060019001A9CE480DF002F94FF48060B0
:10050000019001A9C9480DF0FBF84FF4006001907B
:1005100001A9C7480DF0F4F84FF40060019001A95B
:10052000C2480DF0EDF84FF40060019001A9C148F8
:100530000DF0E6F84FF48050019001A9BB480DF092
:10054000DFF84FF48050019001A9BA480DF0D8F8B7
:100550004FF4E13003904FF48050ADF810000020CC
:10056000ADF812004FF48060ADF814000C20ADF827
:1005700016008001ADF8180003A9AF480DF0C6F9C8
:1005800003A9AE480DF0C2F90121AB480DF046FABF
:100590000121AA480DF042FA012240F22551A64855
:1005A0000DF048FA012240F22551A4480DF042FA1C
:1005B00007B000BD10B50446A148007802280BD151
:1005C00000BF80219D480DF004FB0028F9D0A1B2A6
:1005D0009A480DF090FA0AE000BF802196480DF08D
:1005E000F8FA0028F9D0A1B293480DF084FA10BDB2
:1005F00070B504462A2C03D100209249088070BDB2
:100600000D2C75D1002190488E4A128881540246E3
:100610008C480088401C11548A480088801C115462
:1006200010460078322804D0362874D0392873D187
:1006300040E28548407830380A286ED2DFE800F082
:1006400005A6B0BABBBCBDBEBFC300207E490870C2
:1006500008468078382861D009DCA0F130000828ED
:1006600022D2DFE800F01522912D3846505146285D
:1006700069D006DC392858D0412857D0422813D1F8
:1006800059E0612853D0622856D066287CD15BE0BF
:1006900006F048FD05462A20FFF78CFF28460CF09F
:1006A00072FB0D20FFF786FF6EE02A20FFF782FF26
:1006B000664800880CF092FA0D20FFF77BFF63E09C
:1006C0002A20FFF777FF624800880CF087FA0D2098
:1006D000FFF770FF58E000F0FEFF2A20FFF76AFFE7
:1006E0005C4800880CF07AFA0D20FFF763FF4BE0BE
:1006F00029E259A00CF035FB5B480CF032FB0D20D1
:10070000FFF758FF40E03FE02A20FFF753FF0D209E
:10071000FFF750FF38E06BE014E267E02A20FFF7B4
:1007200049FF0D20FFF746FF2EE02DE000BF4FA050
:100730000CF017FB28E000BF4EA00CF012FB4FA0FE
:100740000CF00FFB20E000BF2A20FFF733FF00244E
:1007500006E04DA1095D48B2FFF72CFF601CC4B252
:100760000B2CF6DD2020FFF725FF002406E049A131
:10077000095D48B2FFF71EFF601CC4B2082CF6DD0D
:100780000D20FFF717FF00BF00BF38E72E48807825
:10079000322800D100BF00BF02204149088025E077
:1007A00029488078302800D100BF00BF02203C4992
:1007B00008801BE000BF00BF00BF00BF00BF0220D9
:1007C0003749088012E020488078392809D12A204A
:1007D000FFF7F0FE0220334908800D20FFF7EAFE04
:1007E00000BF00BF02202E49088000BF00BF06E7FF
:1007F0001548407830380A2870D2DFE800F005EE5E
:10080000EDECEBEAE9E8E7E600200F49087008465E
:100810008078392870D04EDCA0F1300009286AD2E7
:1008200042E000000CED00E00000FA05000002408C
:1008300000040240000C024000100140004800404B
:10084000590000201A0000200A0B00200800002098
:100850000E000020120000204275696C6420746153
:10086000726765743A2000001A030D082A43445049
:100870002B0D00002A5553420D0000002A426C75D2
:1008800065746F6F74680D004170722031342032CE
:100890003031350031353A33363A35350000000015
:1008A0001C00002020000020DFE800F01927E232C1
:1008B0003D3E42464C0061284CD008DC41284AD0DD
:1008C000422853D043286AD0462814D174E06228C5
:1008D0004BD0632862D06628F7D16CE0E8E006F0E0
:1008E00021FC05462A20FFF765FE28460CF04BFA4E
:1008F0000D20FFF75FFEBBE028E02A20FFF75AFE3D
:10090000B04800880CF06AF90D20FFF753FEAFE005
:100910002A20FFF74FFEAC4800880CF05FF90D204D
:10092000FFF748FEA4E0A3E00120A84908809FE06B
:100930000120A74908809BE00120A6490880A6491C
:10094000087095E00120A549088091E00120A449A4
:1009500008808DE000BF2A20FFF72CFEA1480CF094
:1009600012FA0D20FFF726FE82E000BF2A20FFF7D3
:1009700021FE9D48C078432803D09B48C078632857
:1009800004D19A4800880CF029F903E098480088BF
:100990000CF024F90D20FFF70DFE69E000BF0AF00E
:1009A000E7FA2A20FFF706FE01200CF017F90D20C8
:1009B000FFF700FE5CE000BF8E48007800284CD0B6
:1009C0008C480078102847D208E05EE059E057E0F4
:1009D00055E053E051E04FE04DE04BE0DFE800F040
:1009E0003C080C3C103C1438181C2024282C3034B3
:1009F00081A00CF0B6F92FE084A00CF0B2F92BE046
:100A000088A00CF0AEF927E08DA00CF0AAF923E045
:100A100092A00CF0A6F91FE097A00CF0A2F91BE041
:100A20009CA00CF09EF917E0A1A00CF09AF913E03D
:100A3000A6A00CF096F90FE0ABA00CF092F90BE039
:100A4000B0A00CF08EF907E0B5A00CF08AF903E035
:100A5000BAA00CF086F900BF09E02A20FFF7AAFD32
:100A6000BA4800780CF0BAF80D20FFF7A3FD00BFDC
:100A700000BFC4E500BF00BF00BF00BF00BF00BF94
:100A800000BF0620B249088012E057488078392814
:100A900009D12A20FFF78EFD0220AE4908800D20E3
:100AA000FFF788FD00BF00BF0620A949088000BFEE
:100AB00000BFA4E54C48407830380A2840D2DFE82F
:100AC00000F00520212223242526272B002046493B
:100AD00008700846807830380A2810D2DFE800F025
:100AE00005060708090A0B0C0D0E08E007E006E0F2
:100AF00005E004E003E002E001E000E000BF00BF29
:100B00007DE500BF00BF00BF00BF00BF00BF00BF4A
:100B100009208F49088013E03348807839280AD1AA
:100B20008DA00CF01EF906F060FB05468B49681C91
:100B300006F09DFB00BF00BF09208549088000BF6B
:100B400000BF5CE55BE5864801880088401C844A5C
:100B500010802548445400BF51E510B540F225519E
:100B600080480DF083F808217E480DF032F87D486A
:100B70000CF0C5FFC4B201207B4908702046FFF786
:100B800037FD10BD10B540F2255178480DF06EF8D4
:100B9000082176480DF01DF874480CF0B0FFC4B27F
:100BA0000220714908702046FFF722FD10BD10B5E4
:100BB00007F013FA10B107F026FA08B9012010BDAA
:100BC0000020FCE7080000200E0000203800002074
:100BD0002C000020360000205300002032000020AE
:100BE0002E00002065004D000A0B002004FF0F08B6
:100BF00000FF0F08510000202A49534F203931349B
:100C0000312D32202843415242290D002A49534FA9
:100C10002031343233302D3420284B5732303030AD
:100C2000290D00002A49534F203531392D34202811
:100C30005341452D4A313835302050574D290D004C
:100C40002A49534F203531392D3420285341452D21
:100C50004A3138353020565057290D002A49534F14
:100C60002031353736352D34202843414E2031315F
:100C70002D323530290D00002A49534F20313537A8
:100C800036352D34202843414E2031312D3530303A
:100C9000290D00002A49534F2031353736352D3480
:100CA000202843414E2032392D323530290D0000A5
:100CB0002A49534F2031353736352D3420284341CA
:100CC0004E2032392D353030290D00002A49534F3E
:100CD0002032373134352D34202843414E203131F4
:100CE0002D323530290D00002A49534F203237313B
:100CF00034352D34202843414E2031312D353030CC
:100D0000290D00002A49534F2032373134352D3414
:100D1000202843414E2032392D323530290D000034
:100D20002A49534F2032373134352D34202843415E
:100D30004E2032392D353030290D00002A534145DF
:100D4000204A313933392D32310D00005000002056
:100D50001C00002020000020A40D00002D040C0821
:100D60001A000020001001405900002000480040F7
:100D700008B54FF440700CF0E7FB25208DF800001B
:100D80000C208DF8010000208DF8020001208DF864
:100D9000030068460CF0DDFB27208DF800000C20D6
:100DA0008DF8010000208DF8020001208DF803006D
:100DB00068460CF0CEFB34208DF800000A208DF838
:100DC000010000208DF8020001208DF80300684624
:100DD0000CF0BFFB2E208DF8000008208DF80100DC
:100DE00000208DF8020001208DF8030068460CF009
:100DF000B0FB1B208DF8000008208DF801000020BA
:100E00008DF8020001208DF8030068460CF0A1FB6C
:100E100032208DF8000008208DF8010000208DF8A8
:100E2000020001208DF8030068460CF092FB0E20B2
:100E30008DF8000009208DF8010000208DF80200D7
:100E400001208DF8030068460CF083FB0C208DF820
:100E5000000009208DF8010000208DF8020001201B
:100E60008DF8030068460CF074FB11208DF800002B
:100E700009208DF8010000208DF8020001208DF876
:100E8000030068460CF065FB40208DF800000B2045
:100E90008DF8010000208DF8020001208DF803007C
:100EA00068460CF056FB42208DF800000B208DF8B0
:100EB000010000208DF8020001208DF80300684633
:100EC0000CF047FB3F208DF800000B208DF801004F
:100ED00000208DF8020001208DF8030068460CF018
:100EE00038FB36208DF8000005208DF80100002029
:100EF0008DF8020001208DF8030068460CF029FBF4
:100F000037208DF8000004208DF8010000208DF8B6
:100F1000020001208DF8030068460CF01AFB18202F
:100F20008DF8000003208DF8010000208DF80200EC
:100F300001208DF8030068460CF00BFB2C208DF887
:100F400000000F208DF8010000208DF80200012024
:100F50008DF8030068460CF0FCFA08BD10B5374860
:100F60000068401C3549086035480088401C3449F9
:100F7000088034480088401C324908803248008884
:100F8000002805DD30480088401E2F49088002E017
:100F9000002005F03DFF294800680A21B0FBF1F26E
:100FA00001FB120030B929480088401C27490880FD
:100FB00002F0FDFB06F013F906F01AF910BD10B5AA
:100FC000012123480DF028FE38B1012120480DF001
:100FD0002CFE01211E480DF03CFE01211D480DF0A4
:100FE0001BFE38B31C481D49097830F81100002851
:100FF0000BDD194A194B1B7832F813105032174B7E
:101000001B7832F8130005F057FF14480078401C95
:101010001249087008460078272801DD0020087072
:1010200002F03BFB01210B480DF0FFFD01210948B7
:101030000DF00FFE10BD01480068704760000020F1
:10104000000000204E000020080100200A000020BF
:1010500000180040001C0040142B00205800002005
:1010600000B587B0012108460CF01CF901212020B1
:101070000CF018F9012108030CF058F9052211466B
:10108000F7480CF0C0FB05220621F5480CF0BBFB2D
:1010900005220721F2480CF0B6FB20200590022023
:1010A0008DF818008DF8190000208DF81A008DF8C1
:1010B0001B0005A9EA480CF023FB4020059005A978
:1010C000E7480CF01DFB8020059005A9E4480CF0D2
:1010D00017FB0220059001208DF8180002208DF8E2
:1010E000190000208DF81A008DF81B0005A9DD48B5
:1010F0000CF006FB0420059005A9DA480CF000FB73
:101100000120059005A9D7480CF0FAFA0721D54827
:101110000CF061FB4FF44040ADF800004FF48270DA
:10112000ADF802000020ADF80400ADF80600ADF8FF
:1011300008004FF40070ADF80A003820ADF80C003C
:101140000020ADF80E00ADF810006946C6480CF05E
:10115000C3FD0121C4480CF0C2FE07B000BD2DE95B
:10116000F04105460F46164633463A462946BFA08B
:101170000BF0D0FA072D06D1C748007840F01000D8
:10118000C5490870AFE10020C4490870C44908701F
:10119000C148007800F01000BF4908700A2D3FD206
:1011A000DFE805F005300D1422293E3E371B0020F4
:1011B000BA490870BA490870B749087034E0B748AE
:1011C000007840F02000B54908702DE0B348007861
:1011D00040F00200B149087026E0B048007840F0C5
:1011E0000200AE4908701FE0AC48007840F00400EF
:1011F000AA49087018E0A948007840F00800A749FB
:10120000087011E0A548007840F00100A34908707B
:101210000AE0A248007840F01000A049087003E0FE
:1012200000209E49087000BF00BF102F77D2DFE872
:1012300007F096080910171819252C3844555C69D1
:1012400077898DE09648007840F00800944908704E
:1012500086E09348007840F00200914908707FE0F2
:101260007EE07DE08E48007840F002008C490870F6
:101270000846007840F00800087071E0884800785F
:1012800040F00100864908706AE08548007840F027
:101290000100834908700846007840F0100008708B
:1012A0005EE07F48007840F001007D490870084604
:1012B000007840F00200087052E07948007840F071
:1012C0000100774908700846007840F00200087075
:1012D0000846007840F01000087041E06F48007840
:1012E00040F040006D4908703AE06C48007840F0EA
:1012F00040006A4908706A48007840F02000684958
:1013000008702DE06548007840F04000634908709F
:101310006348007840F004006149087020E01EE056
:101320005E48007840F040005C4908705C480078F6
:1013300040F004005A4908700846007840F0200048
:1013400008700DE05548007840F04000534908709F
:101350005348007840F001005149087000E000BF98
:1013600000BF102E7AD2DFE806F0BC08091017186B
:1013700019262D3A46585F6C9DAFB3E04648007879
:1013800040F0020044490870ACE04548007840F065
:10139000800043490870A5E0A4E0A3E0404800783D
:1013A00040F080003E4908703B48007840F0020061
:1013B0003949087096E03A48007840F040003849D2
:1013C00008708FE03648007840F0400034490870DB
:1013D0003148007840F004002F49087082E030481E
:1013E000007840F040002E4908700846007840F030
:1013F0008000087076E02A48007840F040002849D4
:1014000008700846007840F0800008702248007894
:1014100040F004002049087064E02048007840F063
:1014200080001E4908705DE01C48007840F0800094
:101430001A4908701848007840F0080016490870EA
:1014400050E01648007840F08000144908701248B7
:10145000007840F001001049087043E041E00000CE
:101460000000024000140240003001405365745FE8
:1014700052656C61793A20636F6D547970652825E7
:1014800064292C2070696E48282564292C207069F5
:101490006E4C282564290D006600002064000020A1
:1014A000650000204A48007840F0800048490870F4
:1014B0004848007840F00100464908700846007826
:1014C00040F0080008700DE04148007840F08000CE
:1014D0003F4908704048007840F040003E4908709D
:1014E00000E000BF00BF00BF3C480088001B05288B
:1014F000FAD3384801783A480CF02EFD02213948D9
:101500000CF06BF93548048800BF34480088001B94
:101510000528FAD33148048800BF022130480CF076
:101520006EFD20B92D480088001B3228F5D32B48CA
:101530000488048800BF022129480CF060FD20B90E
:1015400026480088001B3228F5D32448048800BFB1
:1015500022480088001B0528FAD31F48017820483C
:101560000CF0FAFC1D48048800BF02211C480CF056
:1015700046FD20B919480088001B3228F5D31748CA
:10158000048800BF15480088001B0528FAD31048BE
:10159000017813480CF0E0FC1048048800BF0221D9
:1015A0000F480CF02CFD20B90C480088001B322895
:1015B000F5D30A48048800BF08480088001B0528A6
:1015C000FAD3022107480CF006F9BDE8F0810000CB
:1015D000640000206600002065000020000000205C
:1015E000003001400014024010B51C4800881C491E
:1015F000088001201B49088000F06DF800201A497E
:1016000008801A4908801A49088000F064F8002010
:10161000184908801849088018490880012018498D
:1016200008800020174908801749088000F053F807
:101630000020104908800420144908700BF018FAA3
:1016400000F049F801201249087000201149087083
:10165000114908700349088010BD000000FF0B0805
:10166000080000200E0000201800002022000020AA
:10167000160000200A0000200C000020200000209E
:10168000120000201C0000201E000020520000203C
:1016900055000020560000205700002010B57D2086
:1016A0000BF0AFFC20B10EA00BF034F80BF02DFFC7
:1016B00045F255500EF0E2FC02200EF0E2FC4FF431
:1016C00048600EF0E1FC00200EF0D8FC0EF0DFFCCC
:1016D0000EF0E2FC10BD10B50EF0D9FC10BD0000FC
:1016E00053797374656D2072657374617274656487
:1016F0002064756520746F205761746368646F6738
:10170000207265736574210D000000001CB5012175
:1017100008200BF0C7FD012110200BF0C3FD0121B3
:1017200020200BF0BFFD012140200BF0BBFD4FF44A
:101730004040009001208DF8040002208DF8050043
:1017400000208DF806008DF807006946FE480BF072
:10175000D7FF4FF4A050009001208DF80400022024
:101760008DF8050000208DF806008DF80700694609
:10177000F6480BF0C5FF4FF4E050009001208DF8C3
:10178000040002208DF8050000208DF806008DF879
:1017900007006946EE480BF0B3FF4FF4004000909D
:1017A00001208DF806006946E9480BF0A9FF0120E9
:1017B00000906946E7480BF0A3FF0220009000204C
:1017C0008DF8040002208DF8050000208DF8060039
:1017D0008DF807006946DF480BF092FF4FF4004197
:1017E000DB480BF0FAFF0121DA480BF0F6FF4FF46B
:1017F0008061D7480BF0EFFF1CBD00B587B0012119
:1018000008460BF04FFD012108200BF04BFD012194
:1018100040200BF047FD012110200BF043FD01217A
:10182000C8040BF072FD012148040BF06EFD01218C
:1018300020200BF07BFD08220021C7480BF0E3FFBE
:1018400008220121C4480BF0DEFF07220521BE4813
:101850000BF0D9FF07220621BB480BF0D4FF08226A
:101860000921BC480BF0CFFF08220E21B9480BF02C
:10187000CAFF03220621B5480BF0C5FF01200190E5
:1018800002208DF808008DF8090000208DF80A006C
:1018900001208DF80B0001A9AF480BF031FF0220A9
:1018A000019001A9AC480BF02BFF202001900220F1
:1018B0008DF808008DF8090000208DF80A0001203D
:1018C0008DF80B0001A9A0480BF01AFF40200190F1
:1018D00001A99D480BF014FF4FF400700190022005
:1018E0008DF808008DF8090000208DF80A0001200D
:1018F0008DF80B0001A997480BF002FF4FF48040D0
:10190000019001A993480BF0FBFE4020019001A932
:101910008E480BF0F5FE42F6A00003900020ADF8D3
:101920001000ADF81200ADF814000C20ADF8160050
:101930000020ADF8180003A988480BF0E7FF03A9C1
:1019400087480BF0E3FF03A986480BF0DFFF07B0E1
:1019500000BD10B540F2255181480CF087F9804850
:101960000CF0CDF88049814A128821F812007F4896
:101970000088B0F57A7F04DA7C480088401C7B49F7
:10198000088010BD7FB506460C461546FFF735FFAB
:10199000002173480CF042F8002170480CF03EF82A
:1019A000002170480CF03AF80096092C03D14FF44E
:1019B0008050ADF80400082C02D10020ADF80400DE
:1019C0000020ADF806000DB9ADF80800012D0DD1CD
:1019D0004FF4C060ADF80800072C02D10020ADF82C
:1019E0000400082C02D16002ADF80400022D0CD1D5
:1019F0006802ADF80800072C02D10020ADF8040001
:101A0000082C02D16002ADF804000C20ADF80A00E9
:101A10000020ADF80C00694651480BF077FF01211A
:101A20004F480BF0FBFF7FBD10B5044601F0DDFF12
:101A300010BD1CB50446072C30D2DFE804F004309A
:101A40004374C1D4E7004FF4806141480BF0C5FEF8
:101A50004FF480613D480BF0C0FE4FF480513B488D
:101A60000BF0BBFE012240F225513D480BF0E2FF96
:101A7000002240F2255139480BF0DCFF002240F2F1
:101A8000255138480BF0D6FF4FF480612F480BF0FA
:101A9000A4FE4FF480512D480BF09FFEF6E000228B
:101AA00040F225512E480BF0C5FF012240F225518E
:101AB0002A480BF0BFFF002240F2255129480BF0C5
:101AC000B9FFE3E04FF4806120480BF086FE4FF44D
:101AD00080511E480BF081FE4FF400611C480BF052
:101AE0007AFE4FF480511A480BF077FE4FF4804194
:101AF00015480BF070FE4FF4004113480BF06BFEDD
:101B0000002240F2255116480BF094FF002240F2CB
:101B1000255112480BF08EFF012240F22551114849
:101B20000BF088FFB2E001208DF8040002208DF850
:101B3000050000208DF8060001208DF807000090B8
:101B40006946054814E00000000C02400010024005
:101B5000001402400018024000000240001401403E
:101B6000004C0040004400400806002022000020F5
:101B70000BF0C6FD0121F7480BF02DFE4FF48061FC
:101B8000F5480BF02AFE4FF48061F4480BF025FE77
:101B90004FF48051F1480BF020FE012240F2255114
:101BA000EF480BF047FF002240F22551ED480BF0C3
:101BB00041FF002240F22551EB480BF03BFF65E06E
:101BC000012240F22551E6480BF034FF002240F29A
:101BD0002551E4480BF02EFF002240F22551E24847
:101BE0000BF028FF52E0012240F22551DC480BF0B7
:101BF00021FF002240F22551DA480BF01BFF0022A2
:101C000040F22551D8480BF015FF3FE00021D6489F
:101C10000BF004FF012108200BF044FB2020009072
:101C200001208DF8040002208DF8050000208DF8B9
:101C3000060001208DF807006946CC480BF060FDD6
:101C40004FF48061C5480BF0C8FD4FF48051C34884
:101C50000BF0C3FD2021C5480BF0BDFD4FF4004142
:101C6000C2480BF0B8FD002240F22551BC480BF0F1
:101C7000E1FE002240F22551BA480BF0DBFE0022C3
:101C800040F22551B8480BF0D5FE00BF00BF1CBD87
:101C90007CB505460E46144601208DF8040002204E
:101CA0008DF8050000208DF8060001208DF8070052
:101CB000601E84B2042D04D0052D1ED0082D57D1EE
:101CC0003AE0012000900121A2480BF084FD694612
:101CD000A0480BF015FD01200AF0E5FD01219D480B
:101CE0000BF07BFD30460AF0DEFD012199480BF038
:101CF00072FD20460AF0D7FD3EE04FF48040009090
:101D000001469B480BF067FD694699480BF0F8FCCB
:101D100001200AF0C8FD4FF4804195480BF05DFDAD
:101D200030460AF0C0FD4FF4804191480BF053FD5E
:101D300020460AF0B8FD1FE02020009020218B48AB
:101D40000BF049FD694689480BF0DAFC01200AF0E6
:101D5000AAFD202185480BF040FD30460AF0A3FD86
:101D6000202182480BF037FD20460AF09CFD03E05D
:101D700080A00AF0F6FF00BF00BF7CBD2DE9F04F48
:101D80008BB08046894616469A46149C002500274B
:101D9000AB4641F2883090FBFAF07B490880274639
:101DA0007A480680072E02D14FF0800B06E0082EFD
:101DB00002D14FF4807B01E04FF0000B03E0781E6E
:101DC0000740681C85B2002FF9D1284605EBD07179
:101DD0004910A5EB41018DB2B9F1000F06D0B9F160
:101DE000010F06D0B9F1020F1FD110E0684804803E
:101DF0001CE066480088401C6449088025B904EB53
:101E00000B006349088001E0614804800EE05F48F0
:101E10000088401C5D49088025B104EB0B005C493B
:101E2000088001E05A48048000E000BF00BFB8F11C
:101E3000040F06D0B8F1050F66D0B8F1080F65D1D0
:101E400063E0012108460BF02DFA012108200BF078
:101E50005CFA012120200BF025FA4E480CF078FCAA
:101E6000012009908DF8280002208DF8290000201B
:101E70008DF82A008DF82B00012136480BF0ABFCC1
:101E800009A934480BF03CFC0A200AF00CFD42F68C
:101E9000E060ADF818000020ADF81A004FF6FF70B2
:101EA00007900020ADF8200006A93A480CF093F9FD
:101EB0000020ADF804004FF6FF70039001A93548EB
:101EC0000CF0BBF933480CF09EFE2F4909880844FA
:101ED000014600902F480CF07EFE08212D480CF0A2
:101EE000B8FE012208212B480CF019FC0122082120
:101EF00028480CF0DEFD012116480BF06EFC012194
:101F000024480CF0F2FB02E001E000E000BF00BF5B
:101F100000202149088000BF1F4801881B48008815
:101F2000401C8142F8DB0A200AF0BDFC0BB0BDE882
:101F3000F08F10B5FFF7CFFB1748017801208840DC
:101F400013490988084020B1012102480BF043FCE5
:101F500028E023E00000024000140240001002408C
:101F6000004C00400014014000440040000C0240BE
:101F7000001802404E6F7420696D706C656D656E5F
:101F8000746564210D0000006E0000206C000020CC
:101F900068000020000C00406A0000200121164863
:101FA0000BF01BFC15480088401C144908800846AB
:101FB00000881349098888420EDD01210E480BF084
:101FC0000AFC002208210F480CF0A9FB002208217E
:101FD0000C480CF06EFD0DE00A480CF00EFE0A49AC
:101FE00009884418214607480CF0F5FD08210548EA
:101FF0000CF02FFE10BD0000000002406A0000201F
:102000006C000020000C00406E000020F0B5A1B074
:102010000120F84908600020F74908601020F749BE
:1020200008600020F6490860F64908604820F64933
:1020300008706B204870002507E00020F34941F844
:102040002500F34941F825006D1C202DF5D3012012
:10205000EE490860EE49086000250026012443E0AF
:10206000C6F107010120884000F0F507EFB1601EBE
:10207000E64951F82000083041F82400601EE44988
:1020800051F82000C01C41F82400641C601EDF4988
:1020900051F82000103041F82400601EDC4951F84E
:1020A0002000153041F824001CE0601ED74951F88B
:1020B0002000103041F82400601ED54951F820005E
:1020C0000B3041F82400641C601ED04951F82000F8
:1020D000083041F82400601ECD4951F820000D3031
:1020E00041F82400761C641C082EB9D30121042079
:1020F0000BF0D8F8012108200BF0D4F801210420BE
:102100000BF003F9012102200BF010F90121480521
:102110000BF0C8F803220621BE480BF074FB022224
:102120000D21BD480BF06FFB4FF400501F900220B3
:102130008DF880008DF8810000208DF882008DF8E8
:1021400083001FA9B4480BF0DBFA4FF40051B248EA
:102150000BF043FB40201F901FA9AE480BF0D0FAB4
:10216000AE480CF0F5FAAE480CF0F2FA0020AB499C
:10217000103108804FF6FF71A8480CF02AFD3C2072
:10218000ADF800000020ADF802004FF6FF7001909E
:102190000020ADF808006946A0480CF01CF8782033
:1021A000ADF8000069469E480CF015F83020ADF8F7
:1021B00068000120ADF86A004FF6FF701C90002007
:1021C000ADF874001AA995480CF06AF800220E21A7
:1021D00092480CF0AFFA0122910290480CF0AFFA4D
:1021E0004FF0806003908D48383004904020069076
:1021F000002008904FF48060099080000A908000D1
:102200000B9000200C904FF480300D9000200E9029
:102210000F901090119003A982480CF0B1FE01229A
:10222000102180480CF0FDFE0020ADF85C000A2073
:10223000ADF85E000120ADF860000020ADF862004E
:10224000ADF8640017A976480CF0A5F90020ADF8A8
:1022500048004FF6FF70149012A971480CF020F856
:10226000012202216E480CF05AFA012204216C4826
:102270000CF055FA01216A480CF037FA012021B020
:10228000F0BDF0B502460B46FF210026154625E0BD
:102290004FF0000C80271BE02888384058B101F02F
:1022A000800008B1012400E01C24012000EB410063
:1022B0006040C1B207E0002401F0800000B11D249D
:1022C00084EA4100C1B20CF1010000F0FF0C7F1064
:1022D000BCF1080FE0DB701CC6B2AD1C9E42D7DB20
:1022E000C843C0B2F0BD2DE9FF4F8BB0824601203C
:1022F0004049086080460020414908604A4908601A
:102300000AF0FF060C9880B2ADF804000D9880B278
:10231000ADF806000E9880B2ADF80800189880B2AB
:10232000ADF80A00199880B2ADF80C001A9880B286
:10233000ADF80E001B9880B2ADF810001C9880B26A
:10234000ADF812001D9880B2ADF814001E9880B24E
:10235000ADF816001F9880B2ADF81800002404E014
:102360000020324921F81400641CFF2CF8D93146B2
:1023700001A8FFF786FF814601A820F81690701C7F
:10238000C6B2C8202A490860002485E0002700253D
:102390007EE001A830F81400C7F107020121914046
:1023A00000EA010BBBF1000F44D0B8F1000F10D0D0
:1023B000012000EBC4002844401E1D4951F82000B4
:1023C0007E30012101EBC4012944194A42F8210061
:1023D00054E0012000EBC4002844401E144951F889
:1023E00020004030012101EBC4012944104A42F889
:1023F000210043E0A0000020940000207C00002089
:10240000840000208800002070000020441B002071
:10241000C41B002000080240000C024000080040DD
:102420000004014058600240800000204419002050
:10243000340D0020B8F1000F10D0012000EBC400D3
:102440002844401EFA4951F820004030012101EB98
:10245000C4012944F64A42F821000FE0012000EBB4
:10246000C4002844401EF24951F820007E3001216A
:1024700001EBC4012944EE4A42F821007F1C6D1C87
:10248000B8F1000F02D04FF0000801E04FF0010852
:10249000082FFFF47EAF641CB442FFF477AF012134
:1024A00001EB0610401EE24951F820006430012281
:1024B00002EB0611DE4A42F821000521DD480CF04E
:1024C00088FBDB48DC494866022000EBC600C86593
:1024D0000121D94858300CF08FFD0120D7490880E0
:1024E0000020D74908800121D2480CF06CFB00BFC6
:1024F000D44800680028FBD10120D249086001219E
:10250000CC480CF0F2F830200FB0BDE8F08F10B5D9
:1025100001200022CC4B1A80CC4B1A8000BF002235
:10252000CB4B1A80421ECB4B995C012805D1CAB215
:10253000482A02D00122C54B1A80022805D1CAB20E
:102540006B2A02D00122C14B1A80CAB2C24B1B882F
:102550000344C14C24F81320401C0E2804DABF4A5F
:102560001278921C9042DADBB84A128862B940F2C3
:10257000E732B94B1B880344B74C24F8132022469A
:102580001288024423461A8010BD2DE9F04186B01E
:102590000221B3480CF04CFB012870D14021B14816
:1025A0000BF0FFF808B1012000E000200746AC481E
:1025B0000CF01DFB84B20FB1E01F84B2A14800688B
:1025C000012852D19F49086004F58C71A4480CF091
:1025D00000FB9B480088012841DDA3480068251ABC
:1025E00097480088401E924951F82010944800886E
:1025F000801E8F4A52F820000E1A91480088801ED3
:102600009A4941F820608E480088401E41F82050C9
:1026100006F10F00854202D81E38A8421FD91020AB
:1026200088490860002183480CF05FF80021824847
:1026300058300CF0E1FC40217E480CF02AF93020A3
:10264000ADF804000120ADF806004FF6FF700390CE
:102650000020ADF8100001A976480BF021FE784863
:102660000088401C7649088019E1764800680428F3
:1026700006D104F58C717A480CF0ABFA0FE11EE13B
:1026800070480068022803D06E48006800287DD199
:1026900075480088201A7649764A127821F8120087
:1026A00074490878C11700EB5171C910724A117052
:1026B000002F4ED16E486F49097830F8110060281C
:1026C00019DC644811460978405C11460978694A6A
:1026D0001278A2EBC101C1F1070201219140084328
:1026E000C1B25C48644A1278815462480078401C48
:1026F0006049087068E05E485E49097830F811006A
:10270000A32819DC53485C490978405C5A49097888
:10271000584A1278A2EBC101C1F107026FF0010122
:10272000914008404B49544A1278885451480078E7
:10273000401C5049087047E004F5967148480CF079
:1027400048FA00204B4908704C4908704A49087003
:102750003AE047484749097830F8110060281BDC07
:102760003C4845490978405C43490978414A127818
:10277000A2EBC101C1F107026FF0010191400840D5
:1027800034493D4A127888543A4800E040E00078E5
:10279000401C3849087017E02E4837490978405CDA
:1027A00035490978334A1278A2EBC101C1F1070219
:1027B00001219140084327492F4A127888542D4817
:1027C0000078401C2B4908701E480068022804D17C
:1027D00004F1C80122480CF0FCF9022019490860F4
:1027E0002448007809285AD10846007800F00100F2
:1027F000E0B9002022490870224908601548007895
:102800002149097888424AD101201E49086046E0E2
:102810000C480068082839D111480CF0E8F900F19B
:10282000C80841460E480CF0D4F938E037E0000003
:10283000340D0020000800400060024078000020B5
:10284000B00000207C000020440000200C0000208C
:10285000480000203419002058010020A700002063
:10286000000401400008024094000020441C0020A5
:1028700044190020A4000020A6000020A50000208C
:1028800098000020B4000020700000208D480CF05B
:10289000AEF900F5967841468A480CF09AF98A48D4
:1028A0000460042187480CF0D4F9012204218548F2
:1028B0000BF035FF022183480CF0CBF900BF042157
:1028C00080480CF0B5F9012821D1002204217D486F
:1028D0000BF025FF04217B480CF0BBF97B48006816
:1028E000012815D177480CF085F900F164073946C5
:1028F00074480CF06EF91020744908600421714886
:102900000CF0A7F9012204216E480BF008FF9AE0B1
:102910006E480068042828D110206C490860694876
:102920000CF065F900F59677394666480CF051F9D8
:102930000122042163480BF0F2FE6548007830B1B3
:102940006448007818B10120634908607BE0614861
:10295000007830B100205F49087002205E490860AD
:1029600071E001205C4908606DE058480068022869
:1029700031D154480CF03BF900F58C773946514879
:102980000CF027F9012204214E480BF0C8FE082064
:102990004E4908604F480078012854D100204D4925
:1029A000087005214D480CF014F94D484D49486612
:1029B0000720C86501214B4858300CF01DFB012051
:1029C00049490880012145480CF0FDF801214348A0
:1029D0000BF08BFE37E03D480068082811D110202D
:1029E0003A49086037480CF002F900F59677394605
:1029F00034480CF0EEF80122042132480BF08FFE2F
:102A000021E000203149086038480078002817DDAF
:102A100030480078A0B936480068012810D1334802
:102A20000078344908700020334908703349087031
:102A30002E4908700120324908800020234908608F
:102A400000202B49086006B0BDE8F08110B52D4983
:102A5000244858300CF0A4FB002120480BF045FE20
:102A600010BD10B528491F4828300CF099FB2748A5
:102A7000008838B900214FF080400BF036FE04206A
:102A80001249086018480088401E1749088010BD88
:102A900010B51F491348A0300CF082FB1248008883
:102AA00038B900214FF080400BF01FFE0420074989
:102AB000086016480088401E1449088010BD024670
:102AC0000120704700040140940000207C00002099
:102AD00034190020980000208400002000080040E5
:102AE000340D00200060024078000020A600002085
:102AF000B4000020A7000020A4000020A5000020B2
:102B00004400002000800018008800107A00002097
:102B10000080202000B58BB0012108020AF006FCDD
:102B200007A80CF0A2FB07A80CF069FB01A80CF0A9
:102B3000A2FB00208DF80900019001A930480CF09B
:102B40006FFB01212E480CF0A0FB012240F2052171
:102B50002B480CF0B0FB0BB000BD10B5014600BF18
:102B600041F6797301FB03F266205043254CB0FB1C
:102B7000F4F290B210BD2DE9F04705460C4616461A
:102B80000027B946B846BA460023012229461C4808
:102B90000CF0F9FB00BF14E019480CF09CFB00BFDF
:102BA000022117480CF02EFD0028F9D014480CF033
:102BB00046FC30441FFA80F908EB09001FFA80F840
:102BC0007F1C601EB842E7DA98FBF4F01FFA80FA27
:102BD0005046FFF7C2FFBDE8F08710B52C220A214E
:102BE0000846FFF7C8FF04466E2C01DA012010BD2D
:102BF000A02C03DDD22C01DA0120F8E70020F6E753
:102C0000002001408096980010B50024FD4800780F
:102C1000FC494978884227D0FA48007800F0010042
:102C200018B3F848007800F07200F0B91E20F64999
:102C3000088000BF04E006222046641CF3490A54C1
:102C4000282CF8DB002405E00F222046641CEF4905
:102C500028310A54282CF7DB04F0C1F904F0C6F936
:102C6000E8480078E7494870A5E3E648007800F0B6
:102C70000300032826D1E348007800F0700008BB69
:102C80000120E34908801E20DF490880002404E079
:102C900003222046641CDD490A54282CF8DB00245A
:102CA00005E00F222046641CD84928310A54282CFC
:102CB000F7DB04F094F904F099F9D2480078D1498F
:102CC000487078E3CF48007800F0430043282FD1C4
:102CD000CC48007800F0200050BBFF20CA49088093
:102CE000002404E002222046641CC8490A54282C0F
:102CF000F8DB002411E008222046641CC349283177
:102D00000A5404222046641C0A5402222046641CF1
:102D10000A5401222046641C0A54282CEBDB04F0E0
:102D20005EF904F063F9B7480078B649487042E3A9
:102D3000B448007800F0410041285BD1B1480078E8
:102D400000F02200002855D1FF20AF490880002460
:102D500004E002222046641CAC490A54282CF8DB0B
:102D6000002411E008222046641CA84928310A5496
:102D700004222046641C0A5402222046641C0A5481
:102D800001222046641C0A54282CEBDB002400207E
:102D90009E490875032048750F219C4880F83D1016
:102DA00000209A4988750320C8750F21974880F83C
:102DB0003F10002095490876032048760F2193485C
:102DC00080F841100020914988760320C8760F21B1
:102DD0008E4880F8431000208C49087704F0FFF8F3
:102DE00004F004F900208B49087086480078854972
:102DF0004870E0E28348007800F0130013283BD1CC
:102E00008048007800F06000002835D14FF47A70D7
:102E10007D49088000241AE002222046641C7B4978
:102E20000A542046641C0A542046641C0A54204656
:102E3000641C0A5403222046641C0A542046641C65
:102E40000A542046641C0A542046641C0A54282C48
:102E5000E2DB002405E00F222046641C6B49283188
:102E60000A54282CF7DB04F0BAF804F0BFF86548E0
:102E70000078644948709EE26248007800F03100B2
:102E8000312843D15F48007800F0420000283DD14E
:102E9000002404E002222046641C5C490A54282CC9
:102EA000F8DB002405E00F222046641C5749283136
:102EB0000A54282CF7DB0020544948700120887000
:102EC0000020C8700120087100204871012088711D
:102ED0000020C87101200872002048720875032084
:102EE000487588750020C87508760320487688766E
:102EF0000020C87604F041F804F060F8002045494D
:102F00000870404800783F49487054E23D480078D6
:102F100000F0610061287FD13A48007800F012008B
:102F20000028F8D1FF2038490880002404E002225C
:102F30002046641C35490A54282CF8DB002411E093
:102F400008222046641C314928310A5404222046B4
:102F5000641C0A5402222046641C0A5401222046A2
:102F6000641C0A54282CEBDB0024002027494870FD
:102F7000012088700F21254880F82A10002023495D
:102F8000C870012008710F21204880F82C10002003
:102F90001E494871012088710F211C4880F82E10AD
:102FA00000201A49C871012008720F21174880F8C3
:102FB00030100020154948720875032048750F210C
:102FC000124880F83D100020104988750320C8750C
:102FD0000F210E4880F83F1000200C49087603208E
:102FE00048760F21094880F841100020074988766B
:102FF0000320C8760F21054880F8431000200349BC
:1030000008770AE0C7000020C40000204420002008
:1030100028000020580000200BE003F0AEFF03F072
:10302000E5FF0020FC490870FC480078FB49487027
:10303000C1E1FA48007800F01100112831D1F748B9
:10304000007800F0620060BB002404E00222204609
:10305000641CF3490A54282CF8DB002405E00F22F5
:103060002046641CEE4928310A54282CF7DB002046
:10307000EB4908750320487588750020C8750876E7
:103080000320487688760020C87603F097FF03F087
:10309000A6FF0020E0490870E0480078DF4948704A
:1030A00089E1DE48007800F02100212837D1DB4893
:1030B000007800F0520088BB002404E0062220467D
:1030C000641CD7490A54282CF8DB002405E00F22A1
:1030D0002046641CD24928310A54282CF7DB0020F2
:1030E000CF494870012088700020C8700120087105
:1030F00000204871012088710020C87101200872E9
:103100000020487203F039FF03F070FF0020C2492D
:103110000870C2480078C14948704CE1FFE7BF48D9
:10312000007800F03100312837D1BC48007800F039
:10313000420088BB002404E002222046641CB849F7
:103140000A54282CF8DB002405E00F222046641CDA
:10315000B34928310A54282CF7DB0020B0494870C5
:10316000012088700020C87001200871002048717B
:10317000012088710020C871012008720020487267
:1031800003F0FBFE03F032FF0020A3490870A348C0
:103190000078A24948700EE1FFE7A048007800F0EF
:1031A0003300732847D100241AE002222046641C11
:1031B0009B490A542046641C0A542046641C0A5445
:1031C0002046641C0A5403222046641C0A542046EC
:1031D000641C0A542046641C0A542046641C0A5489
:1031E000282CE2DB002405E00F222046641C8C49D9
:1031F00028310A54282CF7DB002089494870012027
:1032000088700020C87001200871002048710120DA
:1032100088710020C871012008720020487203F0F4
:10322000ACFE03F0E3FE00207B4908707B48007889
:103230007A494870BFE07948007800F0630063285D
:103240005DD17648007800F01000E8BBFF2075499A
:103250000880002404E002222046641C70490A54BD
:10326000282CF8DB002413E008222046641C6C495B
:1032700028310A5404222046641C0A5402222046A3
:10328000641C0A5401222146641C654828304254BB
:10329000282CE9DB002062494870012088700F214A
:1032A0005F4880F82A1000205D49C870012008712D
:1032B0000F215B4880F82C100020594948710120EB
:1032C00088710F21564800E019E080F82E10002088
:1032D0005349C871012008720F21514880F83010FD
:1032E00000204F49487203F048FE03F07FFE0020A3
:1032F0004949087049480078484948705BE04748A8
:10330000007800F02300232837D14448007800F0EB
:10331000500088BB002404E003222046641C40497E
:103320000A54282CF8DB002405E00F222046641CF8
:103330003B4928310A54282CF7DB002038494870D3
:10334000012088700020C870012008710020487199
:10335000012088710020C871012008720020487285
:1033600003F00BFE03F042FE00202B4908702B48AF
:1033700000782A4948701EE0FFE7002404E000229C
:103380002046641C26490A54282CF8DB002405E05A
:103390000F222046641C224928310A54282CF7DBCE
:1033A00003F01DFE03F022FE00201B4908701B489D
:1033B00000781A49487010BD10B5044604F00800A2
:1033C00028B14FF4007118480AF005FA04E04FF4F0
:1033D000007115480AF001FA04F0040020B104213C
:1033E00012480AF0F8F903E0042110480AF0F5F950
:1033F00004F0020020B108210C480AF0ECF903E0C7
:1034000008210A480AF0E9F904F0010080B110210E
:1034100006480AF0E0F90FE058000020C70000203D
:1034200044200020C400002000040240001002409C
:103430001021E6480AF0D1F910BDE5480078704740
:10344000E3490870704710B5E24C2080E24C2280BE
:10345000E24C218010BD10B504462146E0480BF037
:10346000BAFB10BD10B504462146DD480BF0B5FB94
:1034700010BD10B504462146D9480BF0AAFB10BD7B
:1034800010B588B000240020D6490880D1490880B2
:10349000D5490880D1490880D4490880CE490880A0
:1034A0001E20D34908800020C9490870012102204C
:1034B00009F02BFF02220721CE480AF0A4F90222CC
:1034C0000021CD480AF09FF902220121CA480AF0E2
:1034D0009AF9CA480068CA49B0FBF1F0401E84B2AC
:1034E0004FF47A700690ADF814400020ADF81C003F
:1034F000ADF8160005A9BA480AF06DFE6020ADF8D7
:1035000000000120ADF8020000200290ADF80C0090
:103510006946B3480AF0C4FE0821B1480BF00DFA21
:10352000002002906946AE480AF0FFFE0821AC4830
:103530000BF00FFA002002906946A9480AF038FF04
:103540000821A7480BF00DFA0121A5480BF0CDF892
:1035500008B010BD10B54FF48061AA480AF021F9F7
:1035600001280DD1C102A7480AF01BF9012807D193
:103570000103A4480AF015F9012801D1002010BD6B
:103580004FF480619F480AF00CF968B94FF400616C
:103590009C480AF006F9012806D1010399480AF06F
:1035A00000F9012800D1EAE74FF4806195480AF05C
:1035B000F8F801280DD1C10292480AF0F2F840B99A
:1035C0004FF480518F480AF0ECF8012801D1022015
:1035D000D5E74FF480618B480AF0E3F801280CD15D
:1035E000C10288480AF0DDF8012806D101038548A8
:1035F0000AF0D7F808B90320C1E74FF48061814889
:103600000AF0CFF868B94FF400617E480AF0C9F8B3
:10361000012806D101037B480AF0C3F808B9042049
:10362000ADE70020ABE710B5FFF794FF052832D2D5
:10363000DFE800F0030B141E270000206549088016
:10364000664908806449088025E064206149088053
:10365000002062490880604908801CE000205D4924
:10366000088064205D49088000205B49088012E0E2
:10367000002058490880594908806420564908802C
:1036800009E06420534908800020544908806420E0
:103690005149088000BF00BF10BD10B5FDF787FA83
:1036A00030B15948007840F002005749087005E0F1
:1036B0005548007820F0020053490870FFF78DFA52
:1036C00030B15148007840F020004F49087005E0C3
:1036D0004D48007820F020004B4908704B48007896
:1036E00030B14948007840F010004749087005E0C3
:1036F0004548007820F0100043490870444800789D
:1037000030B14148007840F001003F49087005E0C1
:103710003D48007820F001003B490870FFF774FA3B
:103720003C483D490978405C072837D2DFE800F083
:10373000040A11181F262E00002211461046FFF71A
:1037400082FE2BE0002211464FF47A70FFF77BFED9
:1037500024E000224FF47A711046FFF774FE1DE05A
:103760004FF47A7200210846FFF76DFE16E04FF421
:103770007A7200211046FFF766FE0FE000224FF438
:103780007A714FF42F70FFF75EFE07E04FF4167268
:103790004FF47A711046FFF756FE00BF00BF1D4977
:1037A00028311D4A1278885CFFF706FE10BD10B55F
:1037B00008480088FFF75DFE08480088FFF752FEC2
:1037C00005480088FFF747FE10BD000000100240CA
:1037D000C6000020BE000020C2000020C000002063
:1037E00000040040B8000020BA000020BC00002007
:1037F000C4000020000802400004024044010020F0
:1038000080841E0000180240C700002057000020DE
:1038100055000020442000205800002010B5012150
:10382000102009F072FD01221821A2480AF0FFFFC2
:103830007F21A0480BF0C9F900219E480BF0C3F985
:10384000012211469B480AF06AFF0121202009F05D
:103850005CFD01224FF4C06197480AF0E8FF4FF683
:10386000FF7195480BF0B1F9002193480BF0ABF9CB
:103870000122114690480AF052FF0121802009F0F0
:1038800044FD012211028D480AF0D1FF45F6323184
:103890008A480BF09AF945F6323188480BF093F9D3
:1038A0000122114685480AF03AFF012183480AF0B7
:1038B0001CFF10BD10B582480088401C804908805C
:1038C00001217C480BF0C5F910BD10B57D4800788A
:1038D00008B9012000E000207A49087001217648EB
:1038E0000BF0B7F910BD2DE9FF410025002600249B
:1038F0000027684609F067FC002173480AF08EF83B
:10390000002172480AF08AF8002171480AF086F80E
:1039100000207049087070490880039E6F48058830
:1039200013E0FDF7D8FE6D480088401B40F6C41137
:10393000884201D2012000E0002030B90120664910
:103940000880002004B0BDE8F081624800780528B6
:10395000E7DB6348008962490988401A87B2310170
:1039600060480068401C7843B1FBF0F400205949DE
:1039700008705B490880088100215B480AF0B5FEA9
:1039800021465AA008F0C6FE002208212046FDF775
:10399000F9FF20B2D6E710B5022153480BF048F9E1
:1039A000A0B1022150480BF054F94A48007804288D
:1039B0000CDC4D480BF01BF94949464A127821F8B6
:1039C000120044480078401C4249087004214648CF
:1039D0000BF02EF940B149480088401C4749088047
:1039E000042141480BF035F910BD00B589B0012123
:1039F000102009F057FC0121202009F053FC01217F
:103A0000080409F093FC032205213D4809F0FBFE60
:103A10002020079002208DF820008DF82100002042
:103A20008DF822008DF8230007A9354809F068FEBB
:103A30002D480AF08DFE00202B4908824FF6FF71B9
:103A400029480BF0C6F82748008880B2ADF804007A
:103A50000020ADF806004FF6FF7002900020ADF890
:103A60000C0001A920480AF0B6FB0020ADF81000B8
:103A7000ADF812000120ADF814000020ADF81600DA
:103A8000ADF8180004A918480AF085FD022116486F
:103A90000BF0DFF80122022113480AF040FE012258
:103AA000002111480BF005F801210F480AF01DFE16
:103AB00009B000BD0010004000140040001C004090
:103AC000D400002057000020004C004000140140AA
:103AD00000440040CC0000200C000020000000202A
:103AE00094200020D0000020004001404261756415
:103AF000726174653A2025640D00000026000020E4
:103B000000100240F0B589B005460F460020FE497E
:103B1000087000244EE0002004EB8401FB4A42F8C8
:103B2000210004EB840102EB8101486004EB840175
:103B300002EB8101087204EB840102EB81014872FF
:103B400004EB840102EB8101887204EB8401F04AEA
:103B500042F8210004EB840102EB8101486004EB90
:103B6000840102EB8101087204EB840102EB810104
:103B7000487204EB840102EB8101887204EB84013A
:103B800002EB8101C874002610E0002104EB8400E0
:103B9000DE4A02EB80000B30815504EB8400DC4AE6
:103BA00002EB80000B308155701CC6B2082EECDB96
:103BB000601CC4B20F2CAEDB0121022009F072FBA5
:103BC0004FF44050079000208DF8200002208DF81F
:103BD000210000208DF8220001208DF8230007A984
:103BE000CC4809F08DFD6020079002208DF8200060
:103BF0008DF8210000208DF8220001208DF823008F
:103C000007A9C44809F07CFD09220521C14809F033
:103C1000FAFD09220621BF4809F0F5FD01214FF008
:103C2000C06009F072FBBC480BF010FD04A80BF05B
:103C300031FE0A200BF03EFE00208DF816008DF8B4
:103C400017008DF818008DF819008DF81A00012062
:103C50008DF81B0000208DF8120043F60E6085429F
:103C600012D1AEA008F056FD2846B04908800020C9
:103C70008DF8130004208DF8140003208DF8150032
:103C80005A20ADF810006DE043F60960854212D16C
:103C9000A7A008F03FFD2846A449088000208DF821
:103CA000130005208DF8140002208DF815003C202B
:103CB000ADF8100056E043F60360854212D1A0A093
:103CC00008F028FD28469949088000208DF8130047
:103CD00005208DF8140002208DF815001820ADF88D
:103CE00010003FE043F60160854212D198A008F031
:103CF00011FD28468D49088000208DF8130005200D
:103D00008DF8140002208DF815000C20ADF810007D
:103D100028E0B5F5785F13D191A008F0FBFC4FF4D3
:103D200078508249088000208DF8130005208DF816
:103D3000140002208DF815000620ADF8100011E0E7
:103D40008BA008F0E7FC22207849088000208DF83D
:103D5000130006208DF8140003208DF815001A209A
:103D6000ADF8100004A96C480BF089FC0B208DF80D
:103D70000A0001208DF80B000021654801774FF4FF
:103D8000FD606349486100208DF80C00ADF800002B
:103D9000084640694FF6FF7101EA4010ADF8020095
:103DA0000020ADF80400ADF80600ADF808000120D1
:103DB0008DF80D0068460BF0ECFC0C208DF80A0025
:103DC00040F2E970524988620846806A4FF6FF71F6
:103DD00001EA4010ADF8020068460BF0DAFC0D2055
:103DE0008DF80A0040F2EA704949C8630846C06B82
:103DF0004FF6FF7101EA4010ADF8020068460BF083
:103E0000C8FC0E208DF80A0040F2EB7040490865AE
:103E10000846006D4FF6FF7101EA4010ADF8020050
:103E200068460BF0B6FC0F208DF80A0040F2EC70EB
:103E3000374948660846406E4FF6FF7101EA401068
:103E4000ADF8020068460BF0A4FC10208DF80A00C3
:103E500040F2ED702E4988670846806F4FF6FF717B
:103E600001EA4010ADF8020068460BF092FC112008
:103E70008DF80A0040F2EE702549C1F88C00084622
:103E8000D0F88C004FF6FF7101EA4010ADF8020047
:103E900068460BF07EFC12208DF80A0040F2EF70AD
:103EA0001B49C1F8A0000846D0F8A0004FF6FF71EA
:103EB00001EA4010ADF8020068460BF06AFC1820D9
:103EC0008DF80A0000208DF80B000421104880F8BE
:103ED00020112B49C0F81C112A482B4908600120E9
:103EE0008DF80C000A48D0F81C01C0F34F30ADF833
:103EF00000000748D0F81C014FF6FF7101EAC0002E
:103F0000001DADF8020041E0D8000020CC210020C7
:103F1000A0200020000402400068004043414E3AC7
:103F20002033336B6269740D00000000F000002044
:103F300043414E3A2035306B6269740D0000000039
:103F400043414E3A203132356B6269740D000000F6
:103F500043414E3A203235306B6269740D000000E7
:103F600043414E3A203530306B6269740D000000D9
:103F700043414E3A2039356B6269740D00000000F0
:103F800000F1DA1800FFFF1FE4000020F948006884
:103F9000C0F34F30ADF80400F648006801EAC000F5
:103FA000001DADF806000020ADF8080001208DF8D6
:103FB0000D0068460BF0EDFB0FB1EF4807600122E2
:103FC0000221EE480BF08EFC01220821EB480BF099
:103FD00089FC0122D103E9480BF084FC0122D102C3
:103FE000E6480BF07FFC01221102E4480BF07AFC5A
:103FF00001221146E1480BF075FC09B0F0BDF0B5A7
:1040000085B005460F460120DD49087000244EE0CA
:10401000002004EB8401DB4A42F8210004EB840118
:1040200002EB8101486004EB840102EB810108721C
:1040300004EB840102EB8101487204EB840102EB82
:104040008101887204EB8401CF4A42F8210004EB1D
:10405000840102EB8101486004EB840102EB8101E1
:10406000087204EB840102EB8101487204EB8401C5
:1040700002EB8101887204EB840102EB8101C874B8
:10408000002610E0002104EB8400BE4A02EB800011
:104090000B30815504EB8400BB4A02EB80000B30EF
:1040A0008155701CC6B2082EECDB601CC4B20F2C0C
:1040B000AEDB0121022009F0F5F860200390022018
:1040C0008DF810008DF8110000208DF812000120ED
:1040D0008DF8130003A9AD4809F012FB012102205D
:1040E00009F0E0F86020039000208DF81000022015
:1040F0008DF8110000208DF8120001208DF81300BA
:1041000003A9A24809F0FCFA4FF4405003900220A2
:104110008DF810008DF8110000208DF8120001209C
:104120008DF8130003A9994809F0EAFA09220C2135
:10413000964809F068FB09220D21944809F063FBB9
:1041400001214FF0C06009F0E0F88C480BF07EFAD6
:1041500068460BF09FFB0A200BF0ACFB00208DF8AB
:10416000060001208DF8070000208DF808008DF86A
:1041700009008DF80A0001208DF80B0000208DF851
:10418000020043F60E6085420CD100208DF803003A
:1041900004208DF8040003208DF805005A20ADF8A6
:1041A00000004EE043F6096085420CD100208DF8F6
:1041B000030005208DF8040002208DF805003C2046
:1041C000ADF800003DE043F6036085420CD10020CD
:1041D0008DF8030005208DF8040002208DF80500FD
:1041E0001820ADF800002CE043F6016085420CD1A8
:1041F00000208DF8030005208DF8040002208DF8C2
:1042000005000C20ADF800001BE0B5F5785F0CD17F
:1042100000208DF8030005208DF8040002208DF8A1
:1042200005000620ADF800000BE000208DF803002B
:1042300006208DF8040003208DF805001A20ADF843
:10424000000069464D480BF01AFA0FB1504807605C
:104250000122022149480BF045FB01220821474871
:104260000BF040FB0122D10344480BF03BFB012241
:10427000D10242480BF036FB012211023F480BF0FD
:1042800031FB05B0F0BD7FB505460C46207800F047
:104290000800E0B3207800F0040078B10421681E23
:1042A00000EB8000374A02EB80000172681E00EBD1
:1042B000800002EB8000616841600DE00021681E13
:1042C00000EB80002F4A02EB80000172681E00EBB9
:1042D0008000616842F8201000260CE004F108001C
:1042E000815D681E00EB8000264A02EB80000B30E7
:1042F0008155701CC6B22078B6EB101FEEDB681E2D
:1043000000EB80001F4901EB8000867276E0FFE73A
:1043100005F10900C0B28DF80A0000208DF80B00ED
:10432000207800F0040020B301208DF80C006068B4
:10433000C0F34F30ADF800004FF6FF71606801EA3E
:10434000C000001DADF802000421681E00EB8000D3
:104350000D4A02EB80000172681E00EB800002EB48
:104360008000616841600F2D30D10A4960680860A3
:104370002CE011E0E4000020DC0000200068004098
:10438000D8000020CC210020A02000200004024002
:10439000E0000020E800002000208DF80C00ADF8BF
:1043A00000004FF6FF71606801EA4010ADF80200AE
:1043B0000021681E00EB8000FE4A02EB80000172C3
:1043C000681E00EB8000616842F82010FA4800681F
:1043D000C0F34F30ADF80400F74800684FF6FF71A6
:1043E00001EAC000001DADF806000020ADF808008D
:1043F00001208DF80D0068460BF0CBF97FBD70B53C
:1044000004460D4629462046FFF73DFF70BD30B5F6
:10441000431E03EB8303E94C04EB83035B68002B2F
:1044200050D1431E03EB830354F82330002B49D1B2
:104430000B7823F00F030B70431E03EB8303DD4C5B
:1044400004EB83031B7A042B0BD10B7843F004039A
:104450000B70431E03EB830304EB83035B684B6029
:104460000AE00B7823F007030B70431E03EB830372
:10447000D04C54F823304B6000220CE0431E03EB79
:104480008303CC4C04EB83030B339C5C01F10803E6
:104490009C54531CDAB2431E03EB8303C54C04EB5C
:1044A00083039B7A9342E9DC0B780F242340441E5C
:1044B00004EB8404BF4D05EB8404A47A43EA04139F
:1044C0000B7048E00B7843F008030B70431E03EBBE
:1044D0008303BA4C04EB83031B7A042B0BD10B78B8
:1044E00043F004030B70431E03EB830304EB8303CD
:1044F0005B684B600AE00B7823F007030B70431EE8
:1045000003EB8303AD4C54F823304B6000220CE0E6
:10451000431E03EB8303A94C04EB83030B339C5C26
:1045200001F108039C54531CDAB2431E03EB8303CE
:10453000A24C04EB83039B7A9342E9DC0B780F24B3
:104540002340441E04EB84049C4D05EB8404A47AB0
:1045500043EA04130B7030BD30B504460D462946BE
:104560002046FFF754FF30BD014601207047014649
:10457000012070471FB50446601E00EB80008F4984
:1045800001EB8000406880B9601E00EB800051F8AC
:10459000200050B904F10900C0B28DF80A000020D3
:1045A0008DF80D0068460BF0F4F8012004B010BD42
:1045B00030B5024600200AE00C5C531E03EB830377
:1045C0007E4D05EB83030B331C54431CD8B2531EA2
:1045D00003EB8303794C04EB83039B7A8342EBDC8C
:1045E00030BD10B50446601E00EB8000734A02EB3C
:1045F000800173480BF07FF910BD10B50446601EB2
:1046000000EB80006D4A02EB80016D480BF073F9FE
:1046100010BD6B48006840F001006949086000BFA8
:104620006748001D006800F001000028F8D06448C9
:10463000006820F0010062490860704710B586B03C
:10464000FF20604908704FF0FF300190029001AAEE
:1046500000215B480BF05FFA00245BE004EB840070
:10466000544901EB8000007AB0B904EB840051F8A2
:104670002000019988424BD1E01C524908700F2458
:104680000978C91E01EB81014A4A02EB810014221C
:1046900001A90BF09AFD3BE004EB8400454901EBD6
:1046A00080004068444909680840434A02991268FA
:1046B0001140884215D10E2C13DAE01C41490870D4
:1046C00008460078404908703E490978C91E01EB48
:1046D0008101384A02EB8100142201A90BF075FD1B
:1046E0000F243A490298096808403249D1F81C1150
:1046F000364A1268114088420AD10E2C08D1022095
:1047000030490870142201A931480BF05EFD0F24D6
:10471000601C84B20F2CA1DB2A480078FF2809DA3C
:104720002C48007818B12C480068804702E02B48DC
:1047300000688047082122480BF086FB06B010BDB8
:1047400010B51F481830046804F0700028B304F056
:104750007000302812D0012021490870002118482B
:104760000BF0A7F9012116480BF0A3F90221144818
:104770000BF09FF912480AF069FF02E00120194985
:1047800008700F481830006820F070000C4918318C
:104790000860C9140A480BF057FB04F0010088B305
:1047A0001048007870BB002105480BF082F9012108
:1047B000034819E0A0200020EC000020CC210020BC
:1047C00000680040F2000020F3000020E400002018
:1047D000B8210020D8000020E0000020DC000020EC
:1047E000F9000020FA0000200BF063F902211248C2
:1047F0000BF05FF910480AF029FF4FF480710E4862
:104800000BF022FB04F0020038B10B480AF01EFF47
:104810004FF4007108480BF017FB4FF400410648B5
:104820000BF012FB10BD10B50120044908700121E6
:1048300001480BF009FB10BD00680040FB000020A0
:1048400010B5FE480078022802D0032804D102E007
:1048500001F024F94AE349E3F8480078C01EF7491B
:1048600008700821F6480BF05CFA00287ED0FF2182
:10487000F248007800EBC00202EB0010F14A02EBB4
:10488000C002F148ED4B1B7830F8130022F81010ED
:10489000EA48007800EBC00202EB0010E94A02EBA4
:1048A000C002E948E54B1B7830F81300401C22F8A1
:1048B0001010E248007800EBC00202EB0010E14A61
:1048C00002EBC002E048DD4B1B7830F81300801C7F
:1048D00022F81010D948007800EBC00202EB00105B
:1048E000D84A02EBC002D848D44B1B7830F81300EA
:1048F000C01C22F81010D148007800EBC00202EB77
:104900000010D04A02EBC002CF48CC4B1B7830F8E5
:104910001300001D22F81010C848007800EBC002F8
:1049200002EB0010C74A02EBC002C748C34B1B781A
:1049300030F81300401D22F81010FF22BF48007805
:1049400000EBC00101EB0010BE4901EBC001BE4805
:10495000BA4B1B7830F81300801D21F81020BA489C
:10496000B649097830F81100C01D00E005E0B649ED
:10497000B24A127821F81200B7E2B048007800EB92
:104980008000B24901EB8000C07A00F0F0002028DE
:104990007DD1AA48007800EB800001EB8000017B0C
:1049A000A648007800EBC00202EB0010A54A02EB1B
:1049B000C002A548A14B1B7830F8130022F8101054
:1049C0009E48007800EB8000A04901EB8000427B0C
:1049D0009A48007800EBC00101EB0010994901EB07
:1049E000C0019948954B1B7830F81300401C21F802
:1049F00010209248007800EB8000944901EB800081
:104A0000827B8E48007800EBC00101EB00108D49DD
:104A100001EBC0018C48894B1B7830F81300801CD7
:104A200021F810208548007800EB8000874901EBD1
:104A30008000C17B8148007800EBC00202EB0010CF
:104A4000804A02EBC00280487C4B1B7830F8130090
:104A5000C01C22F810107948007800EB80007B49D8
:104A600001EB8000027C7548007800EBC00101EB8F
:104A70000010744901EBC0017348704B1B7830F88B
:104A80001300001D21F810206C48007800E050E071
:104A900000EB80006D4901EB8000417C67480078A5
:104AA00000EBC00202EB0010664A02EBC00266484F
:104AB000624B1B7830F81300401D22F810105F483D
:104AC000007800EB8000614901EB8000827C5B484C
:104AD000007800EBC00101EB00105A4901EBC00166
:104AE0005948564B1B7830F81300801D21F81020D0
:104AF00057485249097830F8111053484F4A1278F4
:104B000030F81200C01D814207DA012051490870B7
:104B100051494A4A12788854E7E14B484749097895
:104B200030F81100C01D4849444A127821F812009B
:104B3000DBE14248007800EB8000444901EB800053
:104B4000C07A00F0F000002876D13C48007800EBF5
:104B5000800001EB8000007B7F2810D1374800786F
:104B600000EB800001EB8000807B782807D13A4978
:104B7000324A12788854022036490870B5E12F482D
:104B8000007800EB8000314901EB8000007B7F283A
:104B900010D12A48007800EB800001EB8000807B78
:104BA000212807D12C49254A127888540220294906
:104BB00008709AE12148007800EB8000234901EB5E
:104BC0008000C07A00F00F0021491C4A127821F8B9
:104BD00012002248007800280EDD18480078401E98
:104BE0001F49085C1549097801EBC10202EB01116C
:104BF000144A22F831000FE010480078401E19498D
:104C000011F8100008300D49097801EBC10202EBE0
:104C100001110C4A22F831000848007800EB8000AE
:104C20000A4901EB8000007B0449097801EBC102CD
:104C300002EB0111034A17E08DE00000F2000020B2
:104C40000068004012230020E22A0020A02000205B
:104C5000F62A0020F80000200A2B0020F600002091
:104C6000F82200200223002002EBC1014880FE4808
:104C7000007800EB8000FD4901EB8000407BFA49A1
:104C8000097801EBC10202EB0111F94A02EBC10103
:104C90008880F548007800EB8000F44901EB800043
:104CA000807BF149097801EBC10202EB0111F04A66
:104CB00002EBC101C880EC48007800EB8000EB49B2
:104CC00001EB8000C07BE849097801EBC10202EBEF
:104CD0000111E74A02EBC1010881E348007800EBCB
:104CE0008000E24901EB8000007CDF49097801EB9C
:104CF000C10202EB0111DE4A02EBC1014881DA4830
:104D0000007800EB8000D94901EB8000407CD64957
:104D1000097801EBC10202EB0111D54A02EBC10196
:104D20008881D148007800EB8000D04901EB8000F9
:104D3000807CCD49097801EBC10202EB0111CC4A1C
:104D400002EBC101C8810120CA49C74A12788854C0
:104D5000C9490870C9E0C448007800EB8000C34925
:104D600001EB8000C07A00F0F0001028F2D1BE48BC
:104D7000007800EB800001EB8000017BBF48BA4A5D
:104D8000127820F81210BE48007800280EDDB648D0
:104D90000078401EBB49085CB349097801EBC102A9
:104DA00002EB0111B24A22F831000FE0AE48007860
:104DB000401EB54911F810000830AB49097801EBE5
:104DC000C10202EB0111AA4A22F83100A64800787C
:104DD00000EB8000A54901EB8000407BA2490978E7
:104DE00001EBC10202EB0111A14A02EBC1014880B3
:104DF0009D48007800EB80009C4901EB8000807B9F
:104E00009949097801EBC10202EB0111984A02EBC2
:104E1000C10188809448007800EB8000934901EB41
:104E20008000C07B9049097801EBC10202EB0111BF
:104E30008F4A02EBC101C8808B48007800EB8000EC
:104E40008A4901EB8000007C8749097801EBC102A7
:104E500002EB0111864A02EBC10108818248007809
:104E600000EB8000814901EB8000407C7E4909789D
:104E700001EBC10202EB01117D4A02EBC101488145
:104E80007948007800EB8000784901EB8000807C55
:104E90007549097801EBC10202EB0111744A02EB7A
:104EA000C1018881022073496F4A1278885472497F
:104EB0000870072175486C4A127820F81210704863
:104EC0000078002808DD68480078401E6D4A115CB3
:104ED0001D2000F06BFE08E063480078401E6A4A1F
:104EE00032F810100B2000F061FE00BF00BF10BDB3
:104EF00010B55D480078012804D0022803D00328AB
:104F00007ED197E295E2FCF7E6FB082160480AF0C3
:104F100008FF18B101205F4908708AE25348D0F8B1
:104F20001C01C0F307405C49088008460088B0F5C2
:104F30006E0FF2D008460088B0F56A0FEDD05748E2
:104F40004078098888427DD14848B0F81C01C0F3F8
:104F5000072051490880514800780988884209D0C3
:104F60004D4800884E490978884203D04A48008855
:104F7000FF28D2D101204B49087000204649088003
:104F800049490870394890F81C01484908700FE0F9
:104F9000474841490988405C44490978884202D120
:104FA0000120414908703C480088401C3A4908806B
:104FB0003F4839490988405CFF2807D036480088B7
:104FC0000D2803DA384800780028E1D03948007805
:104FD00010B93548007868B13648007801289CD16E
:104FE0003248007834490978884296D12E480078B2
:104FF000002892D12D4801782D48274A128800E0D8
:1050000019E28154294800782C49097801EBC10143
:105010002B4A5054154890F823012849097801EB90
:10502000C10111444870114890F8240123490978BE
:1050300001EBC101114488700C4890F825011F490B
:10504000097800E077E001EBC1011144C87007481E
:1050500090F826011949097801EBC1011144087142
:10506000024890F827012DE0F2000020A020002047
:10507000122300200A2B0020F8000020F62A00202E
:10508000F6000020F822002002230020E22A00205F
:105090000068004037010020F40000202E010020AD
:1050A0003A010020310100203C0100203D01002098
:1050B000DF6A00203E0100203F0100203601002071
:1050C000844D0020FE49097801EBC101114448716B
:1050D000FC4890F82801FA49097801EBC101114414
:1050E0008871F84890F82901F549097801EBC10168
:1050F0001144C871F34890F82A01F149097801EB8D
:10510000C10111440872EE480078401CEC49087057
:10511000084600780B2801D100200870EA48007882
:10512000EA490978884205D1E94800780128FAD18E
:10513000E84908707DE1E8480088EC28FAD1E148A8
:1051400090F8230120287DD1DE4890F82901F0282D
:105150003CDADC4890F82901E04949788842E9D1F5
:10516000D84890F82A01DD4989788842E2D107F0D1
:1051700065F9DB49DB4A127801F82200D14890F842
:105180002601D84A127801EB82014870D548007890
:10519000D54909780844D249D24A127801EB8201F4
:1051A0008870CF48CF49097810F82100FF28C1D076
:1051B000CC480078401CCB490870CC480078401C93
:1051C000CA4908700120CA49087032E1BD4890F808
:1051D0002801C24909788842ACD1BA4890F829011F
:1051E000BE4949788842A5D1B64890F82A01BB4902
:1051F000897888429ED107F021F9B949B94A1278D5
:1052000001F82200AF4890F82611B548B54A127847
:1052100000EB82004170B3480078B3490978084434
:10522000C1B2AF48AF4A127800EB82008170AC483F
:10523000AC49097810F82100FF28C6D0A9480078A9
:10524000401C00E00AE0A7490870A8480078401C0C
:10525000A64908700120A6490870EAE0994890F82C
:1052600023011028B1D1974890F82901F0286DDA70
:10527000944890F82901994949788842A5D19148E4
:1052800090F82A019549897888429ED107F0D6F88E
:105290009849954A127801F832008A4A92F8271103
:1052A000944A914B1B7812F83300012206F000FA61
:1052B000844890F826118F488B4A127800EBC20080
:1052C0004170804890F827018A49874A127801EB9B
:1052D000C20188707B4890F827118648824A12786C
:1052E00000EBC200C1707F4800787F49097808440C
:1052F000C1B280487C4A127800EBC20081717148CB
:1053000090F824117B48784A127800EBC2000171B2
:105310006C4890F825117748734A127800EBC20068
:10532000417174487049097810F83100FF280CD099
:105330006D480078401C6C4908706F480078401C2C
:105340006D49087001206A49087072E05D4890F864
:1053500028016249097888426BD15A4890F829019E
:105360005E494978884264D1564890F82A015B49E1
:10537000897888425DD107F061F85E495A4A12780F
:1053800001F832004F4A92F827115A4A564B1B78BF
:1053900012F83300012206F08BF94A4890F82601F2
:1053A0005449514A127801EBC2014870454890F8BF
:1053B000270150494C4A127801EBC20188704148DC
:1053C00090F827114B48484A127800EBC200C17090
:1053D000444800784449097808444649424A1278CA
:1053E00001EBC2018871374890F8240141493E4AD7
:1053F000127801EBC2010871324890F825113D483E
:10540000394A127800EBC20041713A4836490978AE
:1054100010F83100FF280CD033480078401C324986
:10542000087035480078401C334908700120304925
:105430000870C9E1C8E131480078C01E2F490870E2
:1054400008212F480AF06DFC00287DD02B480078F9
:10545000401E21490880FF200988C1EB011101EBA2
:10546000C101284A02EB8101274A1B4B1B88D25CF1
:1054700002EBC202885418490988C1EB011101EB03
:10548000C101204A02EB81011F4A134B1B88D25CE9
:1054900002EBC20211444870FF220F480088C0EBA3
:1054A000001000EBC000174901EB800016490A4BC1
:1054B0001B88C95C01EBC10108448270FF2025E014
:1054C00036010020A02000203D0100203F010020E7
:1054D0003E01002040010020F40000202E010020A9
:1054E000E84C00203201002033010020340100206C
:1054F000310100201C4D002035010020F200002069
:1055000000680040E74D002053690020FE490988EB
:10551000C1EB011101EBC101FC4A02EB8101FC4A24
:10552000F94B1B88D25C02EBC2021144C870FF2108
:10553000F5480088C0EB001000EBC000F34A02EB16
:105540008002F348F04B00E034E01B88C05C00EBC5
:10555000C00010440171FF20EB490988C1EB011123
:1055600001EBC101E94A02EB8101E94AE64B1B88E4
:10557000D25C02EBC20211444871FF21E24800886C
:10558000C0EB001000EBC000E04A02EB8002E048F4
:10559000DD4B1B88C05C00EBC00010448171DC480F
:1055A000D9490988405C401CC1B2D948D64A128802
:1055B000815408E1D7480078401ED3490880D54877
:1055C000007800EB8000D44901EB8000C07A401ED7
:1055D000CF49CD4A12888854CB480088C0EB0010D0
:1055E00000EBC000C94901EB8001C948C64A1288D6
:1055F000805C00EBC0000844C07900287ED1C5481B
:10560000007800EB8000C44901EB8000027BBE48BB
:105610000088C0EB001000EBC000BC4901EB80012A
:10562000BB48B94B1B88C05C00EBC0000A54B948AA
:10563000007800EB8000B84901EB8000427BB24863
:105640000088C0EB001000EBC000B04901EB800106
:10565000AF48AD4B1B88C05C00EBC00008444270F3
:10566000AC48007800EB8000AB4901EB8000807B08
:10567000A5490988C1EB011101EBC101A34A02EB65
:105680008101A34AA04B1B88D25C02EBC2021144E9
:105690008870A048007800EB80009F4901EB8000F3
:1056A000C17B99480088C0EB001000EBC000974A0E
:1056B00002EB80029648944B1B88C05C00EBC00054
:1056C0001044C1709348007800EB8000924901EBD0
:1056D0008000007C8C490988C1EB011101EBC101FC
:1056E0008A4A02EB81018A4A874B1B88D25C02EB13
:1056F000C202114408718748007800E056E000EBD0
:105700008000854901EB8000407C7F490988C1EB1E
:10571000011101EBC1017D4A02EB81017C4A7A4B08
:105720001B88D25C02EBC2021144487179480078B0
:1057300000EB8000784901EB8000827C7248008891
:10574000C0EB001000EBC000704901EB8000704915
:105750006D4B1B88C95C01EBC101084482710122B9
:1057600069480088C0EB001000EBC000674901EBFE
:1057700080006749644B1B88C95C01EBC101084488
:10578000C27161480088C0EB001000EBC0005F49A7
:1057900001EB8000007A401C5B490988C1EB0111D4
:1057A00001EBC101594A02EB810108725848564980
:1057B0000988405C401CC1B25548534A1288815444
:1057C00001205649087000BF00BF10BD10B500246D
:1057D00050480078012802D0022873D100E01EE171
:1057E000FBF779FF08214E480AF09BFA002867D1A1
:1057F0004948D0F81C01000C43490880084600883D
:10580000EA285DD008460088EB2859D00846008871
:10581000EC2855D0084600784249097801EB41014F
:10582000414A114488703C4890F81C013D49097870
:1058300001EB41011144487000203349088024E005
:105840003848007800EB40003749084440782E493A
:10585000098801EB4101344A1144497888420FD14B
:105860003048007800EB4000114608448078264913
:10587000098801EB410111448978884200D1012453
:1058800021480088401C204908801F48008825497D
:105890000978884201DA002CD2D08CB90120214944
:1058A000097801EB4101204A50541E480078401C01
:1058B0001C49087008460078312801DD0020087076
:1058C000ADE0FFE713480078C01E12490870084693
:1058D0000078401E0C490880082111480AF021FA7E
:1058E00000287DD10B48007800EB80000A4901EBCD
:1058F0008000C17A0D48044A128800F83210054829
:10590000007800EB800013E0F4000020E74D002059
:1059100053690020F2000020A02000203101002067
:10592000006800403B0100206D6900203F6A0020B4
:10593000554901EB8000007B5449554A128801EB20
:10594000C20148705348007800EB80004E4901EBDB
:105950008000407B4D494E4A128801EBC20188709D
:105960004C48007800EB8000474901EB8000807BC9
:105970004649474A128801EBC201C8704548007881
:1059800000EB8000404901EB8000C07B3F49404A6A
:10599000128801EBC20108713E48007800EB8000DC
:1059A000394901EB8000017C3848394A128800EB04
:1059B000C20041713748007800EB8000324901EBAA
:1059C0008000417C3148324A128800EBC20081716C
:1059D0003048007800EB80002B4901EB800000E0AC
:1059E0001CE0807C29492A4A128801EBC201C87157
:1059F00029482749098800EB8100C07838B901217E
:105A00002548234A128800EB8200817006E00021BD
:105A100021481F4A128800EB8200C17000BF00BFFE
:105A200010BD1C480078801E0A2810D2DFE800F064
:105A300005060708090A0B0C0D0E09E008E007E04F
:105A400006E005E004E003E002E001E000E000BF62
:105A500000BF70470F480078801E0A2810D2DFE888
:105A600000F005060708090A0B0C0D0E09E008E016
:105A700007E006E005E004E003E002E001E000E00A
:105A800000BF00BF70470000A02000203F6A002038
:105A9000F4000020F2000020036A002030B585B039
:105AA0000025FBF718FE924890F823018DF80800B6
:105AB0008F4890F81C018DF810009DF8080000F048
:105AC000F00028B19DF8080000F0F000102869D11E
:105AD00088480078002846D19DF810008649854AFC
:105AE0001278885483480078401C824908708048A6
:105AF000C07A00F00F00814948807D4890F81C0171
:105B00007F49A1F8C8007A4890F824117C48A0F891
:105B1000CA10774890F825117948A0F8CC1074483D
:105B200090F826117648A0F8CE10714890F8271109
:105B30007348A0F8D0106E4890F828117048A0F86B
:105B4000D2106B4890F829116D48A0F8D41068481D
:105B500090F82A116A48A0F8D610012069494870C7
:105B6000694908701EE0634800780A281ADA0024A0
:105B700008E06148005D9DF81010884200D10125C1
:105B8000601CC4B25B4800788442F2DB55B99DF8D2
:105B900010105948574A1278815456480078401CD2
:105BA00054490870FBF797FD05B030BD30B585B09E
:105BB00005460C46FBF78FFD0B2D04D188208DF890
:105BC0000000019406E08C208DF800004F4800EBA7
:105BD0000420019030208DF808004D4801788DF8A0
:105BE00009104C4801788DF80A1000218DF80B102F
:105BF0008DF80C108DF80D108DF80E108DF80F101B
:105C000000208DF8100069460120FEF73CFB0120C2
:105C1000FEF7E7FC05B030BD2DE9F04F8BB005462F
:105C20000C4616461F46DDE916ABDDE91489FBF785
:105C300052FD0B2D06D188208DF8180004F5E06088
:105C400007900DE08C208DF81800332C04D13248D9
:105C500000EB0420079003E02C4800EB04200790A1
:105C60008DF8206006A847728DF822808DF8239069
:105C70008DF824A08DF825B006A918988873199876
:105C8000C87300208DF8280006A8C07B897B06AA6F
:105C9000527B06AB1B7BCDE90232CDE9041006A88E
:105CA000C07A06A9897ACDE9001006A8437A9DF842
:105CB00020201AA0079906F02DFD06A90120FEF765
:105CC000E2FA0120FEF78DFC0BB0BDE8F08F70B555
:105CD00086B004460D461B4844EA000684208DF831
:105CE0000400029601A92846FEF7CDFA06B070BD61
:105CF000A0200020F6000020F8220020F62A002034
:105D0000122300200A2B0020F8000020F100DA18EE
:105D1000FC000020FD000020F100DB1861726249E8
:105D2000643A255820646174613A2558202558202A
:105D3000255820255820255820255820255820252D
:105D4000580D000000F1DA182DE9F041A2B0002052
:105D5000FE490860FE490860FE490860FE49086087
:105D6000FE49897B48B207F0DEF88046FB49497B53
:105D700048B207F0D8F808EB0010F9490870F74965
:105D8000C97A48B207F0CFF88046F449897A48B218
:105D900007F0C9F808EB0010F24908706B20487052
:105DA00000208870C8700871002507E00020EE49C7
:105DB00041F82500ED4941F825006D1C202DF5D353
:105DC0000120E9490860E94908600025002601240E
:105DD00043E0C6F107010120884000F0F507EFB16C
:105DE000601EE14951F82000083041F82400601E8F
:105DF000DE4951F82000083041F82400641C601E80
:105E0000D94951F82000103041F82400601ED749CC
:105E100051F82000103041F824001CE0601ED249E7
:105E200051F82000103041F82400601ECF4951F88D
:105E30002000103041F82400641C601ECA4951F84B
:105E40002000083041F82400601EC84951F82000A5
:105E5000083041F82400761C641C082EB9D30121B7
:105E6000084607F01FFA0121102007F01BFA012154
:105E7000084607F05BFA0121084607F046FA0121BF
:105E8000082007F042FA0121480507F00BFA012229
:105E90000921B74807F0B7FC01220B21B44807F0ED
:105EA000B2FC01220D21B24807F0ADFC01220E2107
:105EB000AF4807F0A8FC01220221AE4807F0A3FC7E
:105EC00001220321AB4807F09EFC0C202090022009
:105ED0008DF884008DF8850000208DF88600022062
:105EE0008DF8870020A9A34807F00AFC4FF4D4409E
:105EF000209020A99E4807F003FC9F4808F028FC4A
:105F00004FF0804008F024FC9C4808F021FC002061
:105F10004FF0804108824FF6FF714FF0804008F04B
:105F200056FE4FF6FF714FF0804008F052FE4FF6DC
:105F3000FF71924808F04BFE3C20ADF804000020B1
:105F4000ADF806004FF6FF7002900020ADF80C008F
:105F500001A94FF0804008F03EF93C20ADF8040064
:105F600001A9864808F037F97820ADF80400002030
:105F7000ADF806004FF6FF7002900020ADF80C005F
:105F800001A97D4808F027F93020ADF86C00012008
:105F9000ADF86E004FF6FF701D900220ADF878004E
:105FA0001BA9400708F0C1F90020ADF878001BA933
:105FB0004FF0804008F0FCF90020ADF84C00401E86
:105FC000159013A96D4808F038F9002211466B4866
:105FD00008F06FFD00220F214FF0804008F0AAFB6F
:105FE00000221021880608F0A5FB0122D102C80476
:105FF00008F0A5FB01221103880408F0A0FB4FF074
:10600000C06004905E4805904020079000200990F1
:106010004FF480600A9080000B9080000C9000206C
:106020000D904FF480300E9000200F901090119042
:10603000129004A9534808F0A3FF4FF0C0600490E9
:106040004F48001D059004A94E48783008F098FF8D
:10605000012210214B4808F0E4FF01221021494899
:10606000783008F0DEFF0020ADF86000ADF8620087
:106070000120ADF864000020ADF86600ADF86800BE
:1060800018A93D4808F087FA0C20ADF86000002000
:10609000ADF8620018A9384808F07DFA0420ADF880
:1060A00060000220ADF8620018A9334808F073FAC6
:1060B0000820ADF860000220ADF8620018A92E4853
:1060C00008F069FA00212C4808F07DFD00212B48DA
:1060D00008F079FD0121284808F007FB0121274835
:1060E00008F003FB01220021234808F0E2FC012212
:1060F0000421214808F0DDFC0A2202210846FBF7B2
:106100002EF8642006F0CFFB012202211A4808F085
:1061100006FB22B0BDE8F0812DE9F14F8AB04FF0C7
:10612000040820200190002600BF0C4A08F101015C
:10613000515C48B206F0F7FE8346084911F8081092
:1061400048B206F0F0FE0BEB00101DE094000020BA
:106150007C00002084000020880000200A0B002022
:10616000990000209A000020441B0020C41B00203E
:10617000001002400000024000000140000C0040FE
:106180003C0000402860024002A921F81600FBF7FD
:10619000A2FA701CC6B2FE4908F10200085C019028
:1061A00008F1030801980028BFD1C97A48B206F067
:1061B000BAFE8346F649897A48B206F0B4FE0BEB84
:1061C0000010F44908700120F3490860F3490860A1
:1061D00000240027012545E0C7F107010120884080
:1061E00000F0F509B9F1000F1DD0681EEA4951F819
:1061F0002000801D41F82500681EE84951F8200064
:10620000001D41F825006D1C681EE34951F820006F
:10621000123041F82500681EE04951F82000143082
:1062200041F825001CE0681EDB4951F820000E30C3
:1062300041F82500681ED94951F820000C3041F87A
:1062400025006D1C681ED44951F820000A3041F821
:106250002500681ED14951F820000C3041F8250076
:106260007F1C6D1C082FB7D3FBF735FA0A9870B95D
:10627000C749C97A48B206F056FE8346C449897AAE
:1062800048B206F050FE0BEB0010C5490870002024
:10629000C4490860002404E00020C34921F8140028
:1062A000641CFF2CF8D9314602A8FBF7EAFF8246AE
:1062B00002A921F816A0701CC6B21E20BB490860B6
:1062C00008460068123048601C20B949086008463A
:1062D000006814304860002497E00027002590E013
:1062E00002A830F81400C7F107020121914000EA2A
:1062F0000109B9F1000F41D0022000EB041028443D
:10630000401EAA4951F82000801D022101EB041112
:106310002944A64A42F82100022000EB0410284438
:10632000401EA34951F82000001D022101EB041179
:1063300029449F4A42F821006D1C022000EB041002
:106340002844401E994951F820001230022101EBE7
:1063500004112944954A42F82100022000EB041060
:106360002844401E924951F820001430022101EBCC
:10637000041129448E4A42F8210040E0022000EB3B
:1063800004102844401E894951F820000E30022193
:1063900001EB04112944854A42F82100022000EB58
:1063A00004102844401E824951F820000C3002217C
:1063B00001EB041129447E4A42F821006D1C0220A1
:1063C00000EB04102844401E784951F820000A30A0
:1063D000022101EB04112944744A42F821000220F1
:1063E00000EB04102844401E714951F820000C3085
:1063F000022101EB041129446D4A42F821007F1C5F
:106400006D1C082FFFF46CAF641CB442FFF465AF41
:10641000012101EB0610401E644951F82000643050
:10642000012202EB0611614A42F82100012101EB31
:106430000610401E5E4951F820006430012202EB34
:1064400006115B4A42F821000121880708F0C3FBCE
:106450000121880708F0C1FB544856494863544855
:106460005449AC310860022101EB06105149C86261
:10647000022101EB06104F49C1F8A40001214D484B
:10648000283008F0B9FD01214A48A03008F0B4FDD9
:10649000012049490880494908800020484908806E
:1064A00000214FF0804008F08EFB00BF4548006897
:1064B0000028FBD10120434908600121800708F032
:1064C00014F9FBF708F900203F49088008460088C6
:1064D000192803DB01203D49088001E0FBF7FBF8A8
:1064E0000BB0BDE8F08F2DE9F047064600202D499E
:1064F0000860002404E000202B4921F81400641CEB
:10650000FF2CF8D9F1B23248FBF7BBFE8046304889
:1065100020F81680761C1E20244908600846006872
:10652000123048601C202249086008460068143078
:1065300048600024BAE000270025B3E0244830F882
:106540001400C7F107020121914000EA0109B9F1E5
:10655000000F64D0022000EB04102844401E1349B1
:1065600051F82000801D022101EB041129440F4A3B
:1065700042F82100022000EB04102844401E0C4980
:1065800051F82000001D022101EB0411294421E0F3
:106590000A0B002099000020441B0020C41B00208F
:1065A0009A0000208000002044190020340D0020B3
:1065B0003411002000600240780000207A000020A2
:1065C000B00000207C000020000000200C00002013
:1065D000F0090020FE4A42F821006D1C022000EB69
:1065E00004102844401EFB4951F8200012300221BB
:1065F00001EB04112944F74A42F82100022000EB84
:1066000004102844401EF24951F8200014300221A1
:1066100001EB04112944EE4A42F8210040E0022037
:1066200000EB04102844401EEA4951F820000E30C7
:10663000022101EB04112944E64A42F8210002201C
:1066400000EB04102844401EE14951F820000C30B2
:10665000022101EB04112944DD4A42F821006D1C9E
:10666000022000EB04102844401EDA4951F82000B3
:106670000A30022101EB04112944D64A42F82100D4
:10668000022000EB04102844401ED14951F820009C
:106690000C30022101EB04112944CD4A42F82100BB
:1066A0007F1C6D1C082FFFF449AF641CB442FFF43B
:1066B00042AF012101EB0610401EC64951F82000EF
:1066C0006430012202EB0611C24A42F82100012186
:1066D00001EB0610401EBE4951F820006430012233
:1066E00002EB0611BA4A42F821000121880708F09E
:1066F00072FA0121880708F070FAB648B649486373
:10670000B348B549AC310860022101EB0610B2492B
:10671000C862022101EB0610AF49C1F8A4000121B3
:10672000AD48283008F068FC0121AB48A03008F0E3
:1067300063FC0120A9490880A94908800020A949D3
:10674000088000214FF0804008F03DFA00BFA648C5
:1067500000680028FBD10120A349086001218007BF
:1067600007F0C3FFFAF7B7FF0020A04908800846EA
:106770000088192803DB01209D49088001E0FAF711
:10678000AAFFBDE8F0872DE9F04705460E46002731
:10679000B846B946012400209549088095490880EB
:1067A00000BF00209149088000BFFAF794FF92488B
:1067B000008818B98D4800888542F6DA8B48008831
:1067C000854202DC01208A4908808948008898BBFC
:1067D000B8F1010F0BDB012E02D04FF0030906E0E8
:1067E00040F2E730834921F81400601C04B283486A
:1067F00090F800A0012E03D10AF101000FFA80FAEF
:1068000000207D49088000270CE007EB09007C4947
:10681000085C784921F81400FAF75DFF601C04B2A7
:10682000781C07B2AAEB0900B842EEDCFAF753FF76
:1068300008F101000FFA80F86D4800880028B0D0F8
:106840006B480088012805D1B8F1010F02DB002058
:1068500067490880601E67490880BDE8F08770B509
:1068600086B000221146674808F023F900216548E8
:1068700008F0A9F963482430006863490860634858
:1068800008F0B5F962490860604808F0B3F9614959
:1068900008605548006801285FD1534908605A488C
:1068A00001683031574808F092F94E4800880228B4
:1068B0004DDD5848006858490968451A494800881C
:1068C000801E444951F8201046480088C01E414AA5
:1068D00052F820000E1A301D854202D8301FA842FF
:1068E00035D91020404908600021800607F0FDFEE0
:1068F00000213948283008F07FFB00213648A030BD
:1069000008F07AFB0020354908803549088040218D
:10691000080607F0CAFF4021080607F0CEFF302026
:10692000ADF804000120ADF806004FF6FF700390AB
:106930000220ADF8100001A9400707F0F6FC002086
:10694000ADF8100001A94FF0804007F031FD254857
:106950000088801C2349088040E1234800680428FF
:1069600006D1294801684831264808F030F935E158
:106970001D480068022803D01B48006800287DD10C
:10698000244800882549264A127821F81200214817
:10699000008821490988401A2249214A127821F8A1
:1069A00012001F490878C11700EB5171C9101E4A27
:1069B00011701C481A49097830F811000D2847DA7F
:1069C0000F4811460978405C11460978144A2DE0B9
:1069D00034110020340D00200060024078000020B7
:1069E0007A000020B00000207C0000200000002081
:1069F0000C0000205801002046000020A7000020C5
:106A000034190020000C0040040100200000014067
:106A1000A8000020AC0000209400002034170020C3
:106A2000A400002044190020A60000201278A2EB48
:106A3000C101C1F10702012191400843DE49DF4A4B
:106A400012788854DE480078401CDD4908702FE039
:106A5000DC48DB49097830F8110018281BDAD648E1
:106A6000D6490978405CD5490978D54A1278A2EB15
:106A7000C101C1F107026FF0010100E09CE091400B
:106A80000840CD49CD4A12788854CD480078401C42
:106A9000CB4908700CE0CC4801686031CB4808F065
:106AA00096F80020C6490870C9490870C3490870A3
:106AB000C8480068022806D1C348006800F12801D0
:106AC000C24808F084F80220C2490860BC48007837
:106AD000092830D10846007800F0010038BBB648DC
:106AE000007800F0080018BBB348007800F00700F9
:106AF000052818D2DFE800F003070B0F130002206F
:106B0000B549087013E00120B34908700FE0022076
:106B1000B14908700BE00320AF49087007E001207D
:106B2000AD49087003E00020AB49087000BF02E0E7
:106B30000020A9490870A248007812284ED1A54823
:106B4000007800F00100002848D19B48407800F010
:106B5000040098B198484078A0490978884209D043
:106B600000209D49087010209A49086000209C4927
:106B7000086033E001209A4908602FE0002098491E
:106B80000860002409E08C4840789649095D8842F5
:106B900002D1012092490860641C9248005D08B14E
:106BA000052CF0D38E480068C0B900208A490870CF
:106BB00010208849086011E086480068082806D13E
:106BC000814801683031814808F001F806E07E48CC
:106BD000006800F15B017D4807F0F9FF824800681A
:106BE000824908600221794808F033F80122022125
:106BF000764807F094FD01220021744807F059FF00
:106C000002217B4808F025F80821794808F021F88E
:106C100006B070BD10B502216C4808F009F80128D3
:106C200026D100220221694807F079FD0022114691
:106C3000664807F03EFF0221644808F00AF86548FC
:106C40000068012815D1614807F0D1FF00F1300438
:106C500021465E4807F0BBFF10205E490860022114
:106C60005A4807F0F6FF01220221584807F057FD65
:106C700099E058480068042812D11020554908604E
:106C8000514801686031514807F0A1FF02214F4887
:106C900007F0DFFF012202214C4807F040FD82E0AF
:106CA0004C48006802284BD1484807F0A0FF00F18B
:106CB00048042146454807F08AFF0221434807F06F
:106CC000C8FF01220221414807F029FD082041495F
:106CD000086041480078012865D1414800680128D2
:106CE00061D100203C4908700121880707F073FF3B
:106CF0000121880707F071FF3E483F4948633F483C
:106D00003D49AC31086010203B49C862C1F8A4007D
:106D100001213948283008F06FF901213648A030A8
:106D200008F06AF9012036490880364908800021B8
:106D3000800707F048FF0121880707F0D6FC32E002
:106D400024480068082812D11020224908601E48F3
:106D5000016860311D4807F03AFF02211B4807F027
:106D600078FF01220221194807F0D9FC1BE000201E
:106D70001849086011480078002814DD1848006898
:106D8000012810D1204908800C4800781F4908705C
:106D900000200B4908700E490870084908700D4919
:106DA00008600F4908600821084807F041FF0128E2
:106DB00001D1FBF7BEF810BD34190020A600002059
:106DC000A40000204419002004010020000C004011
:106DD000A50000207C0000209800002099000020E1
:106DE000000100209A000020A8000020940000204C
:106DF00000000140481B002000600240C81B00202A
:106E0000780000207A00002046000020A700002023
:106E100010B504462146794807F0D9FE10BD10B5DB
:106E200088B000240121080206F06FFA09221146F9
:106E3000734806F0E8FC734800687349B0FBF1F052
:106E4000401E84B2FF200690ADF814400020ADF83B
:106E50001C00ADF8160005A9684807F0BCF96020D1
:106E6000ADF800000120ADF8020000200290ADF85E
:106E70000C006946614807F0E0F908215F4807F017
:106E800054FD01215D4807F030FC0020FFF7C0FFF2
:106E900008B010BD10B50446A1B20022574807F053
:106EA000C6FC10BD5948008810B95948008808B17F
:106EB000012070470020FCE770B504460D46802095
:106EC000FFF7A6FF534890FBF4F63046FFF7E2FFCA
:106ED0004E48058070BD10B54D48008840B14C4803
:106EE00001884D480088FFF7E7FF002048490880E7
:106EF00010BD474A1180484A1080704710B50F21D5
:106F000040F2DC50FFF7D8FF322005F0CCFC0F2117
:106F10004FF4D460FFF7D0FF192005F0C4FC0F2117
:106F200040F29E70FFF7C8FF192005F0BCFC0F214E
:106F300040F67700FFF7C0FF192005F0B4FC0F21E1
:106F400040F68510FFF7B8FF192005F0ACFC0F21C3
:106F500040F6E220FFF7B0FF192005F0A4FC0F2156
:106F600040F6B240FFF7A8FF192005F09CFC0F2166
:106F700040F63C70FFF7A0FF10BD32202749888003
:106F80004FF45C712548A0F8541032202349088141
:106F90004FF45C712148A0F8581032201F498881B5
:106FA0004FF45C711D48A0F85C1032201B49088228
:106FB0004FF45C711948A0F86010704764201749BD
:106FC00048854FF4DC611548A0F87A106420134915
:106FD00048864FF4DC611148A0F882107047002009
:106FE0000E498880088188810882704700200B49FB
:106FF0004885C8854886C886704700000020004044
:10700000001402404401002080841E00080100207A
:107010000A010020109203000C010020142B002014
:1070200010B50121402006F070F901212B4807F02E
:107030005CFB0021294807F0FDFB0021274807F0F1
:10704000C2FD4FF0FF31254807F0BFFD01224FF48C
:107050001671224807F0EBFB10BD2DE9F0470646FC
:107060004FF00009CA4605E0A6F5803609F1010097
:107070001FFA80F9B6F5803FF6D2184807F0C3FD35
:1070800085B2A81987B22C46A04610E04FF0000A3E
:1070900008E0124807F0B7FD84B2444501DA4FF02A
:1070A000010AA046BAF1000FF3D0AC42F1DB5FEA6F
:1070B0000900A9F101011FFA81F9E7D1AF4205DA10
:1070C00000BF064807F09FFDB842FAD800BF03484A
:1070D00007F099FDB842FAD9BDE8F08700180040E2
:1070E00001460020CAB21044C1F307221044C1F384
:1070F00007421044C0B270472DE9F0410446250E06
:1071000024F07F463046FFF7EBFF0746BD4207D02D
:1071100010A21F2114A005F046FB0020BDE8F0815D
:107120003046FBE72DE9F0410025002409E0E006A8
:10713000070E104850F824603078B8400543601CB2
:10714000C4B2042CF3D3ED432846FFF7D5FFBDE8C6
:10715000F0810000496E76616C6964206368656344
:107160006B73756D0D0000007372635C6F74702E2D
:107170006300000024030D0830B502466FF000459F
:107180008A4201D9104600E0084603468A4201D2ED
:10719000104600E008460446181BB0F1004F05D326
:1071A0008A4201D8012030BD0020FCE78A4201D389
:1071B0000120F8E70020F6E7002007E0FF2100EBC0
:1071C00040025A4B03F82210411C88B21428F5D310
:1071D0000021574A11600121564A117070475448E6
:1071E0000068401C52490860704751480068704769
:1071F00070B55048007808B9FFF7DEFF002433E08F
:1072000004EB4400494911F82000FF282AD004EB80
:1072100044020B4603EB82025168454A1068FFF7AF
:10722000ABFF00281ED004EB4400404901EB800076
:10723000856825B940A2522144A005F08EFAFF20AE
:1072400004EB4401394A02F821003948036804EB91
:107250004400114601EB8000214642683FA005F042
:1072600059FAA847601C84B2142CC9D370BD70B5FC
:1072700006460D4625B930A2622134A005F06DFA0C
:10728000002421E072B604EB4400284911F82000E4
:10729000FF2816D104EB4401244A02F8214004EBF4
:1072A0004400114601EB8000466004EB440001EB12
:1072B0008000856062B604EB44001C4911F8200090
:1072C00070BD62B6601C84B2142CDBD32FA2762171
:1072D0001EA005F068FAFF20F2E770B504462546C7
:1072E00072B605EB4500114911F82000A04214D1F7
:1072F000FF2005EB45010D4A02F8210062B60C485B
:10730000036805EB4500094901EB8000214642680E
:1073100023A005F0FFF9012070BD62B623462CA220
:107320008B210AA005F03FFA0020F5E7B42B0020DE
:107330001401002010010020417373657274696F9D
:107340006E206F6363757265640D00007372635C19
:107350006A6F6253636865642E63000045786563F5
:10736000757465206A6F622C206964282564292061
:1073700074696D65282564292063757272656E7461
:1073800054696D65282564290D0000004E6F206644
:10739000726565206A6F627320666F756E640D009A
:1073A00052656D6F7665206A6F622C2069642825AE
:1073B00064292074696D65282564292063757272BB
:1073C000656E7454696D65282564290D0000000000
:1073D0004661696C656420746F2072656D6F7665B7
:1073E000206A6F622C206964282564290D00000042
:1073F00010B5F649F64807F0D3FEF648006838B1F4
:107400000520F449096808700020F249086004E08A
:10741000F1A23B21F8A005F0C6F910BD10B5FB495B
:10742000FB4807F0BDFEFB48006838B10520F9496C
:10743000096808700020F749086004E0E6A24B21C3
:10744000EDA005F0B0F910BD00213CE072B601EBF3
:10745000410000EB0120F04A12F8200078BB012027
:1074600001EB410202EB0122EB4B03F8220000206A
:1074700001EB410202EB012203EB8202908001EB5F
:10748000410202EB012203EB8202D080052001EBD6
:10749000410202EB012203EB82029070002001EB1B
:1074A000410202EB012203EB8202D07062B601EBD3
:1074B000410000EB0120D84A02EB80007047FFE753
:1074C00062B6481C81B20629C0D30020F6E770B529
:1074D0000446002524B9D1A26A21C7A005F03DF9D0
:1074E000206820B9CDA26B21C3A005F036F91FE0BA
:1074F00072B605EB450000EB0520C74901EB8000A3
:107500002168884211D1002005EB450101EB0521DE
:10751000C14A02EB8101C88005EB450101EB052161
:1075200002F82100206062B670BD62B6681C85B2A8
:10753000062DDDD3BEA27B21AFA005F034F900BF3C
:10754000F2E710B5044624B9B4A27F21AAA005F041
:1075500004F9BF48008B062804D3B0A28021A6A05E
:1075600005F0FBF80320207072B6B948018B008B40
:10757000401CB74A1083104640F8214062B610BD47
:1075800070B50546B248008BA04204DCA3A28B2153
:1075900099A005F0E2F82C4607E0AD49601C51F8CF
:1075A000200041F82400601C84B2A948008BA0424E
:1075B000F3DCA748008B401EA549088370BD10B5B9
:1075C00090B0044624B995A299218BA005F0C5F886
:1075D000607820B1012852D002287DD155E08D4835
:1075E000006810B1002010B010BD4FF06060019035
:1075F00000200A904FF400300B9000200C900320E4
:107600000D904020049000200F9006909148029029
:10761000002008900E9009904FF480600790E07869
:1076200048B1E088C21E04F10B01C81E08F08BFDB2
:10763000E088C01EE08004F108000390E088059017
:10764000734807F0FBFB01A9714807F099FC012280
:1076500010216F4807F0E5FC6C496D4807F0A0FD6C
:10766000042020706B480460012280217948001FAB
:1076700006F005FA0121664807F0BEFC71E076A22B
:10768000D0215DA005F069F86BE05248006808B1B0
:107690000020A8E74FF00060019000200A904FF40E
:1076A00000300B9000200C9003200D90402004909F
:1076B00000200F90069072480290002008900E90D3
:1076C00009904FF480600790E07858B1E088C21EBE
:1076D00004F10B01C81E00E028E008F034FDE0884A
:1076E000C01EE08004F108000390E088059038484F
:1076F00007F0A4FB01A9364807F042FC0122102143
:10770000334807F08EFC4149314807F049FD042019
:10771000207030480460012280215948001F06F083
:10772000AEF901212A4807F067FC1AE060780528C5
:1077300007D2637853A24FF484712FA005F033F879
:1077400009E06078574901EB800357A24FF4867136
:1077500029A005F028F8052020705BA005F001FBAA
:1077600000BF00BF01203EE710B5002409E0002063
:1077700004EB440101EB0421274A02F82100601CBC
:1077800084B2062CF3D3002405E00020304941F8F0
:107790002400601C84B2062CF7D300202C490883F7
:1077A0000121880505F07EFD0121480505F07AFDDF
:1077B00010BD10B504462CB918A240F22F110EA02E
:1077C00004F0CBFF206800B182E087E00080002851
:1077D000B864024018010020556E657870656374C6
:1077E000656420696E74657272757074206F63636E
:1077F00075726564000000007372635C6D736748A6
:10780000616E646C65722E630000000020800020B1
:10781000706002401C010020A42C0020417373659D
:107820007274696F6E206F6363757265640D00001A
:10783000446964206E6F742066696E6420627566A8
:1078400066657220746F2072656C656173650000F7
:10785000FC4400200448004073656E644D7367204B
:10786000746F204344502073686F756C64206E6F92
:107870007420656E64207570206865726500000074
:107880000410014073656E644D736720746F20258A
:1078900064206973206E6F7420737570706F7274DA
:1078A00065640D0038030D0873656E644D736720C1
:1078B000746F202573206973206E6F742073757048
:1078C000706F727465640D002A2D310D0000000088
:1078D000FAA004F01FFF0620216808700020206035
:1078E000E071208110BD10B504463CB9AFF2D4025E
:1078F0004FF49E71AFF2001004F02FFF00202060C3
:10790000FF20207100216171A1710020E0712081B0
:1079100010BD70B504460D463CB9AFF200124FF4ED
:10792000A371AFF22C1004F018FFE07918B902200F
:10793000E07100202081E079022807D0AFF2241204
:1079400040F24D11AFF2501004F007FF208920B132
:10795000012807D0022825D109E025712089401C83
:1079600020815CE065712089401C208157E0A57171
:107970002089401C20812079012812D0FFF764FD66
:107980002060206838B9AFF26C1240F25F11AFF29C
:10799000981004F0E2FE20792168487000202168E8
:1079A000C8803CE0A179607941EA0026207901286D
:1079B00003D12846F8F71CFE1DE02089B0F5806F42
:1079C00012DA206838B9AFF2AC124FF4BA71AFF2E4
:1079D000D81004F0C2FE2068C188481C2268D080FC
:1079E00020680830455406E0C0A240F27911AFF299
:1079F000F81004F0D8FE2089401C80B22081C01EFF
:107A0000B0420BD12079012805D020792168487037
:107A10002068FFF796FD00202060E07100BF00BFE6
:107A200070BD70B506460C46042C07D3AFF2142285
:107A300040F29311AFF2402004F08FFE72B6B548C9
:107A400050F82400C8B3B34850F82400C088B0F5FB
:107A5000806F25DAAF4850F82400C188AD4850F84F
:107A60002400C088401CAB4A52F82420D080A9488A
:107A700050F8240008304654A64850F82400807876
:107A8000401C052805DDA34850F824008078401CE0
:107A900000E005209F4951F82410887062B670BD3F
:107AA00001209C4951F82410887062B600BF9948A3
:107AB00050F824000028FAD101E0FFE762B604E0A4
:107AC000FFF7C2FC934941F82400924850F8240083
:107AD0000028F5D08F4850F8240044708D4850F8A5
:107AE000240000F108050120287000206870A870AB
:107AF0000320884951F82410C880864850F8240093
:107B0000C188844850F82400C088401C814A52F83B
:107B10002420D0807F4850F82400083046540520A7
:107B20007C4951F82410887000BFB8E770B5002474
:107B300037E0784850F82400002830D0754850F8D5
:107B400024008078401EC0B2724951F82410887019
:107B500028BB704850F82400C088032807DAAFF229
:107B6000443240F2CF11AFF2703004F0F6FD6948B4
:107B700050F82400C088C01E86B2664850F8240021
:107B800000F10805300A6870AE70624951F82400AF
:107B9000FFF7D7FC00205F4941F8240000BF601CBC
:107BA000C4B2042CC5D370BD70B50646FFF74CFCBB
:107BB0000446B6F5806F07DDAFF2A0324FF4F171E5
:107BC000AFF2CC3004F0C9FD3CB9AFF2B03240F2B4
:107BD000E311AFF2DC3004F0C0FDFF20607004F16F
:107BE0000805287000206870A8700320E0802046F7
:107BF00070BD2DE9F04104460F4690463CB9AFF206
:107C0000E4324FF4FA71AFF2104004F0A6FD2068A0
:107C100038B9AFF2F83240F2F511AFF2244004F077
:107C20009CFD2068C088032807DAAFF210424FF4A9
:107C3000FB71AFF23C4004F090FD2068C088C01E8C
:107C400086B220684770206800F1080585F800803A
:107C5000300A6870AE702068FFF773FC0020206067
:107C6000BDE8F0812DE9F04707460D46904699465C
:107C7000FFF7EAFB04463CB9AFF2604240F20A214A
:107C8000AFF28C4004F069FD84F8018004F108062D
:107C900086F80090280A7070B5700320E080E288B2
:107CA000314650182A46394608F008FAE088284438
:107CB000E0802046FFF745FCBDE8F0875761726E13
:107CC000696E673A206461746120696E2072656331
:107CD00065697665722077696C6C206265206469DD
:107CE000736361726465640D00000000427566662E
:107CF000657220746F6F20736D616C6C202D6461F0
:107D00007461206973206469736361726465640DD2
:107D100000000000EC44002038B5002417E004EB1C
:107D2000440000EB04201A4901EB80000090009809
:107D30000078052802D0062805D100E000BF68467B
:107D4000FFF7C5FB00E000BF00BF601C84B2062C3B
:107D5000E5D3002417E00F4850F8240038B9AFF2FB
:107D6000445240F23621AFF2705004F0F6FC09495B
:107D700051F82400FFF723FC18B12046FFF700FC60
:107D800001E0601C84B20348008BA042E3DC38BDF4
:107D9000A42C0020FC4400201CB50121084605F05D
:107DA00081FA4FF48070009000208DF804000220CA
:107DB0008DF8050000208DF806008DF80700694653
:107DC0009B4805F09DFC0121022005F06BFA4FF461
:107DD0000070009001208DF8040002208DF805004D
:107DE00000208DF806008DF807006946914805F0DF
:107DF00087FC0320009002208DF8040069468D481E
:107E000005F07EFC0121042005F04CFA8020009052
:107E100002208DF804008DF8050000208DF8060082
:107E20008DF807006946844805F06AFC1F20009021
:107E300003208DF8040000208DF8070069467E4875
:107E400005F05EFC4FF44040009001208DF80400E6
:107E500002208DF8050000208DF806008DF807003F
:107E60006946764805F04CFC0121102005F01AFA0D
:107E70001E20009001208DF8040002208DF80500DE
:107E800000208DF806008DF8070069466C4805F063
:107E900037FC4020009002208DF8040069466848B5
:107EA00005F02EFC4FF4C070009000208DF8040007
:107EB00001208DF807006946614805F021FC012189
:107EC000202005F0EFF90820009002208DF8050031
:107ED00000208DF806008DF807008DF80400694633
:107EE000584805F00DFC4FF4C040009001208DF87B
:107EF000070000208DF804006946524805F000FC98
:107F00004FF40070009002208DF8040069464D483F
:107F100005F0F6FB4FF4C050009001208DF80400EE
:107F200002208DF8050000208DF806008DF807006E
:107F30006946444805F0E4FB0121402005F0B2F910
:107F40004FF4E050009001208DF8070000208DF8DC
:107F5000040069463C4805F0D3FB802000900120D6
:107F60008DF8040002208DF8050000208DF8060031
:107F70008DF807006946344805F0C2FB38200090B0
:107F800001208DF8040002208DF8050000208DF8F6
:107F9000060001208DF8070069462B4805F0B0FB6C
:107FA0001CBD1CB50121880305F0C0F90D2102207C
:107FB00008F03CF8684607F0F2FF4FF400500090DC
:107FC00000208DF804000C208DF8050001208DF8AC
:107FD0000600684607F09CFF1CBD10B54FF4005129
:107FE000184805F0DEFB08B1012010BD0020FCE7B9
:107FF00010B54FF48041134805F0D3FB08B10120C0
:1080000010BD0020FCE710B54FF480710C4805F05E
:10801000C8FB08B1012010BD0020FCE710B580218D
:10802000074805F0BEFB08B1012010BD0020FCE7A9
:10803000000002400004024000080240000C024020
:10804000001002400014024000180240002005E029
:108050000021FC4A22F81010411C88B21E28F7DBD0
:10806000704710B5F84AD2784AB9F74A127932B94E
:108070000122F64B1A700022F54B1A7052E00420D0
:1080800000210022F14B1A7047E0EF4A125C302ABF
:1080900010DBED4A125C392A0CDCEB4A125C303AF8
:1080A000EB4BEA4C24781A55E84A1278521CE74BFD
:1080B0001A7030E0E44A125C612A10DBE24A125C7A
:1080C000662A0CDCE04A125C573AE14BDF4C24781C
:1080D0001A55DE4A1278521CDC4B1A701BE0DA4A41
:1080E000125C412A10DBD84A125C462A0CDCD64AC4
:1080F000125C373AD64BD54C24781A55D34A1278AD
:10810000521CD24B1A7006E001210122CF4B1A708B
:108110000022CF4B1A70821CD0B2CB4A125C0AB13B
:108120000029B2D010BD2DE9F04188B004242027E9
:108130000026002404E00020C24921F81400641C39
:10814000142CF8D30120C34908800020C2490880BC
:10815000C2490880C2490880C24908800022022121
:108160000320F8F7FCFF642004F09DFBF9F74EFFB5
:10817000002004900590069001230790CDE900307F
:108180000290F1236A22682103900520FAF7ABF8E8
:1081900000F03000302802D00120B14908800020D2
:1081A000B0490880AE490880AF49088000BFF9F7A0
:1081B00092FAAC48008801280AD1FAF7A8F9A84831
:1081C000008810B90020A84908800020A449088030
:1081D000A5480088C828EADB9A48007A412802D0DE
:1081E00001209F4908809E48008800287ED19FA0DA
:1081F00004F0B7FDA448007820F04000A2490870C0
:108200000120A24908700620A149087000BFF9F7B3
:1082100062FA01208F4908809E480088012866D1B3
:108220008F4800880028FAD19A4908800424202722
:10823000002500BFF9F74FFA834A611C515C48B230
:1082400004F071FE80468049095D48B204F06BFE7F
:1082500008EB0010904948557B49A01C0F5C6D1C31
:10826000E41C002FE6D100207E490880F9F7CEFEFD
:1082700000207D4908807349088000BFF9F72BFA78
:1082800074480088012830D18348807A8249497A2D
:10829000814A127A804BDB79CDE90432CDE90610B0
:1082A0007D4880797C4949797B4A12797A4BDB7821
:1082B000CDE90032CDE90210774883784278017821
:1082C0002846FAF710F800F03000302802D00120DC
:1082D000634908806248008810B900205D49088021
:1082E0000020604908806049088001E0A6E069E05C
:1082F0005C48008801280AD1FAF709F95848008833
:1083000010B9002058490880002055490880564877
:108310000088C828B2DB4B48008838B30026012407
:108320002A20F8F747F900BFF9F7D5F9454830F8A2
:10833000140040F2E731884203D12620F8F73AF9D9
:1083400007E0404931F8140004F095FC2020F8F7CC
:1083500031F900203B4921F81400641C08460088CC
:10836000401EA042E0D20020088012E0701CC6B27D
:108370002A20F8F71FF9FF2004F07DFC052E05DD0B
:108380000120374908803549088002E0002034493F
:108390000880012403E000202B490855641C40F2AA
:1083A00026208442F7D9012404E00020254921F841
:1083B0001400641C40F226208442F6D90D20F8F700
:1083C000F9F81EE035480088062811D1002033490D
:1083D00008801D488078302802D131A004F0C1FC0B
:1083E0001948807832280CD120A004F0BAFC08E0AB
:1083F00019480088012804D118490880002016492E
:1084000008801648008800283FF401AF144800880F
:10841000012813D12349087000201C4908706420EA
:1084200004F034FA2A20F8F7C5F82120F8F7C2F84A
:108430000D20F8F7BFF801201B49087008B0BDE80F
:10844000F0810000580100200A0B002028010020C4
:10845000200100202C0000203600002034000020E5
:108460000C00002044000020000000202A49534F47
:10847000203531392D3420285341452D4A313835A6
:108480003020565057290D00C7000020570000200B
:108490005100002032000020400A00201C00002073
:1084A0002A310D00560000205400002010B5002095
:1084B000FE4908800120FE49087000BFF9F70BF95A
:1084C000FC480088012877D1F9F705F90120FDF76C
:1084D00023FEF948008818B901216420FEF753F9FA
:1084E000F548008801282AD10020F3490880EF4888
:1084F0000088401CED490880C82004F0D4F9012010
:10850000FDF70AFEEC48008818B901216420FEF747
:108510003AF9E9480088012807D1FF20E749488057
:10852000012008800020E4490880E04800880528F0
:1085300008DD0120E2490880DF49088002E00020D0
:10854000DA49088001242A20F8F734F800BFF9F747
:10855000C2F8DA4830F8140040F2E731884203D11B
:108560002620F8F727F80BE0D44931F8140004F07E
:1085700082FB2020F8F71EF80020D04921F81400D3
:10858000601C04B2CD480088A042E0DA0020CB494C
:108590000880012404E00020CA490855601C04B288
:1085A00040F226208442F6DD0020C24908800D20DA
:1085B000F8F700F820E0FFE7C3480088062812D14A
:1085C0000020C1490880BF488078302803D1AFF22D
:1085D000301004F0C6FBBB48807832280CD1BBA019
:1085E00004F0BFFB08E0C0480088012804D1B4496A
:1085F00008800020BC490880B148008820B9AE48F6
:10860000008800283FF45AAFAB480088012813D1F6
:10861000B64908700020A6490870642004F036F9B5
:108620002A20F7F7C7FF2120F7F7C4FF0D20F7F73F
:10863000C1FF0120AE49087010BD13B5FAB000208B
:108640001190109001209A490870AAA07B9A7A99FB
:1086500004F060F80020769008E0002112AA7698D5
:1086600022F810107698401CC0B276907698C828F0
:10867000F3DB0020A5490870A5490870799017E040
:10868000002078900EE00021799800EBC00202EB08
:108690000010A04A02EBC002789822F810107898D7
:1086A000401C789078986328EDD37998401C799095
:1086B00079980928E4D300BFF9F70DF800207990E4
:1086C00006E00021944A799811547998401C7990D9
:1086D00079980928F5D37748008801287ED1794810
:1086E000C078502802D10120109001E000201090A5
:1086F00000208A4908701098002870D07148407F87
:1087000040B2069004F00FFC04466E48007F40B271
:10871000069004F008FC04EB0010C0B20F9069480A
:10872000807E40B2069004F0FEFB04466548407E21
:1087300040B2069004F0F7FB04EB0010C0B20E90BC
:108740006048C07D40B2069004F0EDFB04465D48F1
:10875000807D40B2069004F0E6FB04EB0010C0B24E
:108760000D905848007D40B2069004F0DCFB0446B2
:108770005448C07C40B2069004F0D5FB04EB0010D6
:10878000C0B20C904F48407C40B2069004F0CBFB46
:1087900004464C48007C40B2069004F0C4FB04EB55
:1087A0000010C0B20B904748807B40B2069004F0A6
:1087B000BAFB04464348407B40B2069004F0B3FB4A
:1087C00004EB0010C0B20A903E48C07A40B2069056
:1087D00004F0A9FB04463B48807A01E07CE33CE0DE
:1087E00040B2069004F09FFB04EB0010C0B2099069
:1087F0003448007A40B2069004F095FB04463148B4
:10880000C07940B2069004F08EFB04EB0010C0B2B9
:1088100008902C48407940B2069004F084FB04464E
:108820002848007940B2069004F07DFB04EB00106C
:10883000C0B20790DDE90C23DDE90E10CDE902237B
:10884000CDE90410DDE90A01CDE900017A9840B2D2
:1088500007A90EC9FDF7E0F9D5E01A48807E40B2BD
:10886000079004F060FB04461648407E40B2079033
:1088700004F059FB04EB0010C0B20F901148C07D0A
:1088800040B2079004F04FFB04460E48807D40B292
:10889000079004F048FB04EB0010C0B20E900948AA
:1088A000007D40B2079004F03EFB39E02400002038
:1088B00057000020320000200C000020580100204A
:1088C000340000200A0B00201C0000202A49534FCE
:1088D000203531392D3420285341452D4A31383542
:1088E000302050574D290D00360000205600002042
:1088F00054000020454F42445F43414E2049643DAF
:10890000202578204164723D20257800FC0000205D
:10891000FD000020122300200A2B0020F800002078
:108920000446FE48C07C40B2079004F0FCFA04EB19
:108930000010C0B20D90F948407C40B2079004F09E
:10894000F2FA0446F548007C40B2079004F0EBFAD6
:1089500004EB0010C0B20C90F048807B40B207904E
:1089600004F0E1FA0446ED48407B40B2079004F081
:10897000DAFA04EB0010C0B20B90E848C07A40B2BB
:10898000079004F0D0FA0446E448807A40B2079099
:1089900004F0C9FA04EB0010C0B20A90DF48007A74
:1089A00040B2079004F0BFFA0446DC48C07940B2F8
:1089B000079004F0B8FA04EB0010C0B20990D74851
:1089C000407940B2079004F0AEFA0446D3480079EB
:1089D00040B2079004F0A7FA04EB0010C0B2089070
:1089E000DDE90C23DDE90E10CDE90223CDE9041009
:1089F000DDE90A01CDE900017A9840B2DDE90823FA
:108A00007B99FDF709F90020C549088000BFF8F7F8
:108A100062FE109818B1C348007800B103E0C04866
:108A200000883728F3DB00BF0020BD490880BD481F
:108A3000007800287ED000BFF8F74DFE0020799026
:108A400009E0B9497998085C022801D1B549087054
:108A50007998401C799079980928F2D30020799070
:108A600011E0B1497998085C782809D10220AD4914
:108A700008700020AA4908800021AB4A7998115457
:108A80007998401C799079980928EAD30020799048
:108A900075E1A5497998085C21287CD10220A1497B
:108AA000087000209E49088000219F4A799811543F
:108AB000642003F0F8FE109800286DD09748407F9E
:108AC00040B2069004F02FFA04469448007F40B26A
:108AD000069004F028FA04EB0010C0B20F908F4803
:108AE000807E40B2069004F01EFA04468B48407E19
:108AF00040B2069004F017FA04EB0010C0B20E90DA
:108B00008648C07D40B2069004F00DFA04468348C2
:108B1000807D40B2069004F006FA04EB0010C0B26B
:108B20000D907E48007D40B2069004F0FCF90446AA
:108B30007A4800E032E1C07C40B2069004F0F3F9DC
:108B400004EB0010C0B20C907448407C40B2069018
:108B500004F0E9F904467148007C40B2069004F044
:108B6000E2F904EB0010C0B20B906C48807B40B27D
:108B7000069004F0D8F904466848407B40B206905D
:108B800004F0D1F904EB0010C0B20A906348C07A37
:108B900040B2069001E0EFE041E004F0C4F9044681
:108BA0005E48807A40B2069004F0BDF904EB0010F4
:108BB000C0B209905948007A40B2069004F0B3F967
:108BC00004465648C07940B2069004F0ACF904EB74
:108BD0000010C0B208905148407940B2069004F0AD
:108BE000A2F904464D48007940B2069004F09BF982
:108BF00004EB0010C0B20790DDE90C23DDE90E1094
:108C0000CDE90223CDE90410DDE90A01CDE9000137
:108C10007A9840B207A90EC9FCF7FEFFACE03F48C6
:108C2000807E40B2079004F07EF904463B48407EC7
:108C300040B2079004F077F904EB0010C0B20F9037
:108C40003648C07D40B2079004F06DF904463348C1
:108C5000807D40B2079004F066F904EB0010C0B2CA
:108C60000E902E48007D40B2079004F05CF9044657
:108C70002A48C07C40B2079004F055F904EB00107C
:108C8000C0B20D902548407C40B2079004F04BF9EB
:108C900004462248007C40B2079004F044F904EBFB
:108CA0000010C0B20C901D48807B40B2079004F0C9
:108CB0003AF904461948407B40B2079004F033F972
:108CC00004EB0010C0B20B901448C07A40B2079079
:108CD00004F029F904461148807A40B2079004F064
:108CE00022F904EB0010C0B20A900C48007A40B29E
:108CF000079004F018F904460848C07940B207907C
:108D000004F011F904EB0010C0B209900348407957
:108D100040B2079004F007F9044607E00A0B002070
:108D200000000020F80000200A2B0020FE480079F7
:108D300040B2079004F0F7F804EB0010C0B20890BE
:108D4000DDE90C23DDE90E10CDE90223CDE90410A5
:108D5000DDE90A01CDE90001799800EBC00101EBE2
:108D60000010F24911F83000079001467A9840B29D
:108D7000DDE90823FCF750FF7998401C7990799839
:108D80000928FFF486AEEA48008841F2883188421B
:108D900004DAE848007802283FF44EAE0020E649A5
:108DA00008800120E5490880002077907690E1480E
:108DB0000078012868D10020119000BFE048DF4909
:108DC0000988405C012842D1779848B16FF00202CF
:108DD0007698411CC9B2769112A921F8102001E0C1
:108DE00001207790D548018801EBC10000EB01100C
:108DF000CE4931F8300002B27698411CC9B2769162
:108E000012A921F810200120799000BFF8F763FC27
:108E1000CA48018801EBC10000EB0110C34901EB16
:108E2000C001799831F8100002B27698411CC9B29D
:108E3000769112A921F810207998401C7990C148A8
:108E4000BE49098830F8111079988142DED200209D
:108E5000BB49BA4A12888854B8480088401CB749B0
:108E60000880084600880928A8DB6FF0030276987E
:108E7000411CC9B2769112A921F81020682212A8CB
:108E8000769903F017FF09E01198401CC0B21190C9
:108E90002A20F7F78FFBFF2003F0EDFE119805283D
:108EA00004DD0120A8490880A849088001207990A4
:108EB00006E000219C4A799811547998401C7990D9
:108EC00040F2262179988842F3D90021A0480180F8
:108ED0000D20F7F76FFBD6E19E48008806283AD1AF
:108EE00000209C49088090488078302803D1AFF654
:108EF000502003F036FF8C4880783228EBD196481A
:108F000000780838082825D2DFE800F004080C10A3
:108F100014181C2091A003F024FF1BE096A003F07E
:108F200020FF17E09BA003F01CFF13E0A0A003F0BC
:108F300018FF0FE0A5A003F014FF0BE0AAA003F0B8
:108F400010FF07E0AFA003F00CFF03E0B4A003F0B4
:108F500008FF00BF97E10020B849088000BFF8F77C
:108F6000BAFB012003F092FC7948008818B9B34895
:108F700000881428F3DDB14800881428ABDB0020FA
:108F80006C490870744800780C280BD0724800783F
:108F90000D2807D0704800780E2803D06E4800785E
:108FA0000F2810D10020029003900490059010200B
:108FB000F82122230322CDE900107A9840B27B9950
:108FC000FCF72AFE0DE0002002900390049005902B
:108FD00000900123022201907A9840B27B99FCF71D
:108FE0001BFE00205249088000BFF8F774FB504870
:108FF00000883728F9DB00204D4908804D4800786B
:10900000A0B300BFF8F767FB0020799009E04C4956
:109010007998085C022801D1464908707998401C6B
:10902000799079980928F2D30020799011E0444989
:109030007998085C782809D102203E490870002000
:109040003B49088000213E4A799811547998401C88
:10905000799079980928EAD33548008841F2883117
:10906000884203DA334800780228CBD00020324906
:1090700008800120314908800020779076902D48A3
:10908000007801284ED10020119000BF2C482B49B8
:109090000988405C012842D1779848B16FF00202FC
:1090A0007699481CC0B2769012A820F8112001E0F1
:1090B000012077902148008800EBC00101EB0010EF
:1090C0001A4931F8300002B27698411CC9B2769143
:1090D00012A921F810200120799000BFF8F7FBFABF
:1090E0001648018801EBC10000EB01100F4901EBAC
:1090F000C001799831F8100002B27698411CC9B2CB
:10910000769112A921F810207998401C79900D4889
:109110000A49098830F8111079988142DED200207E
:1091200007498DE0A3E000000A0B00201223002075
:1091300000000020F800002034000020240000205F
:109140000A2B0020F62A00200C0000203600002008
:10915000320000201C000020510000202A49534FFB
:109160002031353736352D34202843414E203131DA
:109170002D323530290D00002A49534F2031353723
:1091800036352D34202843414E2031312D353030B5
:10919000290D00002A49534F2031353736352D34FB
:1091A000202843414E2032392D323530290D000020
:1091B0002A49534F2031353736352D342028434145
:1091C0004E2032392D353030290D00002A49534FB9
:1091D0002032373134352D34202843414E2031316F
:1091E0002D323530290D00002A49534F20323731B6
:1091F00034352D34202843414E2031312D35303047
:10920000290D00002A49534F2032373134352D348F
:10921000202843414E2032392D323530290D0000AF
:109220002A49534F2032373134352D3420284341D9
:109230004E2032392D353030290D00000A00002033
:10924000F94A12888854F8480088401CF64908807A
:10925000084600880928FFF619AF6FF003027698D8
:10926000411CC9B2769112A921F8102003E011988F
:10927000401CC0B211901198052804DD0120EB4973
:109280000880EB4908807A981D2818D111E0E94838
:109290000078801CC0B20F90E748E6490978405C2E
:1092A0000E900F99FCF713FDE2480078401CE1494D
:1092B0000870E0480078E14909788842E7DBDB483C
:1092C000008820B9DA48008800283FF4F5A9D7487B
:1092D0000088012814D10121D94801700020D94902
:1092E0000870642003F0D2FA2A20F7F763F92120EE
:1092F000F7F760F90D20F7F75DF90120D249087002
:109300007CB010BDF0B587B001260027CF480068BB
:1093100006904FF4FC60CE490880401C4880401CF9
:109320008880401CC880401C0881401C4881401C2B
:109330008881401CC8810020C0490870002403E0D7
:109340000020BD490855641C0A2CF9D30E220621C1
:109350000120F7F704FF0821BE4804F03EFA0A2076
:1093600003F0A1FA0020B1490880002403E00020A6
:10937000B9490855641C092CF9D300240FE00025D5
:109380000AE0002004EBC40101EB0411B34A02EB34
:10939000C10121F815006D1C632DF2D3641C092C4A
:1093A000EDD3BDF81800AE49FAF7ACFB0020AD498B
:1093B0000870AD490870AD490870029003900490A0
:1093C0000590009001230222DF2101900B20FCF781
:1093D00023FC0020A649088001E0F8F77CF9A448A6
:1093E0000088192803DCA04800780028F5D0A048A0
:1093F0000088192810DD01209A49087000219D4835
:1094000006F057FB01219B4806F053FB02219948C7
:1094100006F04FFBFBF7FDF80020974908709449D0
:10942000088000BFF8F757F991480088B0F5FA7F37
:1094300006DA9148007818B98A4800780028F1D0F7
:1094400088480078012801D1052631E08A48007853
:1094500001282CD1744908807449088000BF7E48D7
:1094600071490988405C70B16F48008800EBC00109
:1094700001EB0010794901EBC0004088412802D17E
:1094800000206A49088068480088401C66490880B6
:10949000084600880928E2DB64480088012801D1D9
:1094A000022605E00B2708207449087000E0022618
:1094B000022E7DD1002403E0002067490855641C7A
:1094C000092CF9D300240FE000250AE0002004EB6A
:1094D000C40101EB0411614A02EBC10121F815003E
:1094E0006D1C632DF2D3641C092CEDD300205D4963
:1094F00008705D49087002900390049005900090F8
:1095000001230222332101901D20FCF785FB00205E
:109510005749088001E0F8F7DEF855480088192817
:1095200003DC514800780028F5D0514800881928FC
:1095300010DD01204B49087000214E4806F0B9FAB1
:1095400001214C4806F0B5FA02214A4806F0B1FA6A
:10955000FBF75FF80020484908704549088000BFC4
:10956000F8F7B9F842480088B0F5FA7F06DA4248C1
:10957000007818B93B4800780028F1D02F480078CF
:10958000002810DD00242D4800782A49087006E0E4
:10959000A21CD1B2284A105DFCF799FB641C274835
:1095A00000788442F4D33448007801282ED100E0BA
:1095B0002DE01D4908801D49088000BF26481A4932
:1095C0000988405C70B11848008800EBC00101EBCD
:1095D0000010224901EBC0004088412802D1002040
:1095E0001249088010480088401C0F49088008462E
:1095F00000880928E2DB0D480088012801D10326F4
:1096000005E01D270A201D49087000E00326032EEF
:109610007DD1002403E000200F490855641C092C6B
:10962000F9D300243CE00000240000200C000020BE
:1096300036000020F7000020F8220020F60000206D
:109640005600002057000020540000204C030D0855
:1096500002230020001802400A2B002012230020C1
:1096600041480C08F9000020FB000020FA0000200F
:109670000000002000680040F80000205100002099
:1096800000250AE0002004EBC40101EB0411F84AB4
:1096900002EBC10121F815006D1C632DF2D3641C8F
:1096A000092CEDD3BDF81800F249FAF72BFA002087
:1096B000F1490870F1490870002102910391049169
:1096C00010200591F82122230322CDE90010DF218B
:1096D0000B20FCF7A1FA0020E949088001E0F7F728
:1096E000FAFFE7480088192803DCE34800780028DF
:1096F000F5D0E3480088192812DD0120E1490870FF
:109700000021E14806F0D5F90121DF4800E04DE0F5
:1097100006F0CFF90221DC4806F0CBF9FAF779FF21
:109720000020DA490870D649088000BFF7F7D3FF58
:10973000D3480088B0F5FA7F06DAD448007818B923
:10974000D04800780028F1D0D048007801282CD1EA
:10975000CF490880CF49088000BFCF48CC4909884D
:10976000405C70B1CA48008800EBC00101EB0010FA
:10977000BF4901EBC0004088622802D10020C549E2
:109780000880C3480088401CC149088008460088FA
:109790000928E2DBBF480088012801D1042605E042
:1097A0000B270C20BD49087000E00426042E7DD153
:1097B000002403E00020B8490855641C092CF9D3A3
:1097C00000240FE000250AE0002004EBC40101EBB7
:1097D0000411A74A02EBC10121F815006D1C632D8D
:1097E000F2D3641C092CEDD30020AD49087000248D
:1097F00003E00020AB490855641C0A2CF9D3002073
:10980000A04908709C49087002900390049005904C
:109810001020F82122230322CDE9001033211D203E
:10982000FCF7FAF900209649088001E0F7F753FFAA
:1098300093480088192803DC8F4800780028F5D069
:109840008F480088192810DD01208E4908700021FA
:109850008D4806F02EF901218B4806F02AF90221E5
:10986000894806F026F9FAF7D4FE002087490870E7
:109870008349088000BFF7F72EFF81480088B0F5C4
:10988000FA7F09DA8148007830B97E48007818B943
:10989000854800780028EED081480078002811DD46
:1098A00000247F4800788149087007E03CE0A21C52
:1098B000D1B27C4A105DFCF70AFA641C7848007843
:1098C0008442F4D37148007801282CD17049088073
:1098D0007049088000BF70486D490988405C70B1CC
:1098E0006B48008800EBC00101EB0010604901EB00
:1098F000C0004088622802D1002066490880644880
:109900000088401C62490880084600880928E2DB7C
:1099100060480088012801D1002605E01D270E209F
:109920005E49087000E00026052E6FD1002403E098
:10993000002059490855641C092CF9D300240FE074
:1099400000250AE0002004EBC40101EB0411484AA1
:1099500002EBC10121F815006D1C632DF2D3641CCC
:10996000092CEDD3BDF81A004249FAF7CBF80020D4
:1099700044490870404908704049087002900390BB
:1099800004900590009001230222DF2101900B201A
:10999000FCF742F900203A49088001E0F7F79BFE06
:1099A00037480088192803DC334800780028F5D0B0
:1099B00033480088192810DD012032490870002141
:1099C000314806F076F801212F4806F072F802219E
:1099D0002D4806F06EF8FAF71CFE00202B4908709F
:1099E0002749088000BFF7F776FE25480088B0F5C4
:1099F000FA7F06DA2548007818B92248007800284E
:109A0000F1D020480078012801D1002651E01F48FC
:109A1000007801284CD11E4908801E49088000BFEB
:109A20001D481B490988405C70B11948008800EB4B
:109A3000C00101EB00100E4901EBC0004088412835
:109A400002D100201349088011480088401C1049A9
:109A50000880084600880928E2DB0E4800880128B3
:109A600001D1062625E00B2709200C49087020E0CB
:109A70001223002041480C08FB000020FA000020BF
:109A800000000020F900002000680040F8000020DD
:109A9000240000200C0000200A2B00205100002090
:109AA000F6000020F822002053000020F7000020DC
:109AB0000626062E7BD1002403E00020FE4908552F
:109AC000641C092CF9D300240FE000250AE00020D3
:109AD00004EBC40101EB0411F84A02EBC10121F8C7
:109AE00015006D1C632DF2D3641C092CEDD30020EE
:109AF000F3490870002403E00020F2490855641C73
:109B00000A2CF9D30020F0490870F049087002903F
:109B100003900490059000900123022233210190CC
:109B20001D20FCF779F80020E949088001E0F7F7EB
:109B3000D2FDE7480088192803DCE44800780028B3
:109B4000F5D0E3480088192810DD0120DE490870AF
:109B50000021E04805F0ADFF0121DE4805F0A9FF36
:109B60000221DC4805F0A5FFFAF753FD0020DA4991
:109B70000870D749088000BFF7F7ADFDD4480088CA
:109B8000B0F5FA7F09DAD448007830B9CE480078C9
:109B900018B9D24800780028EED0C94800780028CB
:109BA00011DD0024C6480078CD49087007E03CE08C
:109BB000A21CD1B2C34A105DFCF789F8641CC048EE
:109BC00000788442F4D3C448007801282CD1C549D8
:109BD0000880C549088000BFB748C2490988405C71
:109BE00070B1C048008800EBC00101EB0010B34920
:109BF00001EBC0004088412802D10020BA4908800A
:109C0000B8480088401CB7490880084600880928E1
:109C1000E2DBB5480088012801D1072605E01D27B1
:109C20000B20B249087000E00726072E7DD10024E2
:109C300003E00020A0490855641C092CF9D3002436
:109C40000FE000250AE0002004EBC40101EB041141
:109C50009A4A02EBC10121F815006D1C632DF2D365
:109C6000641C092CEDD3BDF81A00A149F9F74AFF8D
:109C7000002095490870954908709E490870029027
:109C80000390049005901020F82122230322CDE9AF
:109C90000010DF210B20FBF7BFFF00208C4908805C
:109CA00001E0F7F718FD8A480088192803DC874887
:109CB00000780028F5D086480088192810DD01209A
:109CC000814908700021834805F0F3FE0121814895
:109CD00005F0EFFE02217F4805F0EBFEFAF799FC54
:109CE00000207D4908707A49088000BFF7F7F3FC2F
:109CF00077480088B0F5FA7F06DA7748007818B917
:109D0000714800780028F1D07348007801282ED1DE
:109D1000744908807449088000BF67487149098800
:109D2000405C80B16F48008800E021E000EBC0019A
:109D300001EB0010614901EBC0004088622802D1AC
:109D400000206949088067480088401C65490880F0
:109D5000084600880928E0DB63480088012801D113
:109D6000082605E00B270D206049087000E0082652
:109D7000082E7DD1002403E000204F490855641CC3
:109D8000092CF9D300240FE000250AE0002004EBA1
:109D9000C40101EB0411494A02EBC10121F815008D
:109DA0006D1C632DF2D3641C092CEDD300204449B3
:109DB0000870002403E0002042490855641C0A2C66
:109DC000F9D3002040490870404908700290039080
:109DD000049005901020F82122230322CDE90010E1
:109DE00033211D20FBF718FF00203949088001E0CE
:109DF000F7F771FC36480088192803DC33480078EF
:109E00000028F5D032480088192810DD01202E499D
:109E1000087000212F4805F04CFE01212D4805F067
:109E200048FE02212B4805F044FEFAF7F2FB002021
:109E3000294908702649088000BFF7F74CFC2448E0
:109E40000088B0F5FA7F09DA2348007830B91E4857
:109E5000007818B9214800780028EED0184800781A
:109E6000002811DD0024164800781D49087007E01D
:109E700057E0A21CD1B2134A105DFBF728FF641C07
:109E80000F4800788442F4D31348007801284DD15C
:109E9000144908801449088000BF074811490988FF
:109EA000405C48B30F48008800EBC00101EB001094
:109EB000024901EBC00020E00A2B00201223002001
:109EC000F6000020F8220020F9000020FB0000200E
:109ED0000000002000680040F8000020530000202F
:109EE000F7000020240000200C000020510000207A
:109EF00041480C08FA00002005E04088622802D1A1
:109F00000020FE490880FE480088401CFC4908806B
:109F1000084600880928C0DBF8480088012801D1DC
:109F2000002603E01D270F20F6490870384607B0C9
:109F3000F0BD2DE9F0474FF0000800240025002671
:109F40003A27A146A2460020EC490880EE49088045
:109F5000EE490870487000BF0020ED490880ED49C7
:109F6000088000BFF7F7B7FBEA480088012803DA4A
:109F7000E74800888742F5DAE5480088874202DC36
:109F80000120DE490880DD48008800284FD1012EDD
:109F90000ADB601C04B240F2E730DB4921F8140010
:109FA0000020DA4908704870601C04B2DA48008862
:109FB000D54921F81400D5480078D4494978084497
:109FC000D2490870D44800784870D348007800F02F
:109FD0003F08D1480088802803DDCF4800888928C1
:109FE0000BDBCE48007800287CD0CB480088C02806
:109FF00078DDC9480088C9287FDA02F045FD601C79
:10A0000004B2C5480088C04921F81400BF48007850
:10A01000BE4949780844BD490870BF480078487077
:10A02000BD480088F12803D00220B449088067E0C9
:10A0300002F02AFD601C04B2B7480088B24921F83A
:10A040001400B2480078B14949780844AF49087013
:10A05000B14800784870002500BF02F015FD601C73
:10A0600004B2681C05B2AC480088A74921F8140066
:10A07000A6480078A54949780844A4490870A6482C
:10A08000007848709D48008808B9A845E5DA701C3A
:10A0900006B29A480088012803D104209749088015
:10A0A0002EE099490C80994800789849497888426F
:10A0B00001D04FF0010A601B401C934931F8100099
:10A0C0007F2810D1601BC01C31F8100078280AD1FD
:10A0D000601B11F8109041F28837601B001F04B21A
:10A0E0000C800DE009E03A2F0AD0601B864931F858
:10A0F0001000484504D13A2702E002207F49088039
:10A100007E48008800283FF427AF7C48008801285B
:10A1100004D1012E02DB00207849088077480088AE
:10A12000022801D1FFF705FFBAF1010F02D101208A
:10A1300072490880BDE8F08710B5012078490870A1
:10A1400000206F49088000BFF7F7C5FA0F2002F022
:10A15000AAFB74480088012870D1F7F7BCFA0521E2
:10A16000012002F0AEFCFFF7E4FE644800880128FD
:10A170003BD1962002F097FB61480088401C604963
:10A18000088000205D4908800121052002F0F1FCD3
:10A19000FFF7CFFE59480088012808D1FF205A490F
:10A1A00048800120088000205449088013E03220B4
:10A1B00002F079FB0521012002F083FCFFF7B9FED4
:10A1C0004E48008838B1FF204F4948800120088060
:10A1D00000204A4908804A480088052808DB0120F9
:10A1E000514908804549088002E000204449088020
:10A1F00001242A20F6F7DEF900BFF7F76CFA42488F
:10A2000030F8140040F2E731884203D12620F6F7F7
:10A21000D1F90BE03C4931F8140002F02CFD20206C
:10A22000F6F7C8F90020384921F81400601C04B280
:10A2300035480088A042E0DA012405E011E0002062
:10A240003A490855601C04B240F226208442F6DDEB
:10A2500000202D490880334908800D20F6F7AAF91F
:10A2600095E033480088012812D1052102F029FC2D
:10A2700001202D4908802A20F6F79CF9012002F0E0
:10A28000ADFC0D20F6F796F90020294908807EE004
:10A2900028480088062811D1002026490880234834
:10A2A0008078302802D1244802F05BFD1F48807876
:10A2B00032286CD121A002F054FD68E0002025492D
:10A2C000088000BFF7F707FA012002F0DFFA15480F
:10A2D000008818B91F4800881928F3DD1D48008838
:10A2E00019284BDB0121052002F043FCFFF721FE7A
:10A2F0000248008801283ED101482DE00C000020D2
:10A3000024000020510000205801002029010020D5
:10A310000000002022000020080600202B01002061
:10A320005700002032000020340000200A0B0020DB
:10A33000360000201C000020A0840C082A49534F3E
:10A340002031343233302D3420284B5732303030E6
:10A35000290D00000A0000200088401CFB490880ED
:10A360004FF4FA7002F09FFA0121052002F001FC7F
:10A37000FFF7DFFD02E00020F4490880F348008881
:10A38000052804DB0120F2490880F2490880F048E2
:10A39000008820B9EF48008800283FF4D5AEED488A
:10A3A0000088012813D1EC4908700020EB4908709F
:10A3B000642002F06BFA2A20F6F7FCF82120F6F769
:10A3C000F9F80D20F6F7F6F80120E549087010BD00
:10A3D00010B50020E3490880E349088000BFF7F783
:10A3E0007AF9E1480088012803DADE480088372836
:10A3F000F5DDDC480088372801DB012010BD002096
:10A40000FCE72DE9F0410646012400274FF0000843
:10A410000020D0490880D4490880D2490880D34917
:10A420000870487000BFF7F756F9CF480088012838
:10A4300003DACC4800888642F5DACA4800888642AA
:10A4400002DC0120C3490880A5B2C2480088002868
:10A4500074D1C7480088C74921F81400084610F88D
:10A460001400C2494870F7F736F900BFFFF7B0FF94
:10A470000746BC480088152827DB37BBBD4830F8A5
:10A480001500482805D1BB49681C31F810006B281D
:10A4900005D02CB20020B5490870487015E0B348CB
:10A4A0000078B44931F81410884201D04FF0010807
:10A4B000601C04B240F2E730AE4921F81400601C81
:10A4C00085B20020A949087048708FB9601C04B299
:10A4D000A7480088A74921F81400A4480078A34998
:10A4E00049780844A1490870A24810F8140048703F
:10A4F000B4F5FA7F01DC002FB8D0B8F1010F02D11A
:10A500000120944908809B4830F81500482805D15F
:10A510009849681C31F810006B2803D001208D4940
:10A52000088009E091480078924931F81410884277
:10A5300002D00120874908808E490C80BDE8F08157
:10A5400010B501208549087000BFF7F7C4F87F49AE
:10A55000098801EBC10202EB0111192202EB410152
:10A5600088B202F0A0F984480088012870D1F7F77A
:10A57000B2F80521012002F0A4FA3C20FFF741FFC8
:10A5800074480088012838D170480088401C6F4901
:10A59000088000206F490880C82002F084F901215A
:10A5A000052002F0E6FA3C20FFF72BFF69480088FF
:10A5B000012805D1FF206F4948800120088012E062
:10A5C000192002F070F90521012002F07AFA3C20EE
:10A5D000FFF717FF5F480088012804D1FF20654975
:10A5E00048800120088059480088052808DB0120A0
:10A5F000574908805749088002E0002053490880E5
:10A6000001242A20F5F7D6FF00BFF7F764F8594870
:10A6100030F8140040F2E731884203D12620F5F7E4
:10A62000C9FF0BE0534931F8140002F024FB20204D
:10A63000F5F7C0FF00204F4921F81400641C4D4875
:10A640000088A042E1DA00204A490880012404E0A1
:10A650000EE0002049490855641C40F2262084423F
:10A66000F7DD0020444908800D20F5F7A3FF3FE007
:10A6700043480088012805D1354908800020404919
:10A68000088035E03F480088062811D100203D4968
:10A6900008803A488078302802D13B4802F061FBBC
:10A6A00036488078322823D138A002F05AFB1FE0C8
:10A6B0000121052002F05DFA3C20FFF7A2FE2548AB
:10A6C0000088012805D121480088401C1F490880C6
:10A6D00002E000201D49088000201E4908801B4818
:10A6E0000088052804DB01201949088019490880E1
:10A6F0001748008800283FF428AF16480088012832
:10A7000013D115490870002014490870642002F024
:10A71000BDF82A20F5F74EFF2120F5F74BFF0D205D
:10A72000F5F748FF01200E49087010BDF8B5044642
:10A73000002500BF06E04FF6FF70194921F815000B
:10A74000681C05B2282DF6DD002531E0240000202C
:10A75000340000200C00002056000020570000208C
:10A7600054000020000000202200002029010020C9
:10A770000806002058010020320000200A0B0020AB
:10A78000360000201C000020A0840C082A49534FEA
:10A7900020393134312D32202843415242290D00D5
:10A7A000F00900200020FD4921F81500681C05B2C1
:10A7B000B5F5FA7FF6DDC220F949088033204880DC
:10A7C000F12088800120C8800881084600884988D7
:10A7D0000844F34989880844F149C9880844F04984
:10A7E00009890844EE4948810020F7F71DF9002047
:10A7F000F7F71FF9132002F073F80CB1022C20D1E7
:10A800000020E849088007E0F6F765FFE648007891
:10A81000012801D10020F8BDE2480088FA28F3DDC4
:10A82000DF48807805230822002100900420F7F7F4
:10A83000A5FAF9F758F8DC480078012801D1002082
:10A84000E9E7DA480088002844D10CB1022C41D154
:10A850000020D4490880D649088000BFF6F73BFFA6
:10A86000D3480088022803DACE4800885A28F5DD4C
:10A87000CC4800885A2804DB0120CC4908800020FD
:10A88000C9E740F6C410FCF7E8FBC44807788678AF
:10A89000C6F1FF00C7490880C7490880C74908803A
:10A8A00002F0F2F802F0F0F8C0480088012801D167
:10A8B0000020B0E7082F01D1082E03D0942F03D138
:10A8C000942E01D10120A6E78F2E01D10220A2E70C
:10A8D0000020A0E70CB1012C7BD10020B3490880F7
:10A8E0000025F6F7F8FE192211460420F7F7D0F9F3
:10A8F0000022082142F6A000F7F744F8C120AD4934
:10A900000880AD490880AD49088002F0BDF8C1203B
:10A91000AB4908804FF4FA70FCF79FFBA0484088D1
:10A92000A4490880A4490880A449088002F0ACF832
:10A930009B484088A24909880844A14908804FF4EF
:10A94000FA70FCF78AFB964880889A4908809A49F1
:10A9500008809A49088002F097F8914880889849C1
:10A9600009880844964908804FF4FA70FCF775FB93
:10A97000812090490880904908809049088002F021
:10A9800083F88F48008881308D4908804FF4FA7031
:10A99000FCF763FB8A48007886490880864908806E
:10A9A0008649088002F070F8002080490880FFF78F
:10A9B000C0FA7E48008848B982480089C12803D07F
:10A9C000804880898F2802D1032024E701E00020FD
:10A9D00021E700201FE72DE9F041074601207A49D1
:10A9E00008807A4908700020794908700120794967
:10A9F0000870FDF736FB0024002072490880764974
:10AA000008806A4908807549088075490880754939
:10AA100008807549088075490870002500BF744892
:10AA2000005D00B95CB17248005D012807D0704834
:10AA3000005D0B2803D06E48005D0C287ED1FDF729
:10AA400005FB6B48005D0B2807D16AA001F062FE90
:10AA50000220FFF76BFE054612E06548005D0C28FA
:10AA600007D16FA001F056FE0120FFF75FFE0546FB
:10AA700006E072A001F04EFE0020FFF757FE0546EB
:10AA8000012D04D0022D71D0032D70D1E9E04FF0DB
:10AA9000000808E04FF6FF70414921F8180008F15E
:10AAA00001000FFA80F8B8F1280FF3DD68203C4967
:10AAB00008806A204880F12088800120C88000201A
:10AAC000088108460078897808443549097908449E
:10AAD0003349897908443249097A0844C0B2304977
:10AAE0004881322001F0DFFE0121052002F041F80B
:10AAF0003C20FFF786FC2D480088012838D16420CF
:10AB000001F0D1FE0121052002F033F83C20FFF7CF
:10AB100078FC2648008801282AD1002500203349E6
:10AB200008704FF4FA7001F0BEFE0120FFF7FEFD41
:10AB300005460121052002F01CF800E0FFE0FFF7C8
:10AB4000F8F91A48008898B9AFF6100002F009F930
:10AB50004248007820F04000404908700320234913
:10AB60000870FDF773FAFFF7E7FAE7E078E0E0E056
:10AB70000E48008880B9AFF2EC3002F0F2F83748A6
:10AB8000007820F04000354908700120174908700E
:10AB9000FDF75CFAFFF7D4FCD0E0000008060020C7
:10ABA000F00900200A000020530000200C000020C3
:10ABB000220000200444004004140140044C0040E2
:10ABC0002A000020580100200E000020550000201F
:10ABD00056000020570000202400002034000020F0
:10ABE00036000020320000202C0000205100002000
:10ABF00020010020436865636B2049534F3931348D
:10AC0000312D3220616E642049534F31343233305C
:10AC10002D3420536C6F7720696E69740D0000002D
:10AC2000436865636B2049534F31343233302D34E0
:10AC3000204661737420696E69740D004368656312
:10AC40006B2049534F393134312D3220616E6420ED
:10AC500049534F31343233302D340D00C7000020BA
:10AC600000BF3C2001F01FFE0121052001F081FF03
:10AC7000FFF75FF9C248008880B1142001F013FE8D
:10AC80000121052001F075FFFFF753F9BC4800884A
:10AC9000012803D100250020BA490870B84800886F
:10ACA000002845D1B8480089412821D0642001F00E
:10ACB000FAFD0121052001F05CFFFFF73AF9B248E7
:10ACC0000089412814D0642001F0EDFD0121052008
:10ACD00001F04FFFFFF72DF9AB480089412807D05D
:10ACE00000250020A74908700120A549088025E01B
:10ACF00027B9AFF6B81002F034F80CE0012F0AD1F2
:10AD0000022D03D1A1A002F02CF804E0032D02D102
:10AD1000A5A002F026F8AB48007820F04000A94931
:10AD20000870022097490870FDF790F9FFF704FAC0
:10AD300004E0002500209349087000BF00BFA2482E
:10AD4000005D00B99CB1A048005D02280FD09E486C
:10AD5000005D03280BD09C48005D042807D09A486A
:10AD6000005D052803D09848005D092865D197A0AB
:10AD700001F0D0FCFDF76AF9002D5ED16FF0604064
:10AD8000974908609749086000207D490880FEF7D0
:10AD9000B9FA06467A48008800284AD1002E48D0E1
:10ADA00078480078083808282CD2DFE800F004083A
:10ADB0000D12171C21268C4801F0D3FF22E08A488F
:10ADC0001C3001F0CEFF1DE08748383001F0C9FF8C
:10ADD00018E08548543001F0C4FF13E08248703019
:10ADE00001F0BFFF0EE080488C3001F0BAFF09E0AF
:10ADF0007D48A83001F0B5FF04E07B48C43001F085
:10AE0000B0FF00BF00BF6F48007820F040006D49E0
:10AE100008700021754803F068FC0B2E04D1DF2177
:10AE20003046FDF70AFC08E033213046FDF705FC0B
:10AE300003E000250020534908706348005D00B915
:10AE40001CB16148005D06283ED169A001F062FC9A
:10AE5000FDF7FCF885BBFAF777FF61206A490880A7
:10AE60006A204880F12088800120C8800020088165
:10AE70000520FBF738FB01216420FBF784FC4248E6
:10AE80000089412802D001203D4908803C480088C3
:10AE900090B904255D4801F064FF4A48007820F02D
:10AEA0004000484908700021504803F01EFC04206F
:10AEB00034490870FDF7FAFA31480088012803D1B7
:10AEC000002500202F4908703F48005D00B91CB1E3
:10AED0003D48005D072812D14DA001F01BFCFDF795
:10AEE000B5F865B9FDF71FF92548008808B90625AA
:10AEF00005E00020224908800025224908703248D8
:10AF0000005D082814D148A001F004FC85B96FF059
:10AF10006040334908603349086001F016FA184868
:10AF2000008808B9072503E00025002015490870AE
:10AF3000601CC4B241480078844205DA25B9404813
:10AF4000007800283FF46BAD01F092FD3D4801F020
:10AF500008FF032001F0A7FC01203B4908700020F6
:10AF60003A4908703A4908703A490880BDE8F081CA
:10AF70000120394908707047002037490870704730
:10AF80000C00002051000020580100202A49534F96
:10AF90002031343233302D3420284B57323030308A
:10AFA0002920536C6F770D002A49534F20313432DA
:10AFB00033302D3420284B57323030302920466131
:10AFC00073740D00C70000202001002043686563F2
:10AFD0006B2049534F31353736352D340D00000085
:10AFE000E4000020EC0000205C910C0800140040FC
:10AFF000436865636B205341452D4A313835302015
:10B0000050574D0D00000000F0090020CC880C08BE
:10B01000436865636B205341452D4A3138353020F4
:10B020005650570D00000000436865636B20534184
:10B0300045204A313933392D32310D0028010020A5
:10B0400053000020A0840C0855000020560000206A
:10B05000570000200E0000202B01002030B585B0E5
:10B0600000250024FE482B460F2201210090FA20E3
:10B0700001F0A2FAFB48056018208DF80E000020B0
:10B080008DF80F0001208DF81000F748D0F81C0152
:10B09000C0F34F30ADF80400F348D0F81C014FF670
:10B0A000FF7101EAC000001DADF80600680BADF8A5
:10B0B0000800084600EAC500001DADF80A0000209F
:10B0C000ADF80C0001208DF8110001A804F061FB1F
:10B0D00000BF06E0002004EB4401E44A5054601C29
:10B0E00084B2322CF6DB002405E00020E04921F890
:10B0F0001400601C84B2B4F57A7FF6DB0020DD49D1
:10B100000870DD490880DD49088000BFF6F7E3FAE2
:10B11000DA480088B0F5FA6FF8DB00241CE004EB95
:10B120004400D2490844817804EB4400D04A22F814
:10B13000101004EB4400CD490844417804EB44006E
:10B14000401C22F810104FF0FF3104EB4400801C2B
:10B1500022F81010601C84B204EB4400C349085C60
:10B160000128DCD0002C0FDD601E84B26FF00101DD
:10B1700004EB4400801CBE4A22F81010601C84B20C
:10B1800004EB440084B204E06FF00100B849088089
:10B19000012468222146B64801F08CFD05B030BD7F
:10B1A0002DE9F0438BB04FF000084FF0FF35002041
:10B1B000B349087000240AE00020B24901EB840181
:10B1C0008870B04901EB8401C870601C84B20F2CF8
:10B1D000F2DBA348AC4B012211460090FA2001F0AB
:10B1E000EBF9AA4DAA48056000208DF82700680BEE
:10B1F000ADF82000281200EAC500001DADF82200BD
:10B200000020ADF8240001208DF8290007A804F0E3
:10B21000C0FA00261FE006F10A00C0B28DF8260031
:10B2200006EB8600904901EB80004068C0F34F3088
:10B23000ADF81C0006EB860001EB800040684FF67D
:10B24000FF7101EAC000001DADF81E0007A804F060
:10B25000A0FA701CC6B20E2EDDDB4FF0FF35814820
:10B26000056018208DF8260000208DF827000120A9
:10B270008DF828007C48D0F81C01C0F34F30ADF8A1
:10B280001C007948D0F81C01290C01EAC000001DFF
:10B29000ADF81E00C5F34F30ADF82000084600EAB7
:10B2A000C500001DADF822000020ADF824000120EB
:10B2B0008DF8290007A804F06CFA00206F49088077
:10B2C0004FF4C877E9E16D480088B84244DD6C4826
:10B2D0000078002840DD002437E06A4800EB840055
:10B2E000807880BB00216B4804F0E3FB01216948B2
:10B2F00004F0DFFB0221674804F0DBFBF9F789F972
:10B30000642001F0D0FA01205E4901EB8401C8708D
:10B3100064275D4803903C208DF80800594800EBF5
:10B32000840040788DF81000564810F824108DF8ED
:10B33000111000218DF8121002A90120F8F7A3FFC7
:10B340000120F9F74EF9601C84B24D480078844220
:10B35000C3DB002049490880F6F7BDF94E48008854
:10B3600001287BD100204C4908804C49497948B2DA
:10B3700001F0D9FD81464949097948B201F0D3FD70
:10B3800009EB0010464988704449097A48B201F037
:10B39000CAFD81464149C97948B201F0C4FD09EBB3
:10B3A00000103F4948703D49C97A48B201F0BBFDE1
:10B3B00081463A49897A48B201F0B5FD09EB00109F
:10B3C00037490870084640782E492D4A127801F80E
:10B3D0002200334800782A4A127801EB8201487033
:10B3E00000212848264A127800EB82008170254807
:10B3F000234A127800EB8200C170FF202949204ABD
:10B40000127801F83200FF2126481D4A127800EB1D
:10B41000C2004170FF202349194A127801EBC20192
:10B4200088702049164A127801EBC201C870FF21CA
:10B430001C48134A127800EBC2000171FF20194921
:10B440000F4A127801EBC201487116490C4A127872
:10B4500001EBC20188711349094A25E057E0000059
:10B46000CD570C08E4000020A02000206D690020CA
:10B47000184500203B010020380000200A00002071
:10B480002D010020036A0020F9FFEA1800FFFF00E9
:10B49000EC000020006800402E0000200A0B002075
:10B4A0002E0100203F6A0020127801EBC201C87112
:10B4B0000025FE4840780004FC49097800EB01258E
:10B4C000FB4800780D281FDA00200090F84800782B
:10B4D000801CC2B22B460121002001F06DF8F44817
:10B4E0000078401CF24908702A20F5F763F8F0490B
:10B4F0000978491E88B201F071FB0D20F5F75AF862
:10B500000020EC49088002E0EBA001F02AFCFA4898
:10B510000088012876D1F6F7DEF80020F649088089
:10B52000F648C07845287DD0F448C078652879D0A1
:10B5300000244FE0F24810F8341004EBC400F14A44
:10B5400022F81010EE4800EBC400417804EBC40070
:10B55000401C22F81010EA4800EBC400817804EB8C
:10B56000C400801C22F81010E54800EBC400C1782C
:10B5700004EBC400C01C22F81010E14800EBC4002A
:10B58000017904EBC400001D22F81010DC4800EB28
:10B59000C400417904EBC400401D22F81010D848C3
:10B5A00000EBC400817904EBC400801D22F8101068
:10B5B000D34800EBC400C17904EBC400C01D22F8DD
:10B5C00010104FF0FF3104EBC400083022F81010C7
:10B5D000601C84B2B64800788442ABDB002C13DDDB
:10B5E00004EBC40084B2601E84B26FF00100C54950
:10B5F00021F81400601C84B268222146C14801F081
:10B6000059FB0BE035E00DE06FF00100BD4908800B
:10B61000012468222146BB4801F04CFB0D20F4F7C1
:10B62000C9FF26E00020A24908704FF4C877A1495D
:10B63000088000240AE00020B34901EB84018870EF
:10B64000B14901EB8401C870601C84B20F2CF2DB9D
:10B65000002405E00020AB4921F81400601C84B2EE
:10B66000B4F57A7FF6DB0020A449C870A7A001F0EA
:10B6700078FBA848008801280FD100208C49087069
:10B68000002405E000209F4921F81400601C84B2CA
:10B69000B4F57A7FF6DB4FF00108B8F1000F04D162
:10B6A0009D48008800283FF40EAE0BB0BDE8F08343
:10B6B000F0B585B004460D461646984840EA042089
:10B6C0009749097840EA01078C208DF8000001971E
:10B6D00011208DF808008DF809508DF80A60FF21BF
:10B6E0008DF80B108DF80C10704801788DF80D1046
:10B6F00041788DF80E1081788DF80F106946012081
:10B70000F8F7C1FD0120F8F76CFF05B0F0BD30B5CA
:10B7100085B004462078814941EA002080490978B3
:10B7200040EA01058C208DF80000019513208DF86A
:10B73000080021798DF8091061798DF80A10617877
:10B740008DF80B10FF218DF80C10584801788DF8FA
:10B750000D1041788DF80E1081788DF80F10694624
:10B760000120F8F790FD0120F8F73BFF05B030BD50
:10B7700070B586B06B4E6C4833460122114600907E
:10B78000FA2000F019FF4FF47F06002033460F2205
:10B790000121009000F010FF4FF0FF146348046097
:10B7A00000208DF81300600BADF80C004FF6FF7011
:10B7B00000EAC400001DADF80E000020ADF8100036
:10B7C00001208DF8150002A803F0E3FF00251FE01B
:10B7D00005F10A00C0B28DF8120005EB850054494E
:10B7E00001EB80004068C0F34F30ADF8080005EB76
:10B7F000850001EB800040684FF6FF7101EAC00050
:10B80000001DADF80A0002A803F0C3FF681CC5B212
:10B810000E2DDDDB4FF468044648046018208DF8D7
:10B82000120000208DF8130001208DF8140040480C
:10B83000D0F81C01C0F34F30ADF808003C48D0F8F8
:10B840001C014FF6FF7101EAC000001DADF80A00AF
:10B85000600BADF80C00084600EAC400001DADF80E
:10B860000E000020ADF8100001208DF8150002A890
:10B8700003F08FFF06B070BD2DE9F04389B0074695
:10B8800000202D490870FF202C49087000202C4909
:10B8900008702C490870804600BF012F56D1002047
:10B8A00002498870FE204870CA204DE02E01002019
:10B8B0002D0100200A0000204572726F722120289D
:10B8C00043616E206E6F7420616464206D6F7265D9
:10B8D0002064617461206C69737420706172616DA1
:10B8E00065746572732C206D6178696D756D206962
:10B8F000732031332E290D00380000200A0B002060
:10B900003F6A002018450020036A00202A45210DC7
:10B910000000000032000020360000200000EC1C77
:10B920003A010020F9FFEA18F14E0C08EC00002063
:10B93000A0200020E40000203E0100203F01002064
:10B94000400100202C01002008702CE0FD494979BD
:10B9500048B201F0E8FA8146FA49097948B201F0A3
:10B96000E2FA09EB0010F8498870F649097A48B202
:10B9700001F0D9FA8146F349C97948B201F0D3FA06
:10B9800009EB0010F0494870EE49C97A48B201F05D
:10B99000CAFA8146EB49897A48B201F0C4FA09EB48
:10B9A0000010E9490870FFF7E3FE4FF00008E54892
:10B9B000007B61280BD0E348007B412807D0E14899
:10B9C000007B702803D0DF48007B502811D1DD496F
:10B9D000897B48B201F0A7FA8146DA49497B48B22F
:10B9E00001F0A1FA09EB0010D84908700120D849EC
:10B9F00008700026D4484078060406F46806D54846
:10BA0000066018208DF80A0000208DF80B00012038
:10BA10008DF80C00D048D0F81C01C0F34F30ADF8C1
:10BA20000000CD48D0F81C014FF6FF7101EAC000BC
:10BA3000001DADF80200700BADF80400084600EAE6
:10BA4000C600001DADF806000020ADF8080001207A
:10BA50008DF80D00684603F09CFE0020BF49087079
:10BA6000BF4805903C208DF81000B74800788DF84D
:10BA70001800B54841788DF8191081788DF81A10A2
:10BA800004A90120F8F7FFFB0120F8F7AAFD002028
:10BA9000B449088000BFF5F71EFEB248008840F6A2
:10BAA000C411884203DAAD4800780028F3D00020A2
:10BAB000AD49088000BF0020AA49088069E0F5F779
:10BAC0000AFE002460E0F5F706FEA84800EBC4007B
:10BAD000C079002853D1A64800EB84008078C0EBE1
:10BAE000001000EBC000A34901EB8000007A9F49E1
:10BAF00001EBC4014978884212DB9C4901EBC40088
:10BB0000FFF705FE0020974908809B480078401EFB
:10BB1000994908700120954901EBC401C8712EE0D4
:10BB2000924800EBC40080799449085C8F4901EB8E
:10BB3000C401C978884222DB8C4B03EBC4039B7998
:10BB4000DFF838C21CF803305B1CDAB2874B03EB1A
:10BB5000C4039978854B13F83400FFF7A9FD002042
:10BB600080490880814800EBC400C0787F4901EB20
:10BB7000C401897808447D4901EBC401C870601C88
:10BB800084B20D2C00DB0024784810F83400FF2824
:10BB900099D179480078002805DD7248008841F67F
:10BBA000583188428BDB00206E49088033E0F5F77E
:10BBB00092FD00242AE0F5F78EFD6D4800EB84002D
:10BBC000C078F0B96A4800EB84008078C0EB0010C0
:10BBD00000EBC000674901EB8000007A644901EB8B
:10BBE0008401497888420CDB00205E490880644863
:10BBF0000078401E6249087001205D4901EB840114
:10BC0000C870601C84B20D2C00DB0024584810F86A
:10BC10002400FF28CFD15A480078002805DD51487C
:10BC2000008841F658318842C1DB4F4800886428BB
:10BC300004DA5448007800283FF43DAF0024002582
:10BC40001AE1F5F748FD494800EBC400C079012826
:10BC500077D1464810F834004B4921F81500681C8C
:10BC600085B2F2E0F5F737FD404800EBC40080797B
:10BC7000C0EB001000EBC0003E4901EB80003B49E7
:10BC800001EBC4018979414A515C01EBC101425C7D
:10BC90002846691C8DB23C4921F81020334800EB3E
:10BCA000C4008079C0EB001000EBC000314901EB0B
:10BCB00080002E4901EBC4018979344A515C01EBC3
:10BCC000C101084442782846691C8DB22E4921F8EA
:10BCD0001020264800EBC4008079C0EB001000EB78
:10BCE000C000244901EB8000204901EBC40189799F
:10BCF000264A515C01EBC101084482782846691C40
:10BD00008DB2214921F81020184800EBC400807939
:10BD1000C0EB001000EBC000164901EB8000134996
:10BD200001EBC4018979194A515C01EBC101084456
:10BD3000C2782846691C8DB2134921F810200B489F
:10BD400026E097E00A0B00202E0100203F01002092
:10BD50003E010020E4000020A0200020310100204E
:10BD6000F9FFEA18000000200A0000201C4D002006
:10BD7000E84C0020E74D00203501002053690020E9
:10BD80003401002040010020184500206069002097
:10BD900000EBC4008079C0EB001000EBC000FE494E
:10BDA00001EB8000FD4901EBC4018979FC4A515C3B
:10BDB00001EBC101084402792846691C8DB2F9499A
:10BDC00021F81020F54800EBC4008079C0EB00108A
:10BDD00000EBC000F04901EB8000F04901EBC40129
:10BDE0008979EF4A515C01EBC10108444279284648
:10BDF000691C8DB2EB4921F81020E84800EBC40023
:10BE00008079C0EB001000EBC000E34901EB80003B
:10BE1000E24901EBC4018979E14A515C01EBC101BE
:10BE2000084482792846691C8DB2DE4921F8102029
:10BE3000DA4800EBC4008079D949085C401CD74936
:10BE400001EBC4018979D64A5054D44800EBC400B0
:10BE50008079D349085CD14901EBC4014978884213
:10BE6000FFF600AF4FF0FF322846691C8DB2CD4976
:10BE700021F81020601C84B2C84810F83400FF2854
:10BE800002D00D2CFFF6DDAE0024F4E0F5F723FC24
:10BE9000C54800EB8400C07801287CD1C24810F866
:10BEA0002400C04921F81500681C85B2CCE0F5F7E4
:10BEB00012FCBD4800EB84008078C0EB001000EB62
:10BEC000C000B54901EB8000B74901EB84018978D6
:10BED000B34A515C01EBC101425C2846691C8DB23A
:10BEE000B04921F81020B04800EB84008078C0EB06
:10BEF000001000EBC000A84901EB8000AA4901EB4B
:10BF000084018978A64A515C01EBC101084442785A
:10BF10002846691C8DB2A34921F81020A24800EBE5
:10BF200084008078C0EB001000EBC0009A4901EB60
:10BF300080009D4901EB84018978994A515C01EBAD
:10BF4000C101084482782846691C8DB2954921F8C0
:10BF50001020954800EB84008078C0EB001000EBC7
:10BF6000C0008D4901EB80008F4901EB8401897885
:10BF70008B4A515C01EBC1010844C2782846691C18
:10BF80008DB2884921F81020874800EB8400807822
:10BF9000C0EB001000E06CE000EBC0007E4901EB5C
:10BFA0008000814901EB840189787D4A515C01EB75
:10BFB000C101084402792846691C8DB2794921F8EB
:10BFC0001020794800EB84008078C0EB001000EB73
:10BFD000C000714901EB8000734901EB840189784D
:10BFE0006F4A515C01EBC101084442792846691C43
:10BFF0008DB26C4921F810206B4800EB84008078EA
:10C00000C0EB001000EBC000634901EB8000664903
:10C0100001EB84018978624A515C01EBC10108445B
:10C0200082792846691C8DB25E4921F810205E484D
:10C0300000EB840080785A49085C401C5A4901EBA7
:10C0400084018978564A5054574800EB8400807820
:10C050005349085C544901EB840149788842FFF652
:10C0600026AF4FF0FF322846691C8DB24D4921F8AA
:10C070001020601C84B24C4810F82400FF2802D025
:10C080000D2CFFF603AF00246BE004EBC40047491E
:10C090000A5C2846691C8DB2424921F8102004EB45
:10C0A000C4004249084442782846691C8DB23D4983
:10C0B00021F8102004EBC4003C490844827828464B
:10C0C000691C8DB2374921F8102004EBC4003749B0
:10C0D0000844C2782846691C8DB2324921F81020E4
:10C0E00004EBC4003149084402792846691C8DB22A
:10C0F0002C4921F8102004EBC4002C490844427953
:10C100002846691C8DB2274921F8102004EBC40091
:10C110002649084482792846691C8DB2214921F8B4
:10C12000102004EBC40021490844C2792846691C48
:10C130008DB21C4921F8102004EBC4001B490844AF
:10C14000027A2846691C8DB2164921F810204FF05A
:10C15000FF322846691C8DB2124921F81020601C5C
:10C1600084B213480078844201DA0B2C8DDB002D59
:10C1700002DD681E85B20AE04FF001080D48007824
:10C18000401C0C4908704FF4C87000F08CFB6FF035
:10C1900001022846691C0FE0E74D00201C4D0020DD
:10C1A0006069002018450020E84C0020844D0020E4
:10C1B000360100202C0100208DB2D54921F8102035
:10C1C000D4480078012804D1D3480078401CD249D3
:10C1D0000870D0480078012804D1CF48007805289D
:10C1E000FFF65BABB8F1010F03D1CB480078022812
:10C1F000F6DB012404E00020C8490855601C84B225
:10C2000040F226208442F6DD3FB968222946C04824
:10C2100000F050FD0D20F4F7CDF90020C049088052
:10C22000C048007809B0BDE8F08330B585B04FF064
:10C23000FF350195022405E069462046F8F723F80A
:10C24000601CC4B20E2CF7DD05B030BD70B5FFF731
:10C25000ECFF0020B449087048708870B14908703C
:10C26000AC490870B1490870B1490870B14908700B
:10C27000B1490870B1490870F5F72DFA002404E0BF
:10C28000FF20AF490855601C84B20D2CF8DB002458
:10C2900004E00020AB490855601C84B20D2CF8DB8B
:10C2A000002404E00020A8490855601C84B20D2C2D
:10C2B000F8DB002409E0FF20A44901F82400002055
:10C2C00001EB8401C870601C84B20D2CF3DB0024E8
:10C2D00009E0FF209E4901F83400002001EBC40171
:10C2E000C871601C84B20D2CF3DB00241CE000201C
:10C2F000C4EB041101EBC101964A02EB8101087203
:10C3000000250DE00020C4EB041101EBC101914AAE
:10C3100002EB810105EBC5021144C871681C85B2AE
:10C320003C2DEFDB601C84B20D2CE0DBF5F7D3F97C
:10C33000002405E0FF20764921F81400601C84B237
:10C34000B4F57A7FF6DB70BD704710B500208249E6
:10C350000880824908808249088082490880824991
:10C3600008806F49088081490880FFF76FFFF5F763
:10C37000B2F90E2206210120F4F7F1FE052000F0AB
:10C3800092FAF9207A490870FFF7DEFF0120FFF7E3
:10C3900073FA0446FFF75AFF012C41D175A000F053
:10C3A000E0FC0021774802F0A0F9012076490870EE
:10C3B00007207649087000BFF5F78DF958480088C6
:10C3C000012804D1FFF742FF0020FFF755FA654826
:10C3D0000088012801D1FEF7E3FE634800880128A8
:10C3E00001D1FEF73BFE6A480088062810D10020E4
:10C3F0006749088049488078302802D165A000F05C
:10C40000B0FC46488078322802D15AA000F0A9FC3E
:10C410005348008838B9504800880028CCD002E042
:10C4200001204D49088001205B49087000205649D1
:10C4300008705A49087000F01BFB10BD30B585B07C
:10C440000024574890F81C015649087000205649AE
:10C4500008700AE03A48005D52490978884202D1E2
:10C46000012051490870601CC4B23548005DFF28A6
:10C4700005D00D2C03DA4C4800780028EAD04B4850
:10C48000007820B94848007808B90D2C0EDB4748E1
:10C490000078012829D14348007845490978884225
:10C4A00023D14148007800BB0D2C1EDA3D480078AE
:10C4B000234908553B48007840F46B0584208DF8EB
:10C4C0000000019519480078194909780844801C32
:10C4D0000F280DDA15490978154A12781144891C7C
:10C4E000C8B26946F7F7CFFE02E0FF202D49087079
:10C4F0002C4800782E490978884205D12B480078CD
:10C50000012801D12B4908702648007805B030BDBC
:10C5100018450020370100202C0100200A0B0020C4
:10C5200032000020310100202E01002032010020C5
:10C5300033010020340100203501002036010020A5
:10C54000DF6A00205369002060690020E84C002069
:10C550001C4D0020E74D00200C000020340000207E
:10C56000360000202E000020380000202C00002083
:10C570003A0100202A534145204A313933392D32BE
:10C58000310D000000140040570000205100002031
:10C590001C0000202A310D0055000020560000200C
:10C5A000A02000203D0100203C0100203E01002091
:10C5B0003F010020400100202DE9F04186B00446F3
:10C5C0000D4616461F46DDF8308008212F4801F041
:10C5D00004F9012D03D184208DF8040002E08020AD
:10C5E0008DF804000297212C05D1414644F25D40AC
:10C5F000F7F788FA17E07D2C05D1414643F2474012
:10C60000F7F780FA0FE0FA2C05D1414643F60160B6
:10C61000F7F778FA07E0B4F5FA7F04D141464FF412
:10C620007850F7F76FFA01A93046F7F72CFE06B0FD
:10C63000BDE8F08130B585B004460D466946284610
:10C64000F7F7E5FE20788DF8080061788DF809107D
:10C65000A1788DF80A10E1788DF80B1021798DF80A
:10C660000C1061798DF80D10A1798DF80E10E1791B
:10C670008DF80F1000208DF8100069462846F7F756
:10C6800002FE2846F7F7ADFF05B030BD00180240A6
:10C690002DE9F341044638E02078252830D1641C88
:10C6A0002078632814D064280BD0732802D078280F
:10C6B00020D116E0019820C80190284600F051FBD7
:10C6C0001DE0019840C80190304600F05CFB16E088
:10C6D000019810F8041BCFB2019078B2F3F76AFF0B
:10C6E0000DE0019810F8041BCFB20190384600F01D
:10C6F000C2FA04E0217848B2F3F75CFF00BF03E020
:10C70000217848B2F3F756FF641C20780028C3D183
:10C71000BDE8FC810FB438B53748007810B938BC93
:10C720005DF814FB354804783348007833490870C5
:10C7300005A8009000990498FFF7AAFF0020009038
:10C740002E48047000BF00BFE9E710B504462A4830
:10C7500004702BA0FFF7DEFF10BD0FB4F8B505463F
:10C760000C4625480078E0B1244806782248007835
:10C770002249087009A80090284600F0F2FA24A087
:10C7800000F0EFFAA0B200F029FA22A000F0E9FAD6
:10C7900000990898FFF77CFF00200090174806706A
:10C7A00000BF00BFFEE70FB4F8B505460C461248BF
:10C7B000007810B9F8BC5DF814FB104806780E48F4
:10C7C00000780E49087009A80090284600F0C9FAC0
:10C7D0000FA000F0C6FAA0B200F000FA0DA000F021
:10C7E000C0FA00990898FFF753FF00200090034813
:10C7F000067000BF00BFDDE74101002059000020A6
:10C80000547261636520456E61626C65640D000061
:10C810002028000029203A0010B50020184908708F
:10C8200018484078352828D11648807830380A28AA
:10C8300021D2DFE800F0050C0D131A1B1C1D1E1F72
:10C8400001200F49087010A000F08BFA13E012E0ED
:10C8500000200B490870FEF7BEF80CE000200849E4
:10C8600008700120FEF7B7F805E004E003E002E0FD
:10C8700001E000E000BF00BF10BD00BFFCE700000A
:10C88000540000200A0B00202A310D0070B5044628
:10C890001148058800BFF4F71EFF0F480088401BB1
:10C8A000A042F8D370BD70B504460C48058800BF9F
:10C8B000F4F711FF09480088401BA042F8D370BD6F
:10C8C00010B5044600BFF4F706FF2000A4F10101F3
:10C8D0008CB2F8D110BD00000A000020000000203A
:10C8E00010B504464FF40041654800F074FF012084
:10C8F000FFF7D9FF0121634800F06DFF4FF40041BD
:10C900005F4800F06AFF152C78D2DFE804F08C0B4A
:10C9100011178C8C1D23292F353B41474D535963EB
:10C920006D788200002201210420F4F718FC80E0D9
:10C93000002202210420F4F712FC7AE000220321F5
:10C940000420F4F70CFC74E0002206210420F4F724
:10C9500006FC6EE0002207210420F4F700FC68E0EA
:10C96000002208210420F4F7FAFB62E000220921EA
:10C970000420F4F7F4FB5CE000220A210420F4F721
:10C98000EEFB56E000220B210420F4F7E8FB50E018
:10C9900000220C210420F4F7E2FB4AE000220D21E2
:10C9A0000420F4F7DCFB44E000220E210420F4F71D
:10C9B000D6FB3EE000220F210420F4F7D0FB38E044
:10C9C0000F220D210420F4F7CAFB01212D4800F0AD
:10C9D00004FF2EE00F220C210420F4F7C0FB0121FC
:10C9E000284800F0FAFE24E00F220B210420F4F77F
:10C9F000B6FB0121234800F0F0FE1AE013E00F22FD
:10CA000007210420F4F7ABFB01211E4800F0E5FEEE
:10CA10000FE0022203210420F4F7A1FB01211948B1
:10CA200000F0DBFE05E0002207210420F4F797FB6D
:10CA300000BF00BF6420FFF736FF10BD70B505468C
:10CA40000C4601210F4800F0C8FE4FF400410C488D
:10CA500000F0C3FE1CB901210A4800F0BCFE2246CA
:10CA600029460420F4F77BFB6420FFF71CFF70BD10
:10CA700010B5002211461046F4F771FB10BD0000FE
:10CA8000001402400018024010B54C4804880020F1
:10CA90004B49088000BFF4F71EFE49480088012872
:10CAA00005DA04F15000454909888842F3DA04F1B7
:10CAB000500042490988884202DC0120414908802F
:10CAC00010BD2DE9F04780460C46042500BF002725
:10CAD00000BFF4F700FE3C4A691C515C48B200F00C
:10CAE00022FA82463849495D48B200F01CFA0AEB46
:10CAF0000016642104FB01F0FAF7AFFAB0B2334933
:10CB000008803349088033490880FFF7BDFF374468
:10CB10002D49A81C11F80090ED1CB9F1000FD8D1D7
:10CB2000B8F1000F03D0B8F1010F10D100E01DE003
:10CB3000642104FB01F0FAF790FAF8B22349088067
:10CB40002349088023490880FFF79EFF0EE06421F7
:10CB500004FB01F0FAF781FAB8B21C4908801C49BD
:10CB600008801C490880FFF78FFF00BF00BFBDE8A9
:10CB7000F08770B505460E46002400BFF4F7ABFD04
:10CB8000642105FB01F0FAF768FA134830F8140045
:10CB90000E4908800E4908800E490880012E01D1F7
:10CBA000FFF772FF641C0C4830F814004FF6FF7159
:10CBB000884201D0282CE1DB70BD00000A00002073
:10CBC000220000200C0000200A0B0020044400403A
:10CBD00004140140044C0040F00900202DE9F0410C
:10CBE00086B0064642F2107096FBF0F0019040F2DB
:10CBF000712101984843A6EB00144FF47A70B4FBFE
:10CC0000F0F00290029800EB4001C1EBC010A4EBE1
:10CC1000C0046420B4FBF0F00390039800EBC00163
:10CC200001EB0010A4EB80040A20B4FBF0F00490A8
:10CC3000049800EB8000A4EB400005904FF0000842
:10CC4000012513E05DF8250018B9059818B9052DE0
:10CC500001D14FF00108B8F1010F06D11DF82500F0
:10CC60003030C7B278B2F3F7A5FC6D1C062DE9DBB6
:10CC700006B0BDE8F08170B504462046E11704EB2C
:10CC800011710E11092E01D8303600E0373670B21E
:10CC9000F3F790FC2046E11704EB11710911A4EBA6
:10CCA0000115092D01D8303500E0373568B2F3F7AA
:10CCB00081FC70BD2DE9F04105460F4616462A203D
:10CCC000F3F778FC002448E0482E01D0682E1CD1F0
:10CCD00035F91400401C18B135F91400C01C18B9FE
:10CCE0002620F3F767FC2CE035F91400801C18B9F6
:10CCF0002320F3F75FFC24E035F91400001D00B396
:10CD000015F81400FFF7B7FF1BE035F91400401CBD
:10CD100018B135F91400C01C18B92620F3F74AFCE5
:10CD20000FE035F91400801C18B92320F3F742FCFA
:10CD300007E035F91400001D18B115F81400FFF7CD
:10CD40004DFFB81EA04206DD35F91400C01C10B11D
:10CD50002020F3F72FFC601C84B2BC42B4DBBDE89A
:10CD6000F08110B5044604E014F8012B50B2F3F73B
:10CD700021FC20780028F7D110BD10B504462046CC
:10CD8000F3F718FC10BD2DE9F0418CB0064672484F
:10CD9000B6FBF0F00290714902984843A6EB40249C
:10CDA0006F48B4FBF0F003906E4903984843A4EB3E
:10CDB00000246D48B4FBF0F004906C49049848439B
:10CDC000A4EBC0146A48B4FBF0F0059043F6095197
:10CDD00005984843A4EB80146648B4FBF0F0069035
:10CDE00040F6354106984843A4EB401442F21070D7
:10CDF000B4FBF0F0079040F2712107984843A4EB90
:10CE000000144FF47A70B4FBF0F00890089800EB2F
:10CE10004001C1EBC010A4EBC0046420B4FBF0F0EF
:10CE20000990099800EBC00101EB0010A4EB80040D
:10CE30000A20B4FBF0F00A900A9800EB8000A4EB03
:10CE400040000B904FF00008012515E001A850F8B4
:10CE5000250018B90B9818B90A2D01D14FF0010817
:10CE6000B8F1010F07D101A810F825003030C7B282
:10CE700078B2F3F79FFB6D1C0B2DE7DB0CB0BDE820
:10CE8000F08170B505462C0F092C01D8303400E034
:10CE9000373460B2F3F78EFBC5F30364092C01D875
:10CEA000303400E0373460B2F3F784FBC5F3035449
:10CEB000092C01D8303400E0373460B2F3F77AFB44
:10CEC000C5F30344092C01D8303400E0373460B294
:10CED000F3F770FBC5F30334092C01D8303400E0BC
:10CEE000373460B2F3F766FBC5F30324092C01D88D
:10CEF000303400E0373460B2F3F75CFBC5F3031461
:10CF0000092C01D8303400E0373460B2F3F752FB1B
:10CF100005F00F04092C01D8303400E0373460B23A
:10CF2000F3F748FB70BD0146302904DB392902DCE8
:10CF3000A1F130007047612904DB662902DCA1F110
:10CF40005700F7E7412904DB462902DCA1F137004D
:10CF5000F0E73020EEE7000000CA9A3B65CD1D00E7
:10CF600000E1F505E1F50500809698002D310100FE
:10CF700040420F00A0860100094880470948004749
:10CF8000FEE7FEE7FEE7FEE7FEE7FEE7FEE7FEE779
:10CF9000FEE7FEE704480549054A064B70470000D6
:10CFA00019ED0C0885010C08506B00205071002011
:10CFB000506D0020506D0020FA48006840F00100DC
:10CFC000F84908600020F74908310860F548006812
:10CFD000F5490840F3490860F448091D0860081F36
:10CFE000006820F48020091F08600020ED490C3102
:10CFF000086070470021EB4A921C117011460870BE
:10D00000704710B501460022002300204A11012A72
:10D0100002D1E44C236808E0022A03D1E14C7034C9
:10D02000236802E0DF4C7434236801F01F020124FE
:10D0300094401C400CB1012000E0002010BD38B528
:10D04000002000900024002500BF3120FFF7D9FF09
:10D0500005460098401C00901DB90098B0F5A06FDF
:10D06000F3D13120FFF7CDFF08B1012400E0002407
:10D07000204638BD01460020CA4A106820F0F8005A
:10D0800040EAC10010607047C94908607047C8494C
:10D0900008667047F0B5DDE9054541EA82160127CB
:10D0A000C7EB530746EA0746064346EA046646EAE4
:10D0B0000576BC4F3F1D3E60F0BDBD498866704798
:10D0C000820142EA0172B74B84331A60704701460D
:10D0D0000020B44A0832106820F0030008431060B2
:10D0E0007047B0480830006800F00C0070470146F7
:10D0F0000020AC4A0832106820F0F00008431060AD
:10D10000704701460020A74A0832106820F4E0501A
:10D1100008431060704701460020A24A0832106898
:10D1200020F4604040EAC1001060704739B19D4A68
:10D130000D32127802439B4B0D331A7006E0994A68
:10D140000D3212788243974B0D331A7070470021CD
:10D15000944A703211701170012802D004280AD14B
:10D1600004E001218F4A7032117005E005218D4ADB
:10D170007032117000E000BF00BF70478D49086039
:10D180007047002100F44072B2F5407F0AD1854A11
:10D190000832116821F4F811874A02401143814A8C
:10D1A000083211607F4A70321268C0F30B031A43D1
:10D1B0007C4B70331A6070477E4944390860704771
:10D1C0007E4908607047F0B5002100220024022546
:10D1D00000260223734F08373F6807F00C0121B186
:10D1E000042905D0082937D105E0754F076036E0DE
:10D1F000744F076033E06B4F3F1D3F68C7F38056A5
:10D20000684F3F1D3F6807F03F036EB16D4FB7FB9E
:10D21000F3F7DFF890C10CF1040CDCF800C0CCF39C
:10D22000881C07FB0CF40CE0654FB7FBF3F7DFF845
:10D2300074C10CF1040CDCF800C0CCF3881C07FBB3
:10D240000CF4584F3F1D3F68C7F301477F1C7D001A
:10D25000B4FBF5F7076002E0594F076000BF00BF5D
:10D26000504F08373F6807F0F0010909564F7A5CC4
:10D270000768D74047604B4F08373F6807F4E051D5
:10D28000890A514F7A5C4768D7408760454F083715
:10D290003F6807F46041490B4B4F7A5C4768D740C1
:10D2A000C760F0BD39B13F4A3032126802433D4B8E
:10D2B00030331A6006E03B4A303212688243394B01
:10D2C00030331A60704739B1364A3432126802433B
:10D2D000344B34331A6006E0324A343212688243E7
:10D2E000304B34331A60704739B12E4A38321268E5
:10D2F00002432C4B38331A6006E02A4A383212684F
:10D300008243284B38331A60704739B1254A40327E
:10D3100012680243234B40331A6006E0214A403230
:10D32000126882431F4B40331A60704739B11D4A5F
:10D330004432126802431B4B44331A6006E0194A18
:10D34000443212688243174B44331A60704739B134
:10D35000144A103212680243124B10331A6006E06E
:10D36000104A1032126882430E4B10331A60704715
:10D3700039B10C4A1432126802430A4B14331A6052
:10D3800006E0084A143212688243064B14331A60CE
:10D390007047D9B1034A183212680243014B18335F
:10D3A0001A6018E000380240FFFFF6FE103000243B
:10D3B00000004742800E4742FFFCFF0F5C014742DE
:10D3C0000024F40040787D0150030D085B4A126888
:10D3D00082435A4B1A60704739B1584A0832126872
:10D3E0000243564B08331A6006E0544A083212686A
:10D3F0008243524B08331A60704739B14F4A0C329E
:10D40000126802434D4B0C331A6006E04B4A0C3253
:10D4100012688243494B0C331A60704739B1474A4E
:10D42000383212680243454B38331A6006E0434AEB
:10D43000383212688243414B38331A60704739B131
:10D440003E4A3C32126802433C4B3C331A6006E0D1
:10D450003A4A3C3212688243384B3C331A60704778
:10D4600039B1364A403212680243344B40331A60B5
:10D4700006E0324A403212688243304B40331A6031
:10D48000704739B12D4A4832126802432B4B48335A
:10D490001A6006E0294A483212688243274B483313
:10D4A0001A60704739B1254A4C3212680243234B47
:10D4B0004C331A6006E0214A4C32126882431F4BFB
:10D4C0004C331A6070471E49086070471D49C86494
:10D4D000704702460020194B103B186820F0EC60A2
:10D4E00042EA01031843154B103B1860704702468F
:10D4F0000020124B103B186820F0784042EA0103EC
:10D5000018430E4B103B186070470C485C300068A5
:10D5100040F0807009495C31086070470146002086
:10D52000064A0C3A12680A400AB1012000E00020C5
:10D53000704702490A3908707047000018380240E5
:10D54000400E47420000474231490143314A1160D1
:10D55000704770B5002100230F22C47804B32D4C0E
:10D56000246804F4E064C4F5E064210AC1F1040312
:10D57000CA40447804FA03F1847814402143090135
:10D58000254C0678A155047804F01F050124AC4011
:10D5900005786D11AD0005F1E025C5F8004109E001
:10D5A000047804F01F050124AC401C4D0678761168
:10D5B00045F8264070BD1A4A0A400243154B1B1F0E
:10D5C0001A60704739B1134A121D12680243114B99
:10D5D0001B1D1A6006E00F4A121D126882430D4B94
:10D5E0001B1D1A607047042808D14FF0E02109691B
:10D5F00041F004014FF0E022116107E04FF0E0211B
:10D60000096921F004014FF0E02211617047000028
:10D610000000FA050CED00E000E400E080E100E02D
:10D6200080FFFF1F10B504468848844208D10121BD
:10D630000846FFF78CFE00210120FFF788FE5EE020
:10D640008348844208D101210220FFF780FE002197
:10D650000220FFF77CFE52E07E48844208D101217F
:10D660000420FFF774FE00210420FFF770FE46E05F
:10D670007948844208D101210820FFF768FE002183
:10D680000820FFF764FE3AE07448844208D1012183
:10D690001020FFF75CFE00211020FFF758FE2EE05F
:10D6A0006F48844208D101212020FFF750FE00215D
:10D6B0002020FFF74CFE22E06A48844208D1012175
:10D6C0004020FFF744FE00214020FFF740FE16E017
:10D6D0006548844208D101218020FFF738FE0021EF
:10D6E0008020FFF734FE0AE06048844207D1012120
:10D6F0008015FFF72CFE0021A015FFF728FE10BDB6
:10D70000F0B50A4600210023002400BF3DE00125BA
:10D7100005FA01F3156805EA03049C4234D1056853
:10D720004F000326BE40B543056015794E00B54055
:10D730000668354305601579012D02D01579022D53
:10D7400016D185684F000326BE40B54385605579E4
:10D750004E00B540866835438560456801268E4099
:10D76000B5434560456896798E40B6B2354345600D
:10D77000C5684F000326BE40B543C560D5794E004D
:10D78000B540C6683543C560491C1029BFD3F0BDFC
:10D790004FF6FF7101600021017141718171C1710A
:10D7A00070470246002013690B400BB1012000E0D6
:10D7B000002070470146086980B270470246002089
:10D7C00053690B400BB1012000E000207047014677
:10D7D000486980B2704701837047418370470AB13E
:10D7E000018300E0418370474161704742694A40CC
:10D7F000426170474FF480320A43C261C161C26125
:10D80000C269C2697047F0B5002300244D07ED0ED0
:10D8100002FA05F3CE1000F1200555F826504E0708
:10D82000F70E0F26BE40B543CF1000F1200646F894
:10D830002750CE1000F1200555F8265045EA030484
:10D84000CE1000F1200545F82640F0BD0000024052
:10D850000004024000080240000C02400010024098
:10D860000014024000180240001C02400020024048
:10D8700010B50446F748844208D101211020FFF773
:10D88000BCFD00211020FFF7B8FD3EE0F2488442C5
:10D8900009D101214804FFF79FFD00214FF400301A
:10D8A000FFF79AFD31E0ED48844209D10121880457
:10D8B000FFF792FD00214FF48020FFF78DFD24E05B
:10D8C000E748844209D10121C804FFF785FD002102
:10D8D0004FF40020FFF780FD17E0E248844209D1B1
:10D8E00001210805FFF778FD00214FF48010FFF7B4
:10D8F00073FD0AE0DC48844207D101212020FFF7B4
:10D900007CFD00212020FFF778FD10BD2DE9FF47A9
:10D9100005460E460024A14600BFA046B08900B1CE
:10D9200000BF2C8A24F44054F08804432C82AC8934
:10D9300041F20C608443B0883189084371890843FF
:10D940000443AC81AC8A24F44074B0890443AC82B3
:10D950006846FFF738FCBF48854202D0C24885427E
:10D9600002D1DDF80C9001E0DDF80890A88900F400
:10D97000004040B109EBC90000EB091031684900D3
:10D98000B0FBF1F707E009EBC90000EB09103168C3
:10D990008900B0FBF1F76420B7FBF0F00401200927
:10D9A000642101FB1078A88900F4004040B13220C6
:10D9B00000EBC800B0FBF1F000F00700044308E002
:10D9C000322000EB08106421B0FBF1F000F00F00F2
:10D9D00004432C81BDE8FF874FF4165101600021FC
:10D9E0008180C18001810C214181002181817047AA
:10D9F00010B502460020108A20F470600B884C8815
:10DA000023438C882343CC8823431843108210BDC2
:10DA10000021018041808180C180704721B18289CD
:10DA200042F40052828104E082894DF6FF731A406D
:10DA300082817047F0B503460024002600250020AF
:10DA400040F66A17B94200D100BF1846C1F342142C
:10DA500001F01F06012707FA06F5012C01D10C3051
:10DA600004E0022C01D1103000E014301AB1076834
:10DA70002F43076002E00768AF430760F0BD1AB1AB
:10DA8000838A0B43838202E0838A8B4383827047BD
:10DA9000028A4FF6F0731A400282028A0A43028217
:10DAA000704782894FF2FF731A40828182890A434C
:10DAB0008281704721B1828942F00202828104E0B2
:10DAC00082894FF6FD731A4082817047028A4FF6B1
:10DAD000DF731A400282028A0A430282704721B130
:10DAE000028A42F48042028204E0028A4BF6FF730B
:10DAF0001A4002827047C1F30802828070470146D3
:10DB00008888C0F308007047818941F00101818154
:10DB10007047028BD2B20283028B42EA0122028357
:10DB20007047028B02F47F420283028B0A43028316
:10DB3000704721B1828A42F02002828204E0828A08
:10DB40004FF6DF731A408282704721B1828A42F019
:10DB50001002828204E0828A4FF6EF731A408282BA
:10DB6000704721B1828A42F00802828204E0828AF0
:10DB70004FF6F7731A408282704721B1828942F4CE
:10DB80000042828103E08289C2F30E0282817047E3
:10DB900021B1828A42F40062828204E0828A4FF2DA
:10DBA000FF731A4082827047828A4FF6FB731A40D5
:10DBB0008282828A0A438282704721B1828A42F03D
:10DBC0000202828204E0828A4FF6FD731A4082824A
:10DBD000704702460020B1F5007F00D100BF1388D6
:10DBE0000B400BB1012000E00020704701F40072EF
:10DBF000B2F5007F00D100BFCA430280704770B504
:10DC00000246002400230025002040F66A16B14297
:10DC100000D100BFC1F3421501F01F03012606FA2F
:10DC200003F3012D02D19689334006E0022D02D183
:10DC3000168A334001E0968A33400C12012606FA18
:10DC400004F41688344013B10CB1012000E0002028
:10DC500070BD00000010014000440040004800403A
:10DC6000004C0040005000400014014010B500225C
:10DC7000002340F66A14A14200D100BF0A12012419
:10DC80009440A3B2DC43048010BD000010B50446EC
:10DC9000F348844208D101218014FFF7AEFB002134
:10DCA000A014FFF7AAFB16E0EE48844208D1012138
:10DCB0000014FFF791FB00212014FFF78DFB0AE011
:10DCC000E948844207D10121C013FFF785FB0021F9
:10DCD000E013FFF781FB10BD10B50022028802F4AB
:10DCE00041520B884C8823438C882343CC882343A0
:10DCF0000C8923434C8923438C892343CC892343B8
:10DD00001A430280838B4FF2FF74234083830B8A74
:10DD1000038210BD2DE9F04F0026022300240127C5
:10DD200000220025944690469146B0F81CA04FF280
:10DD3000400B0AEA0B0AA0F81CA04FF0020AA0F858
:10DD400020A0868BD1F808A0BAF1020F01D100BF44
:10DD50008CE0B1F804A0BAF1000F01D1012700E076
:10DD60000227DFF808A3DAF800A00AF0005ABAF197
:10DD7000005F33D1DFF8F8A2DAF800A00AF4000A55
:10DD8000BAF1000F09D0DFF8E8A2DAF800A02AF40F
:10DD9000000ADFF8DCB2CBF800A0DFF8D4A20AF169
:10DDA0007C0ADAF800A0CAF38818DFF8C4A20AF1E6
:10DDB0007C0ADAF800A0CAF30279DFF8B4A2AAF16B
:10DDC000040ADAF800A00AF03F0CDFF8A8A2BAFBB8
:10DDD000FCFA0AFB08FABAFBF9F515E0DFF890A2A5
:10DDE000AAF1040ADAF800A0CAF38812DFF880A2C8
:10DDF000AAF1040ADAF800A0CAF3027AB2FBFAFA2E
:10DE0000DFF874B20AFB0BF5B1F806A0BAF5007F93
:10DE10000ED14FEA152A0AEB8A0A4FEA4A0AD1F8CC
:10DE200008B0BAFBFBFA0AF1050A1FFA8AF20FE002
:10DE30004FEA471AB5FBFAFA0AEB8A0A4FEA4A0A8E
:10DE4000D1F808B0BAFBFBFA0AF1050A1FFA8AF208
:10DE50004FF00A0AB2FBFAF202F00104A2EB040A44
:10DE6000CAF34F034FF6FF7A0AEA0424022B01DBC0
:10DE7000FF2B01DD02230024B1F806A04AEA040AC0
:10DE80004AEA030AA0F820A0B1F804A0B1F80CB047
:10DE90004AEA0B0AB1F802B04AEA0B0AB1F800B03C
:10DEA0004AEA0B0A4AF4006A4AEA06068683BDE893
:10DEB000F08F0021018041808180C18001814181FA
:10DEC0008181C18107210182704700210180418049
:10DED0008180C1800221816000218181704721B150
:10DEE000028842F04002028004E002884FF6BF73CD
:10DEF0001A400280704721B1828B42F48062828393
:10DF000004E0828B4FF6FF331A408283704730B5AE
:10DF1000002400230C110125A540ABB21AB185885D
:10DF20001D43858002E085889D43858030BD21B1F9
:10DF3000828842F01002828004E082884FF6EF73FC
:10DF40001A40828070471AB183880B43838002E0B5
:10DF500083888B438380704781817047014688891D
:10DF600070474FF6FF62914204D0028842F48072FB
:10DF7000028004E002884FF6FF631A400280704777
:10DF800021B1828842F00402828004E082884FF648
:10DF9000FB731A408280704702884FF2FF731A4069
:10DFA000028002880A4302807047018841F4805150
:10DFB0000180704721B1028842F40052028004E0DF
:10DFC00002884DF6FF731A40028070470246002017
:10DFD000012901D0108B00E0908A70470146088A21
:10DFE0007047B1F5804F04D1028842F4804202802C
:10DFF00004E002884BF6FF731A4002807047024625
:10E00000002013890B400BB1012000E00020704775
:10E01000CA4302817047F0B5024600200024002365
:10E02000002501F00F070126BE40B4B20B110126F6
:10E030009E40B3B2968806EA03051689264016B1BB
:10E040000DB1012000E00020F0BD10B5002201F06C
:10E050000F040123A3409AB2D343038110BD0000F3
:10E060000030014000380040003C0040002004E047
:10E070000838024040787D0140420F0010B5044648
:10E08000FC48844208D101210846FFF7B6F9002177
:10E090000120FFF7B2F99DE0B4F1804F08D10121D2
:10E0A0000846FFF799F900210120FFF795F991E063
:10E0B000F148844208D101210220FFF78DF90021A7
:10E0C0000220FFF789F985E0EC48844208D101215C
:10E0D0000420FFF781F900210420FFF77DF979E0A2
:10E0E000E748844208D101210820FFF775F9002193
:10E0F0000820FFF771F96DE0E248844208D1012160
:10E100001020FFF769F900211020FFF765F961E0A1
:10E11000DD48844208D101212020FFF75DF900216C
:10E120002020FFF759F955E0D848844208D1012151
:10E130000220FFF762F900210220FFF75EF949E0B3
:10E14000D348844209D101210804FFF756F9002180
:10E150004FF48030FFF751F93CE0CE48844209D1BA
:10E1600001214804FFF749F900214FF40030FFF77F
:10E1700044F92FE0C848844209D101218804FFF7FF
:10E180003CF900214FF48020FFF737F922E0C34823
:10E19000844208D101214020FFF71EF900214020D0
:10E1A000FFF71AF916E0BE48844208D10121802009
:10E1B000FFF712F900218020FFF70EF90AE0B948B5
:10E1C000844207D101218015FFF706F90021A0152F
:10E1D000FFF702F910BD00220288A64B98420ED02C
:10E1E000AA4B98420BD0B0F1804F08D0A24B984276
:10E1F00005D0A24B984202D0A14B984203D122F005
:10E2000070024B881A439F4B984206D09E4B98420F
:10E2100003D022F440720B891A4302804B68C36218
:10E220000B880385934B984202D0984B984201D1BA
:10E230008B7A038601238382704730B50024002245
:10E240000023058C25F001050584028C8388048B4E
:10E2500024F0700424F003040D882C4322F0020201
:10E260008D892A434D882A43824DA84202D0874D8A
:10E27000A8420FD122F00802CD892A4322F00402DD
:10E280008D882A4323F4807323F400730D8A2B4373
:10E290004D8A2B43838004838D684563028430BD9F
:10E2A00070B5002400220023058C25F0100505849C
:10E2B000028C8388048B24F4E04424F440740D8899
:10E2C0004FF6FF7606EA05252C4322F020028D89C1
:10E2D00006EA05152A434D8806EA05152A43654DC9
:10E2E000A84202D0694DA84219D122F08002CD89FE
:10E2F0004FF6FF7606EA05152A4322F040028D8884
:10E3000006EA05152A4323F4806323F400630D8A8B
:10E3100006EA85052B434D8A06EA85052B43838053
:10E3200004838D688563028470BD70B5002400226B
:10E330000023058C25F480750584028C8388848BEA
:10E3400024F0700424F003040D882C4322F400729E
:10E350008D894FF6FF7606EA05252A434D8806EAA1
:10E3600005252A43434DA84202D0484DA84219D161
:10E3700022F40062CD894FF6FF7606EA05252A438E
:10E3800022F480628D8806EA05252A4323F480530F
:10E3900023F400530D8A06EA05152B434D8A06EA3D
:10E3A00005152B43838084838D68C563028470BD0B
:10E3B00070B5002200230024058C25F480550584C7
:10E3C000038C8488828B22F4E04222F440720D8810
:10E3D0004FF6FF7606EA05252A4323F400538D897C
:10E3E00006EA05352B434D8806EA05352B43214DBA
:10E3F000A84202D0254DA84207D124F480440D8ABA
:10E400004FF6FF7606EA85152C43848082838D685B
:10E410000564038470BD828B22F440628283828B08
:10E420004FF6FF7303EA01231A4382837047F0B566
:10E430000C461546002100220026078C27F4805741
:10E440000784818B028C4FF6FF7707EA043621F4AC
:10E45000734107EA052739434FF6FF7707EA033789
:10E46000394322F4204246F480573A4381830284A0
:10E47000F0BD000000000140000400400008004022
:10E48000000C004000100040001400400004014057
:10E490000040014000440140004801400018004095
:10E4A000001C004000200040828B22F00C0282837E
:10E4B000828B0A4382837047F0B50C4615460021D3
:10E4C00000220026078C27F480770784818B028C3A
:10E4D0004FF6FF7707EA042621F0F30107EA031756
:10E4E0002F43394322F4206246F480773A438183F4
:10E4F0000284F0BD028B22F440620283028B4FF64D
:10E50000FF7303EA01231A4302837047F0B50C46F8
:10E510001546002100220026078C27F010070784EB
:10E52000018B028C4FF6FF7707EA041621F4734142
:10E5300007EA033739434FF6FF7707EA05273943E0
:10E5400022F0A00246F010073A4301830284F0BD96
:10E55000028B22F00C020283028B0A430283704773
:10E5600070B50C46154600210022068C26F00106E7
:10E570000684018B028C21F0F3014FF6FF7606EA48
:10E5800003162E43314322F00A0244F001063243BF
:10E590000183028470BD70B505460C46208850B9D1
:10E5A0002389A28861882846FFF7DAFFE188284698
:10E5B000FFF7CEFF25E0208804280AD12389A2880E
:10E5C00061882846FFF7A2FFE1882846FFF792FFFF
:10E5D00017E0208808280AD12389A2886188284664
:10E5E000FFF76AFFE1882846FFF75EFF09E023890D
:10E5F000A28861882846FFF71AFFE1882846FFF7BE
:10E600000AFF70BD2DE9F04105460C4600260127A2
:10E61000608808B9022600E00026A088012801D100
:10E62000022700E001272088A0B92389A2886188F9
:10E630002846FFF795FFE1882846FFF789FF2389E1
:10E640003A4631462846FFF761FFE1882846FFF742
:10E6500051FF13E02389A28861882846FFF756FFFF
:10E66000E1882846FFF746FF23893A463146284687
:10E67000FFF776FFE1882846FFF76AFFBDE8F081E3
:10E680000A884B881A438B881A43CB881A430B8914
:10E690001A434B891A438B891A43A0F844207047C8
:10E6A0004FF0FF3141600021018001814180817282
:10E6B0007047002101804180818081608181C1811A
:10E6C00001824182704700210180418001218180C7
:10E6D0000021C1800181704700210180418081803B
:10E6E000C180018141818181704721B1028842F05E
:10E6F0000102028003E0028822F0010202807047DA
:10E7000031B1B0F8442042F40042A0F8442005E0C2
:10E71000B0F8442022F40042A0F8442070471AB117
:10E7200083890B43838102E083898B438381704714
:10E730008182704741EA0203A0F8483070471AB15D
:10E7400083890B43838102E083898B4383817047F4
:10E75000018921F00701018170470A4600210189E2
:10E7600021F0700111430181704730B504460D4618
:10E7700029462046FFF7F1FF208940F0070020815D
:10E7800030BD2DE9F04104460D4616461F46602D6A
:10E7900006D13B46012231462046FFF7B7FE05E091
:10E7A0003B46012231462046FFF7DAFE2946204645
:10E7B000FFF7D3FF208940F007002081BDE8F081FA
:10E7C00030B50C4600210189C9B24FF6FF7505EA44
:10E7D0000325154325432943018130BD2DE9F0412F
:10E7E00005460E4617469846002443463A463146AB
:10E7F0002846FFF7E5FF2C8924F0070444F00704BE
:10E8000024F0700444F070042C81BDE8F081F0B570
:10E8100004460D4616461F463B46324629462046CC
:10E82000FFF7CEFF208940F480402081F0BD0185B4
:10E83000828270470A460021018821F0700111434D
:10E8400001807047F0B50C4615461E460021002297
:10E8500000230189028B038C21F00701214340F240
:10E860000337BA4340F201173A4323F022034FF62D
:10E87000FF7707EA06172F433B4301810283038496
:10E88000F0BD0A460021018B21F070011143018384
:10E8900070470A460021018B21F4E0414FF6FF73D7
:10E8A00003EA02231943018370470A460021818B42
:10E8B00021F070011143818370470A460021818B4A
:10E8C00021F4E0414FF6FF7303EA022319438183E9
:10E8D000704721B1028842F08002028003E0028882
:10E8E00022F080020280704721B1828842F0040247
:10E8F000828003E0828822F004028280704721B186
:10E90000828842F00802828003E0828822F00802B6
:10E910008280704721B1828842F00102828003E048
:10E92000828822F00102828070470A460021018B12
:10E9300021F008011143018370470A460021018B31
:10E9400021F400614FF6FF7303EA022319430183A8
:10E9500070470A460021818B21F008011143818311
:10E9600070470A460021818B21F400614FF6FF7346
:10E9700003EA02231943818370470A460021018B71
:10E9800021F004011143018370470A460021018BE5
:10E9900021F480614FF6FF7303EA022319430183D8
:10E9A00070470A460021818B21F0040111438183C5
:10E9B00070470A460021818B21F480614FF6FF7376
:10E9C00003EA02231943818370470A460021018B21
:10E9D00021F080011143018370470A460021018B19
:10E9E00021F400414FF6FF7303EA02231943018328
:10E9F00070470A460021818B21F0800111438183F9
:10EA000070470A460021818B21F400414FF6FF73C5
:10EA100003EA02231943818370470A460021018CCF
:10EA200021F002011143018470470A460021018C44
:10EA300021F008011143018470470A460021018C2E
:10EA400021F020014FF6FF7303EA021319430184FA
:10EA500070470A460021018C21F080014FF6FF73B8
:10EA600003EA02131943018470470A460021018C0E
:10EA700021F400714FF6FF7303EA02231943018466
:10EA800070470A460021018C21F400614FF6FF73A4
:10EA900003EA02231943018470470A460021018CCE
:10EAA00021F400514FF6FF7303EA02331943018446
:10EAB000704730B5002301248C40A3B2048C9C43E2
:10EAC0000484048C02FA01F5ADB22C43048430BDF9
:10EAD00030B5002304248C40A3B2048C9C430484EE
:10EAE000048C02FA01F5ADB22C43048430BD70B53C
:10EAF0000346002000241846183001258D40ACB292
:10EB00001D8CA5431D8409B108290AD100EB6100C1
:10EB100005684FF68F76354005600568154305603A
:10EB20000FE00D1FC5F34E052844056848F6FF7633
:10EB30003540056005684FF6FF7606EA0226354344
:10EB4000056070BD21B1028842F00202028003E03C
:10EB5000028822F002020280704721B1028842F04E
:10EB60000402028003E0028822F00402028070475F
:10EB700021B1828842F08002828003E0828822F004
:10EB8000800282807047028822F008020280028898
:10EB90000A4302807047828822F070028280828855
:10EBA0000A4382807047028922F0070202810289AB
:10EBB0000A4302817047028922F0800202810289A1
:10EBC0000A430281704741627047C16270474163E6
:10EBD000704781637047C163704701647047028862
:10EBE00022F44072028002880A4302807047014684
:10EBF000486B70470146886B70470146C86B704789
:10EC00000146086C70470146486A70470146088D06
:10EC10007047A0F85010704702460020138A0B403E
:10EC20000BB1012000E000207047CA430282704708
:10EC300030B50246002000230024158A05EA0103AE
:10EC4000958905EA010413B10CB1012000E0002010
:10EC500030BDCA43028270470CB50020019000907D
:10EC60006B48006840F480306949086000BF68481C
:10EC7000006800F4003000900198401C019000985A
:10EC800018B90198B0F5A06FF1D16148006800F49F
:10EC9000003010B10120009001E0002000900098A9
:10ECA000012838D15A4808300068594908310860AD
:10ECB0000846006840F4004008600846006840F4D8
:10ECC000A05008605348091F0860081F006840F002
:10ECD0008070091F086000BF4D48006800F0007098
:10ECE0000028F9D040F204704B49086048480830C9
:10ECF000006820F0030046490831086008460068B3
:10ED000040F00200086000BF41480830006800F091
:10ED10000C000828F8D10CBD10B53D48006840F043
:10ED200001003B4908600020394908310860384833
:10ED300000683A490840364908603948091D0860AA
:10ED4000081F006820F48020091F08600020304957
:10ED50000C310860FFF780FF32483349086010BD6E
:10ED600070B500200022022300240221284D08351E
:10ED70002D6805F00C0020B1042806D0082834D1F5
:10ED800007E02A4D2A4E356033E02A4D284E356083
:10ED90002FE01F4D2D1D2D68C5F380541C4D2D1DDA
:10EDA0002D6805F03F0154B1224DB5FBF1F5184E29
:10EDB000361D3668C6F3881605FB06F209E01B4DC2
:10EDC000B5FBF1F5124E361D3668C6F3881605FB05
:10EDD00006F20F4D2D1D2D68C5F301456D1C6B000E
:10EDE000B2FBF3F5124E356003E0104D104E356066
:10EDF00000BF00BF064D08352D68C5F303150E4E44
:10EE0000705D0B4D2D68C540094E356070BD00002A
:10EE100000380240193C4005003C0240FFFFF6FE6E
:10EE20001030002400000C0808ED00E00024F4007D
:10EE30004401002040787D0148010020016821F054
:10EE4000010101600021016041608160C1600161D8
:10EE500021214161DC49884204D13D21DA4A103A3E
:10EE600091608CE0D8491831884205D14FF4746123
:10EE7000D54A103A916082E0D3493031884205D1B9
:10EE80004FF47411D04A103A916078E0CE4948317D
:10EE9000884205D14FF07461CB4A103A91606EE020
:10EEA000C9496031884204D1C849C74A103AD16083
:10EEB00065E0C5497831884204D1C549C24A103A53
:10EEC000D1605CE0C0499031884204D1C149BE4A5A
:10EED000103AD16053E0BC49A831884205D14FF0C7
:10EEE0003D51B94A103AD16049E0BB49884204D14A
:10EEF0003D21B94A083A116041E0B74918318842CA
:10EF000005D14FF47461B44A083A116037E0B24950
:10EF10003031884205D14FF47411AF4A083A11607C
:10EF20002DE0AD494831884205D14FF07461AA4ABD
:10EF3000083A116023E0A8496031884204D1A3490E
:10EF4000A54A121F11601AE0A3497831884204D102
:10EF50009F49A14A121F116011E09F4990318842D8
:10EF600004D19C499C4A121F116008E09A49A831BB
:10EF7000884204D14FF03D51974A121F11607047EB
:10EF800010B500220268954B1A40CC680B682343E9
:10EF90004C6923438C692343CC6923430C6A234384
:10EFA0004C6A23438C6A23434C6B23438C6B23436F
:10EFB0001A430260426922F00702D1E90B3423436D
:10EFC0001A4342610B6943604B6883608B68C3607E
:10EFD00010BD0021016041608160C160016141613B
:10EFE0008161C1610162416281620421C1620021CB
:10EFF000016341638163704721B1026842F00102FD
:10F00000026003E0026822F00102026070470146DC
:10F0100000200A6802F001020AB1012000E000208D
:10F02000704710B501F080034BB122B1436943F042
:10F030008003436103E0436923F080034361802937
:10F040000BD02AB1036801F01E042343036004E0DF
:10F05000036801F01E04A343036010BD0146486825
:10F0600080B2704741607047014600204A6902F053
:10F070003800704721B1026842F02002026003E0CC
:10F08000026822F020020260704721B1026842F457
:10F090000042026003E0026822F40042026070470E
:10F0A00022B1036843F40023036003E0036823F400
:10F0B000002303600161704721B1026842F480229D
:10F0C000026003E0026822F48022026070470AB105
:10F0D000016100E0C1607047014600200A6802F447
:10F0E00000220AB1012000E00020704730B503463D
:10F0F0000A4600200024384DAB4202D23249103972
:10F1000001E03549103902F000550DB14C6800E0BE
:10F110000C68334D2C4004EA02050DB1012000E0DB
:10F12000002030BD02462C4B9A4202D226481038AD
:10F1300001E02948103801F000531BB1284B0B4067
:10F14000C36002E0264B0B408360704770B50246F7
:10F15000002000240025204EB24202D21A4B103B60
:10F1600001E01D4B103B1F4E0E4036B11E2606EA35
:10F17000D124166806EA040502E0566906F0800507
:10F1800001F000560EB15C6800E01C68144E34407B
:10F1900004EA010616B10DB1012000E0002070BDA7
:10F1A00002460D4B9A4202D20748103801E00A4845
:10F1B000103801F000531BB1094B0B40C36002E053
:10F1C000074B0B4083607047106002403D000020F9
:10F1D000400F002000003D20106402403F801CF0E2
:10F1E0007D0F7D0F3C0F3C0F10B501210802FEF78B
:10F1F00004F900214FF48070FEF7FFF810BD0021E4
:10F20000FA4A1168FA4A1140D0E900231A43836888
:10F210001A43C3681A431143F64AC2F804137047ED
:10F2200030B50246002000235068F34C20400D7991
:10F230000C6844EA0524204350609068EF4C20405D
:10F24000D1E903542C438D682C434D7944EA45049D
:10F2500020439060D06A20F470000C7D641EE4B2FC
:10F26000234340EA0350D06230BD00210160416079
:10F270008160C1607047002101600171417181604E
:10F28000C160016101210175704721B1826842F0BE
:10F290000102826003E0826822F00102826070470E
:10F2A00021B1826842F48072826003E0826822F4B5
:10F2B00080728260704710B50B460021D9B20124DC
:10F2C00004FA01F11AB144680C43446002E0446856
:10F2D0008C43446010BD816841F08041816070477B
:10F2E000014600208A6802F480020AB1012000E091
:10F2F0000020704721B1826842F00202826003E080
:10F30000826822F002028260704721B1826842F472
:10F310008062826003E0826822F4806282607047CB
:10F3200021B1826842F40072826003E0826822F4B4
:10F3300000728260704739B1AC4A126842F40052E0
:10F34000AC4BC3F8042306E0A84A126822F400522A
:10F35000A84BC3F80423704710B50A4600210023C8
:10F36000416821F46041531E41EA4331416010BDC0
:10F3700021B1426842F40062426003E0426822F434
:10F38000006242607047F0B504460D46002000213F
:10F39000092D11DDE068A5F10A0606EB46070726F0
:10F3A00006FA07F18843A5F10A0606EB460603FABA
:10F3B00006F10843E0600CE0206905EB45070726ED
:10F3C00006FA07F1884305EB450603FA06F1084300
:10F3D0002061072A0FDA606B561E06EB86071F2690
:10F3E00006FA07F18843561E06EB860605FA06F173
:10F3F0000843606322E00D2A0FDA206BD61F06EB6C
:10F4000086071F2606FA07F18843D61F06EB8606F5
:10F4100005FA06F10843206310E0E06AA2F10D0648
:10F4200006EB86071F2606FA07F18843A2F10D06B0
:10F4300006EB860605FA06F10843E062F0BD0146D8
:10F44000C86C80B270476948001D0068704721B1E0
:10F45000426842F48062426003E0426822F48062C3
:10F460004260704721B1426842F48052426003E03A
:10F47000426822F48052426070470A460021816847
:10F4800021F470211143816070470A460021816890
:10F4900021F44011114381607047816841F480017B
:10F4A00081607047014600208A6802F480020AB138
:10F4B000012000E000207047F0B50446154600200A
:10F4C00000220026092911DDE068A1F10A0707EBF7
:10F4D000470C072707FA0CF29043A1F10A0707EB44
:10F4E000470703FA07F21043E0600CE0206901EBE4
:10F4F000410C072707FA0CF2904301EB410703FA8E
:10F5000007F210432061A06BC0F30156EF1C06F117
:10F51000010CA7EB0C0707EB870C1F2707FA0CF26F
:10F520009043EF1C06F1010CA7EB0C0707EB8707D4
:10F5300001FA07F21043A063F0BD10B50A4600219E
:10F540000023816B21F44011531E41EA0351816372
:10F5500010BD08B5002300930090009B0B4400935E
:10F56000009B1A6008BD08B502460020009000927A
:10F5700001F12800009B184400900098006880B2B8
:10F5800008BD0A46002141681D4B194011434160E6
:10F5900070474162826270470A460021416821F04B
:10F5A0001F0111434160704738B11049096841F4A7
:10F5B0000001104AC2F8041306E00C49096821F45E
:10F5C00000010C4AC2F80413704738B107490968B2
:10F5D00041F48001074AC2F8041306E003490968B0
:10F5E00021F48001034AC2F8041370470423014048
:10F5F000E030FCFF00200140FFFEFFFCFDF7FFC0F4
:10F60000FFFD3FFF0246002013680B400BB10120B5
:10F6100000E000207047CA430260704770B50246A0
:10F620000020002300240B12556801268E4005EAB5
:10F63000060415681D4015B10CB1012000E0002042
:10F6400070BD00220A12D3430360704710B5044610
:10F65000FD48844209D101214806FDF7BDFE002185
:10F660004FF00070FDF7B8FE08E001218806FDF7B5
:10F67000B3FE00214FF08060FDF7AEFE10BD30B547
:10F68000024600200023146824F002041460146869
:10F6900044F00104146000E05B1C546804F00104B1
:10F6A0001CB94FF6FF74A342F6D1546804F001046C
:10F6B0000CB900206CE08C79012C04D1146844F062
:10F6C0008004146003E0146824F080041460CC7992
:10F6D000012C04D1146844F04004146003E0146861
:10F6E00024F0400414600C7A012C04D1146844F016
:10F6F0002004146003E0146824F0200414604C7AA1
:10F70000012C04D1146844F01004146003E0146860
:10F7100024F0100414608C7A012C04D1146844F095
:10F720000804146003E0146824F008041460CC7A20
:10F73000012C04D1146844F00404146003E014683C
:10F7400024F0040414608C78A407CD7844EA05649E
:10F750000D7944EA05444D7944EA05540D886D1E3F
:10F760002C43D461146824F001041460002300E0E9
:10F770005B1C546804F001041CB14FF6FF74A342F3
:10F78000F6D1546804F001040CB1002000E001201F
:10F7900030BD10B50021837A012202FA03F1AB4A91
:10F7A000126842F00102A94B1A60A84A1C32126882
:10F7B0008A43A64B1C331A60027BCAB9A34A0C3297
:10F7C00012688A43A14B0C331A604288C38842EA0C
:10F7D00003439E4A4032847A42F834300288838858
:10F7E00042EA0343994A4032847A02EBC4025360EE
:10F7F000027B012A19D1954A0C3212680A43934BB5
:10F800000C331A604288038842EA03438F4A40322D
:10F81000847A42F83430C288838842EA03438B4AB0
:10F820004032847A02EBC4025360C27A3AB9874A02
:10F83000121D12688A43854B1B1D1A6006E0834A1D
:10F84000121D12680A43814B1B1D1A60028932B9CE
:10F850007E4A143212688A437C4B14331A60028940
:10F86000012A06D1794A143212680A43774B1433BD
:10F870001A60427B012A06D1744A1C3212680A437C
:10F88000724B1C331A60714A126822F001026F4BEE
:10F890001A6010BD00218171C171017241728172C3
:10F8A000C1728170C1700321017102214171012176
:10F8B000018070476549096841F00101634A1160A0
:10F8C0001146096843F60E729143604A1160114671
:10F8D000096841EA002111601146096821F001011F
:10F8E000116070471AB143690B43436102E04369F9
:10F8F0008B434361704710B502460020936803F0C4
:10F900008063B3F1806F00D110E0936803F000636F
:10F91000B3F1006F01D1012008E0936803F0805338
:10F92000B3F1805F01D1022000E00420042874D0EC
:10F9300002F5C07303EB00131B6803F0010402F52A
:10F94000C07303EB00131C600B7A7BB94B7A0C88F5
:10F9500043EA445302F5C07404EB001424682343C3
:10F9600002F5C07404EB0014236010E00B7A4C68BD
:10F9700043EAC4034C7A234302F5C07404EB001439
:10F980002468234302F5C07404EB001423608B7ACF
:10F9900003F00F038B7202F5C07303EB00135B6877
:10F9A00023F00F0402F5C07303EB00135C6002F553
:10F9B000C07303EB00135B688C7A234302F5C074B9
:10F9C00004EB001463608B7B1C064B7B44EA03440E
:10F9D0000B7B44EA0323CC7A234302F5C07404EB87
:10F9E0000014A3608B7C1C064B7C44EA03440B7C14
:10F9F00044EA0323CC7B234302F5C07404EB0014D8
:10FA0000E36002F5C07303EB00131B6843F00104CD
:10FA100002F5C07303EB00131C6010BD024600200A
:10FA200021B1012914D0022930D120E0936803F0DC
:10FA3000010340EA8300936803F0020318439368CC
:10FA4000C3F38063184323E0006400400066004075
:10FA5000936803F4807340EA9310936803F400738F
:10FA600040EA13209368C3F3C063184310E093681F
:10FA700003F4803340EA9330936803F4003340EAA0
:10FA800013409368C3F30073184301E0002000BFE4
:10FA900000BF20B1052804D0072806D103E00220CA
:10FAA00005E0002003E0012001E0002000BF00BFCE
:10FAB000704721B1012907D002290FD109E08268DE
:10FAC00042F0800282600AE0826842F40042826072
:10FAD00005E0826842F40002826000E000BF00BFDF
:10FAE000704721B9C26842F02002C26003E0026997
:10FAF00042F02002026170470246002019B9D36823
:10FB000003F0030006E0012903D1136903F00300A9
:10FB100000E00020704730B505460C46134605F559
:10FB2000D87000EB0410006800F004001872187A16
:10FB300050B905F5D87000EB0410006840F2FF7171
:10FB400001EA5050186009E005F5D87000EB041088
:10FB500000686FF0604101EAD000586005F5D87088
:10FB600000EB0410006800F00200587205F5D87030
:10FB700000EB0410406800F00F00987205F5D87093
:10FB800000EB04104068000AD87405F5D87000EB4B
:10FB900004108068D87205F5D87000EB04108068F6
:10FBA000010A197305F5D87000EB04108068010C88
:10FBB000597305F5D87000EB04108068000E987337
:10FBC00005F5D87000EB0410C068D87305F5D8703F
:10FBD00000EB0410C068010A197405F5D87000EB39
:10FBE0000410C068010C597405F5D87000EB0410BE
:10FBF000C068000E987421462846FFF772FF30BD9A
:10FC000021B1026842F48032026003E0026822F40B
:10FC1000803202607047014600200A6822F001022B
:10FC200042F002020A604A6802F00302022A00D18E
:10FC30000120704701464FF6FF7200200B6823F049
:10FC400002030B6000E0521E4B6803F00203022B1C
:10FC500001D1002AF7D14B6803F00203022B00D038
:10FC60000120704710B50246002001F4700343B133
:10FC70009369C1F3130423400BB101202DE0002050
:10FC80002BE001F0807343B15368C1F313042340A8
:10FC90000BB1012021E000201FE001F0006343B11F
:10FCA0009368C1F3130423400BB1012015E0002039
:10FCB00013E001F0007343B1D368C1F31304234090
:10FCC0000BB1012009E0002007E01369C1F3130420
:10FCD00023400BB1012000E0002010BD0022834B27
:10FCE000994202D10023836111E0C1F3130201F0B4
:10FCF00000730BB1C2600AE001F080630BB10261D6
:10FD000005E001F000630BB1826000E042607047E3
:10FD10000246002002EA01030BB1012000E00020AE
:10FD2000704770B504460D460026606928400028DB
:10FD300071D0B5F5807F5CD010DC082D35D006DCA5
:10FD4000012D20D0022D24D0042D77D127E0102DB5
:10FD500031D0202D35D0402D70D138E0B5F5004F91
:10FD600060D009DCB5F5007F49D0B5F5806F4CD087
:10FD7000B5F5006F62D14FE0B5F5803F2DD0B5F5F8
:10FD8000003F5BD12FE0A0685949FFF7C1FF06464D
:10FD900056E0E0680321FFF7BBFF064650E0E0684D
:10FDA0000821FFF7B5FF06464AE0E0681021FFF79B
:10FDB000AFFF064644E020690321FFF7A9FF06468E
:10FDC0003EE020690821FFF7A3FF064638E02069DE
:10FDD0001021FFF79DFF064632E060680821FFF71B
:10FDE00097FF06462CE060681021FFF791FF06465A
:10FDF00026E0A0690121FFF78BFF064620E0A069FD
:10FE00000221FFF785FF06461AE0A0690421FFF7EB
:10FE10007FFF064614E014E0A0697021FFF778FF29
:10FE200006460DE0A0697721FFF772FF064660687D
:10FE30000421FFF76DFF064302E0FFE7002600BF45
:10FE400000E00026304670BDB1F5007F3AD00FDCEF
:10FE5000202928D006DC01291CD004291DD008291E
:10FE600040D11DE0402921D0B1F5807F3AD126E074
:10FE7000B1F5004F31D006DCB1F5806F25D0B1F57A
:10FE8000006F2FD124E0B1F5803F12D0B1F5003FD3
:10FE900028D111E0164A826025E00822C26022E0E3
:10FEA0001022C2601FE0082202611CE010220261E1
:10FEB00019E00822426016E01022426013E004229A
:10FEC000426010E0042242600DE0042242600AE039
:10FED000002282610422426005E000228261042245
:10FEE000426000E000BF00BF704700007000F030CB
:10FEF00001010100002044490860091D0860091D36
:10FF00000860091D086041483F4914310860704786
:10FF100000213D498279002A3AD00A4612680368D6
:10FF20009A430B461A600A1D126803689A430B1D18
:10FF30001A60027911440A6803681A430A60324A57
:10FF40000832126803689A432F4B08331A601A1D4F
:10FF5000126803689A432C4B0C331A604279102ABA
:10FF60000ED11A1F126803681A43274B08331A6010
:10FF70001A1D126803681A43234B0C331A600DE0F4
:10FF80002149427911440A6803681A430A6005E06E
:10FF9000027911440A6803689A430A607047002195
:10FFA000016001710C214171002181717047164976
:10FFB000103109680143144A10321160704701463C
:10FFC0000020114A143212680A400AB1012000E0F0
:10FFD000002070470C49143108607047014600202A
:10FFE0000022094B1B6803EA0102074B14331B680C
:10FFF0000B4013B10AB1012000E000207047024914
:02000004080DE5
:100000001431086070470000003C0140FFFF1F00F2
:1000100010B501218803FDF7F0F900214FF480406D
:10002000FDF7EBF910BD13490860704730B50022A9
:100030008B071C0F0F2303FA04F20E4B08338C10AE
:1000400053F8243093430B4C08348D1044F825307A
:1000500023468C1053F824308C07240F00FA04F444
:100060002343044C08348D1044F8253030BD024938
:100070000860704700380140DC0027420E490860E4
:1000800070470D49486070470B49886070474AF6D1
:10009000AA200949086070474CF6CC400649086020
:1000A000704701460020044AD2680A400AB1012084
:1000B00000E000207047000000300040032A40F2BA
:1000C000308010F0030C00F0158011F8013BBCF1FA
:1000D000020F624498BF11F801CB00F8013B38BF12
:1000E00011F8013BA2F1040298BF00F801CB38BF20
:1000F00000F8013B11F0030300F06780083AC0F0FC
:10010000088051F8043B083A51F804CBA0E80810E5
:10011000F5E7121D5CBF51F8043B40F8043BAFF318
:100120000080D20724BF11F8013B11F801CB48BF72
:1001300011F8012B24BF00F8013B00F801CB48BFA8
:1001400000F8012B7047431A28BF9A427FF6B6AFDA
:10015000032A1044114440F2268010F0030F1EBF02
:1001600011F8013D521E00F8013D10F0030F7FF41D
:10017000F6AF11F0030300F07080083AC0F00B8076
:1001800051F8043D083A51F804CD40F8043D40F8D8
:1001900004CDFFF7F3BF121D5CBF51F8043D40F8DA
:1001A000043DAFF30080D20724BF11F8013D11F8E0
:1001B00001CD48BF11F8012C24BF00F8013D00F823
:1001C00001CD48BF00F8012C704710B5203AC0F0AF
:1001D0000B80B1E81850203AA0E81850B1E8185048
:1001E000A0E81850BFF4F5AF5FEA027C24BFB1E885
:1001F0001850A0E8185044BF18C918C0BDE81040F6
:100200005FEA827C24BF51F8043B40F8043B08BFFE
:100210007047D20728BF31F8023B48BF11F8012BC5
:1002200028BF20F8023B48BF00F8012B70477047F9
:1002300070477047431A28BF9A427FF6C6AF1044F2
:1002400010F0030F11441EBF11F8013D521E00F8BB
:10025000013D10F0030F7FF4F6AF103AC0F00A80B2
:1002600010B531E91850103A20E91850BFF4F9AF31
:10027000BDE81040530724BF31E9081020E90810F9
:1002800044BF51F8043D40F8043D12F0030F08BF8D
:100290007047D20728BF31F8023D48BF11F8012C42
:1002A00028BF20F8023D48BF00F8012C7047754672
:1002B00000F028F8AE4605006946534620F00700D6
:1002C000854618B020B5FCF765FEBDE820404FF02C
:1002D00000064FF000074FF000084FF0000B21F030
:1002E0000701AC46ACE8C009ACE8C009ACE8C009FD
:1002F000ACE8C0098D4670470446AFF30080204645
:10030000EFF797FF00487047EC6A0020014918207A
:10031000ABBEFEE72600020070474344502B5F65EA
:100320004F4244000378FF1F0078FF1F0278FF1F31
:100330000178FF1F007AFF1F504300004344500024
:1003400045585400444932004A564300013E003E9D
:10035000000000000102030401020304060708096B
:1003600080030D080000002058010000C0010C08A7
:1003700094030D0858010020F86F0000FC010C08E0
:1003800001D1027512940E27071901020304060712
:040390000809000058
:02000004080FE3
:04FF00007500000088
:02000004080FE3
:04FF04007500000084
:04000005080C01855D
:00000001FF
